:1000000000800020BD01000055CF00000DCF000092
:100010000DCF00000DCF00000DCF00000DCF000070
:100020000DCF00000DCF00000DCF000055CF000018
:1000300055CF00000DCF0000D5C50000D9C6000087
:1000400055CF000055CF000055CF000055CF000020
:1000500055CF000055CF000055CF000055CF000010
:1000600055CF000055CF000055CF000055CF000000
:1000700055CF000055CF000055CF000055CF0000F0
:1000800055CF000055CF000055CF000055CF0000E0
:1000900055CF000055CF000055CF000055CF0000D0
:1000A00011AB00001DAB000055CF000055CF000084
:1000B00055CF000055CF000055CF000055CF0000B0
:1000C00055CF000055CF000055CF000055CF0000A0
:1000D00055CF000055CF000055CF000055CF000090
:1000E00055CF000055CF000055CF000055CF000080
:1000F00055CF0000C1EF000055CF0000EDF000002B
:1001000055CF00002DD9000055CF000055CF00007D
:1001100055CF000055CF000055CF000055CF00004F
:1001200055CF000055CF000055CF000055CF00003F
:1001300055CF000055CF000055CF000055CF00002F
:1001400055CF000055CF000055CF000055CF00001F
:10015000C5C70000D9C70000EDC7000001C80000F6
:1001600055CF000049DC000055CF000055CF0000FE
:1001700055CF000055CF000055CF000055CF0000EF
:1001800055CF000055CF000055CF000055CF0000DF
:1001900055CF000055CF000055CF000055CF0000CF
:1001A00055CF000055CF000055CF000055CF0000BF
:1001B00055CF000055CF000055CF0000564B4CF2F4
:1001C000205210B51A804DF628121A8000BF00BFC9
:1001D0000CF0C4FE514B4FF010621A60504A9A6006
:1001E000504ADA60504A136813F4807304D14F49BF
:1001F0000B604FF4A85313604D4B1A78110703D5C9
:100200001A7842F008021A704A4B4B492A221A7097
:100210004A4A4B4B8B4204D252F8040F43F8040B6A
:10022000F8E7484B484900228B4202D243F8042B9E
:10023000FAE74649464A002352F8230041F82300D2
:1002400001336F2BF8D1434B434A802103F8011B44
:100250009342FBD1414B3D4A1A60414B8A221A70AE
:10026000A3F5805324225A70A0221A709A7992071B
:10027000FCD59A79D406FCD43A4A937903F00C035E
:10028000082B384BF9D103221A7140225A719A79FE
:100290009006FCD5334A9179324B4906FBD5324A58
:1002A000324911600221516020221A709A7902F0BD
:1002B0000C020C2AFAD12E4B2E4A1A602E4B2F4AD2
:1002C0001A6000225A60072243F8042C2C4AC3F813
:1002D0000C2D62B60DF0F2F9144B1B68DA0705D548
:1002E00028480CF0BFFF284B284A1A60284B1B787F
:1002F0005B0609D5244C254B22689A4204D121483B
:100300000CF0B0FF0023236010F0AAF90CF02CFED3
:100310000CF05AFDFEE700BF0E200540308004407F
:10032000823F04000100002B10D0034014D0034092
:1003300002D0074000E007405C9BFF1F4C3F0100DC
:100340004088FF1F5C9BFF1F54A3FF1F0082FF1FFD
:100350000000000000E400E05FE400E008ED00E0E1
:100360000050064000400640448004400000030165
:1003700004800440C010050014E000E0FF76010096
:10038000000020208F763F5F1CE00340A5C3945AF5
:1003900000F00740FFFFFFFFFFFFFFFFFFFFFFFF32
:1003A000FFFFFFFFFFFFFFFFFFFFFFFFFFFFFFFF5D
:1003B000FFFFFFFFFFFFFFFFFFFFFFFFFFFFFFFF4D
:1003C000FFFFFFFFFFFFFFFFFFFFFFFFFFFFFFFF3D
:1003D000FFFFFFFFFFFFFFFFFFFFFFFFFFFFFFFF2D
:1003E000FFFFFFFFFFFFFFFFFFFFFFFFFFFFFFFF1D
:1003F000FFFFFFFFFFFFFFFFFFFFFFFFFFFFFFFF0D
:10040000FFFFFFFFFFFFFFFFFFFFFFFFDEF9FFFF23
:1004100010B5054C237833B9044B13B10448AFF33E
:1004200000800123237010BD5C9BFF1F00000000B3
:10043000503F0100084B10B51BB108490848AFF305
:1004400000800848036803B910BD074B002BFBD0A0
:10045000BDE81040184700BF00000000609BFF1F70
:10046000503F01005C9BFF1F0000000038B50446B0
:10047000104621700A491D460FF0D4FE01464FF088
:100480007E500FF083FF07490FF0CCFEE5606060FF
:10049000256165610DF0A2F8E061204638BD00BF1E
:1004A000DB0FC9400024744938B50446104621705A
:1004B00009491D460FF0B6FE01464FF07E500FF081
:1004C00065FF06490FF0AEFEE5606060256165617D
:1004D0000DF084F8E06138BDDB0FC9400024744999
:1004E00038B503780446032B20D8DFE803F01A1848
:1004F0001002C16840690FF08BFD0D490546606828
:100500000FF044FF014628460FF040FF38BD084970
:1005100040680FF03BFFE1680FF084FE38BDC06813
:1005200038BDC16840690FF073FD38BD002038BD8B
:100530000024744970B504460E460DF04FF8054688
:10054000E069281A0FF01AFEE3682361E56166612D
:10055000A061014660680FF019FF0146A0601048D5
:100560000FF014FF0FF0EAF90EF08AFE0FF0FCFC1A
:10057000054601464FF07E500FF04AFD61690FF0CD
:1005800051FE2169064628460FF04CFE01463046D2
:100590000FF040FDE0602046BDE87040FFF7A0BFCF
:1005A000000080BF08B50E200CF0E8FA114B1B8844
:1005B000012B19D0104B1B88984213DB40F6FF71BA
:1005C0008842D4BFC3EB0001C3EB0101C1EB013191
:1005D000C3F57F630F33282091FBF3F1BDE808409A
:1005E0000CF052BE0021F3E70146BDE8084014209C
:1005F0000CF04ABE949DFF1F2C9CFF1F10B50446B3
:100600000CF0BEF8204610BD70B44C88A04220D932
:1006100001230133DBB21CB2660031F8144084427E
:100620001D46F6D3A04211D005F10045013D965B71
:1006300031F8151032F81530401AF21A00FB02F0AA
:10064000641A90FBF4F4E01870BC7047905B70BCC7
:10065000704702260125E5E700280CDA064A4342E6
:1006600082FB0320DA17C2EB600000EB4000A3EB33
:100670008000C0F10C007047ABAAAA2AF0B40E8823
:1006800086420DD203F10043013B31F813508542FD
:1006900002D9F0BCFFF7B8BF32F81300F0BC7047C6
:1006A0001088F0BC704700BF094B1B880C2B09D881
:1006B000084A80B252F8232028B143F6FE739842CC
:1006C00003D9108C7047108870470349FFF79CBF0F
:1006D000B29BFF1FD0190100141C01004B4B4C4A68
:1006E0002DE9F0471E8814684A4BB442B3F80080E5
:1006F000494B33DB4445A8BF4446A6421C60C8BFF3
:1007000000202DDDC6EB0807B7F5804F33DB8003F3
:100710007B1C90FBF3F0FFF7C7FF404A404B158866
:100720001B88C0F3C61909FB05F57F2D8246A8BFBB
:100730007F252BB3A64253DC4445D4BFC6EB04044B
:10074000C6EB08049F42CCBF03FB04445C43354B1B
:10075000C8BF013794FBF7F71F6013E034461E60F3
:10076000C6EB0807A045D4BFC6EB0800C6EB0400E3
:10077000B7F5804FCBDAC0EB803090FBF7F0CAE7DB
:10078000284A1360284C2368994508D0274B1B88BA
:10079000002B34D1264B1B886BBBC4F80090254C32
:1007A00023689A4506D0214B1B885A1F032A19D962
:1007B000C4F800A0204C23689D420FD01F4B18881E
:1007C00048B11A4B1E4A1B88D35C834203D0C0B287
:1007D000E9B208F0C7FA2560BDE8F087BDE8F08708
:1007E0000024AFE7164AD05C2030C0B20AF07F0187
:1007F00008F0B8FADCE7484608F028FBCDE7104AD5
:100800004946D05C08F0AEFAC4E700BF2C9CFF1F3D
:10081000909DFF1FE89DFF1F809BFF1F949BFF1F64
:10082000969BFF1FF09DFF1FE09BFF1F769DFF1F04
:10083000229CFF1FAC9BFF1F249CFF1F869DFF1F58
:100840009889FF1F2DE9F04F172089B00DF0DAF8D5
:10085000AF4B186016200DF0D5F8AE4BAE4A1B8892
:1008600010600C2B00F03B81AC4BAD4A1988009313
:10087000AC4B52F8214000221A70AB4BAB4D1B8899
:10088000AB4A2E88013B32F91370002E5CD0A94B85
:10089000A94A1B88A9491278013B31F91380002A23
:1008A00040F0DF8011200DF0ADF8A54B0193D3F897
:1008B00000A00646B24540F3DF80A24BDFF8A492C9
:1008C0001B88A14A012BD9F80030B2F800B09F4A2A
:1008D00002922046C8EB030800F09A820FF04EFC0B
:1008E000029A52F82B100FF09DFC014600200FF0E9
:1008F0008FFB0FF05DFECAEB0802B045B8BFB046F3
:100900009042CAEB080880F2968200FB0888013208
:1009100098FBF2F08E4BDFF850820293D8F800304B
:10092000034403EBD3735B10C8F800302B88012B12
:1009300012D1884BDFF834B20393874BDBF80050B9
:1009400004934FF0000A47E07D4B0193DFF81492C7
:100950007F4BDFF8148202937E4B03931D460F20DA
:100960000DF050F82B689842824641DA754A128899
:10097000012A00F01D82744A05931288734D049277
:1009800020460FF0FBFB049ADFF8E0B155F8221087
:10099000DBF800500FF046FC014600200FF038FB5A
:1009A0000FF006FEEF1B059B5745A7EB0302B8BFF0
:1009B0005746FF1A9042BABF013200FB0777474300
:1009C00097FBF2F7D8F80020634B0493BB1803EBB6
:1009D000D3735B10C8F80030604B1B88013B032BBE
:1009E00000F2B082DFE813F06301A901C4008601C0
:1009F000594B04931B68984240F3C281514A1288B4
:100A0000012A00F0A682504A079311884F4A0691A6
:100A1000204605920FF0B2FB059A0699DFF84CB11B
:100A200052F82110DBF800500FF0FCFB0FF0C0FD76
:100A3000079B2F445745A7EB0302A8BF5746FF1A51
:100A4000D8F800309042BABF00FB07770132474325
:100A500097FBF2F73B4403EBD3735B10C8F800300D
:100A6000BAE715200CF08AF8354B0193D3F800A0B3
:100A70000646B2453FF721AF354B0293D3F800A0AD
:100A8000B24580F289812F4BDFF8D8901B882E4A1F
:100A9000012BD9F80030B2F800B02C4A039220465E
:100AA000984400F070820FF069FB039A52F82B1003
:100AB0000FF0B8FB0FF07CFDB045CAEB0802A8BFF1
:100AC000B046CAEB08089042B6BF00FB088800FB9E
:100AD00008F8013298FBF2F0DFF88C801EE7204B1B
:100AE0001B78002B3FF4C0AE0C4B0D4A19880093C5
:100AF0000C4B52F8210001221A700FF03FFB4FF00F
:100B00007C510FF08FFB0FF053FD0446B5E600BF9C
:100B1000D89BFF1FC29DFF1F0C9EFF1FDC9BFF1F6A
:100B20005889FF1F8A9BFF1F2089FF1F309DFF1FD1
:100B3000D81D0100A889FF1FA69DFF1FCC1B010027
:100B4000109EFF1F109CFF1FCC9BFF1FF01D01007C
:100B5000049CFF1FB49DFF1F289DFF1F2E89FF1FB0
:100B6000749DFF1F789BFF1FCC9DFF1FB09DFF1F33
:100B700028460FF003FBB2490FF054FB05465046E0
:100B80000FF0FCFAAF490FF04DFB014628460FF07D
:100B900041FA0FF00DFD0546CBF80050D9F80000E2
:100BA0000FF0ECFAA6490FF03DFB074630460FF078
:100BB000E5FAA4490FF036FB014638460FF02AFA51
:100BC0000FF0F6FCC9F800009F4AA04B1688198860
:100BD0009F4AA04B12681B889F4FC6EB050E3544F9
:100BE000039EC6F800E0461A084404990D60019976
:100BF0000E6002993E8808609A4280F28981002541
:100C0000C3EB060E954974450F6880F27681611C2E
:100C10009F4205FB01F50EF1010E95FBFEF5C0F2BA
:100C2000BE81BE42A8BF3E46F61A01FB06F494FB05
:100C3000FEF49A4200F33681BB42C0F23381884C05
:100C400020680FF09BFA87490FF0ECFA86490FF005
:100C5000E1F90FF0ADFCA0F5FF531C3B082B98BF4A
:100C60004FF40050D8F80030184400282060C0F23B
:100C70004281B0F5804F80F252817C4B1B781BB1D2
:100C8000B0F5005F40F05381794D2B78002B40F098
:100C90005481784D20682B68714C984204D080B202
:100CA00008F03EF923682B6009B0BDE8F08F2846B4
:100CB0000FF064FA70490FF0B5FA054650460FF090
:100CC0005DFA6E490FF0AEFA014628460FF0A2F920
:100CD0000FF06EFC0546CBF80050D9F800000FF07D
:100CE0004DFA65490FF09EFA074630460FF046FA76
:100CF00062495FE728460FF041FA5A490FF092FA2D
:100D0000054650460FF03AFA5D490FF08BFA01465E
:100D100028460FF07FF90FF04BFC0546CBF800504A
:100D2000D9F800000FF02AFA4E490FF07BFA074677
:100D300030460FF023FA52493CE728460FF01EFADE
:100D400050490FF06FFA054650460FF017FA4E491A
:100D50000FF068FA014628460FF05CF90FF028FC06
:100D60000546CBF80050D9F800000FF007FA4549C6
:100D70000FF058FA074630460FF000FA424919E7DB
:100D8000D8F80030DFF810B103EBD3735B10DBF859
:100D90000050C8F800301FE6DFF80081DFF800914E
:100DA000D8F8003003EBD3735B10C8F80030BDE512
:100DB000364A06931188364A059120460492DFF898
:100DC000D8B00FF0DBF9049A0599DBF8005052F81F
:100DD00021100FF027FA0FF0EBFBEF1B069B574596
:100DE000A7EB0302B8BF5746FF1AD8F8003090426D
:100DF000BABF013200FB0777474397FBF2F73B444A
:100E000003EBD373234A04925B10C8F80030E3E588
:100E10000FF0B4F9029A52F82B100FF003FA0FF00A
:100E2000C7FBCAEB0802B045B8BFB0468242CAEB66
:100E300008083FF76AAD00FB08F898FBF2F069E597
:100E4000CDCC4C3FCDCC4C3EA489FF1F2C89FF1F3D
:100E5000D89BFF1F8C9DFF1FC49BFF1F0C9EFF1F75
:100E60008C89FF1F9A99193FCDCC4C45C29EFF1F1C
:100E7000219CFF1F2489FF1F3333733FCDCC4C3D92
:100E8000CDCCCC3E6666663FCDCCCC3DCC9BFF1F27
:100E9000F01D0100289DFF1FB09DFF1FCC9DFF1F6F
:100EA000789BFF1F009B1B88002B3FF4C8AE2B1BB9
:100EB000002BB8BF5B42092B47DD05F50050013020
:100EC000001B0FF05BF93B493B4C0FF0ABF90546BB
:100ED00020680FF053F939490FF0A4F9014628466C
:100EE0000FF098F80FF064FBD8F800301844002891
:100EF0002060BFF6BEAE002213E09F4205FB04F562
:100F0000B8BF002195FBFEF54BDA91FBFEF490E6AD
:100F1000B242D4BFC3EB0205C3EB060570E643F64D
:100F2000FF72274B22601B78002B3FF4ADAE05F01B
:100F300093F9244B01221A70ABE605F089F90023DE
:100F40002B70A6E6D9F800003EE64FF400501A4C8C
:100F500088E61D491D4A069320460D8805920FF02C
:100F60000DF9059ADFF868B052F82510DBF800504B
:100F70000FF058F9014600200FF04AF80FF018FB67
:100F80002F44069B56E50FF0F9F8039A52F82B1000
:100F90000FF048F9014600200FF03AF88AE51E46A6
:100FA00042E6B742D4BFC3EB0701C3EB060104FB23
:100FB00001F1AAE7CDCCCC3E8C89FF1F9A99193F4D
:100FC000C29EFF1F219CFF1FCC9BFF1FF01D010035
:100FD000B09DFF1F08B5244B1B88FBB1234B1B782A
:100FE000FBB1234B1B78E3B1224B1B78CBB1224BD7
:100FF0001B78B3B1214B22481A78C2B9214A224941
:101000000088128809680244B1EB620F09DD0122F1
:101010001A706420BDE8084005F032B9174A11780B
:1010200001B908BD1370BDE8084007F043BF154A79
:1010300016490088128809680244B1EB620FF0DD9E
:1010400000221A7007F036FF642005F019F96420B9
:1010500005F016F9642005F013F94FF41670BDE899
:1010600008400CF0DDBA00BF329DFF1F179EFF1F26
:10107000E29DFF1FE39DFF1FE49DFF1FB09BFF1F2D
:10108000C49BFF1F8C9DFF1FD89BFF1F0C9EFF1F43
:1010900038B5114C232025780BF070FD0F4A42F82B
:1010A0002500131F02F1C400002253F8041F8342DD
:1010B0000A44FAD123780A4907480A4C0133DBB2C3
:1010C000322B81FB025108BF0023D217C2EB211241
:1010D0000370226038BD00BF989BFF1F3C9CFF1F20
:1010E0001F85EB51889DFF1F2DE9F04FB84CB94D7E
:1010F0002068B94F83B00FF041F8B8490FF092F86B
:10110000064610200CF07EFC0FF038F8B4490FF0C2
:1011100089F831460EF07EFF0FF04AFA29882060E8
:1011200088423B8843DA9E465B1A7F2B4FF00002D1
:1011300047DDD2015E1C92FBF6F2AA4EDFF8C882B0
:10114000B6F800C0C8F80020BCF1190F00F0DF802D
:10115000BCF11A0F00F01781BCF11E0F00F02081C6
:101160000126B146A04A1288002A00F09D808842DC
:10117000C0F207817045D4BFC1EB0000C1EB0E0087
:101180009A42BABF02FB00000133504390FBF3F3D5
:10119000964A1360964B1888C0B9964A1288AAB925
:1011A000954B197801B11A7003B0BDE8F08F9842E1
:1011B000D4BFC1EB0002C1EB03029E465B1A7F2B3A
:1011C000B7DCC2EBC21292FBF3F2B6E72988D4F87F
:1011D00000E0DFF80082DFF8F8A171456CDCDFF891
:1011E00018C29CF80020002A2ED14FF0010B0428D1
:1011F0008CF800B028D1002E40F094817D4B1888E7
:101200000028D1D0B9F1000FCED023682C883A88BD
:10121000A34280F265810023141B7E2C774DD5BF3D
:10122000C3EB8313C3EBC3135B00013493FBF4F4F0
:101230002B680134A34203D0C0B2E1B207F092FDA3
:101240002C6003B0BDE8F08F012800F0F680022882
:1012500000F0EB800328D1D1694B1B88092BCDD03E
:10126000002ECBD023682E883A88B34280F27B814F
:101270000023961B7E2EDFF88CA1D5BFC3EB831312
:10128000C3EBC3135B00013693FBF6F6DAF80030CC
:101290000136B34203D0F1B24A2007F063FDCAF829
:1012A0000060ABE716469146BCF11E0F7FF472AFAB
:1012B0000022DFF858817EE04F4B1A78002A3FF475
:1012C00073AF002401281C7000F0A480022840F0B5
:1012D0000E81002E00F0A3804A4D2B68002B00F0F9
:1012E0009E800420214607F03DFD424B2C6018886B
:1012F00000283FF459AFB9F1000F3FF455AFC0B229
:10130000002107F02FFD3D4B00221A604CE7DFF86B
:10131000FC8098F80020C2B1DFF8D890B9F800A09E
:10132000BAF1000F11D0DFF8E89099F800B09345BA
:1013300078D05FFA8AF07F2107F014FD98F800302A
:10134000B6F800C089F8003010E0DFF8C49099F8D2
:1013500000A0924566D0274B0021187807F002FDC7
:1013600098F80030B6F800C089F800301E4B1A8893
:10137000002A97D0BCF11E0F40F006810026B1462E
:1013800019E00020FCE6DFF8848098F80020002AAD
:101390000BBF012600264FF000094FF00109E1E6DE
:1013A000DFF86880104B98F800601A88B6FA86F665
:1013B00076094FF0000998F80030002B3FF4E8AEB2
:1013C0002988B7F800E02068C1EB0E03CFE600BF24
:1013D000D09BFF1F389DFF1F349DFF1F9A99193F17
:1013E000CDCCCC3EC29DFF1FF49DFF1F349CFF1F40
:1013F000D69BFF1FD29DFF1FC99DFF1FB89BFF1FDC
:10140000769DFF1F389CFF1FA89DFF1F749DFF1F27
:101410009C9BFF1F1EB1614D2B68002B7BD1604B45
:10142000188865E70026B1469CE6002E3FF4E6AE3C
:10143000DFF868A1DAF800202EE0002E3FF4DEAEDF
:10144000B7F80080F045D4BFC1EB0802C1EB0E0233
:10145000C1EB0808B8F17E0FDFF840A1D5BFC2EBA1
:101460008212C2EBC212520008F1010892FBF8F896
:10147000DAF8002008F10108424506D05FFA88F149
:101480000120009307F06EFC009B1888CAF80080CA
:1014900002287FF4DFAE42462168B5F80080388824
:1014A000414559DA0021C8EB0008B8F17E0FD3BFDF
:1014B000C1EB8111C1EBC11108F10108490091FB99
:1014C000F8F808F10108904506D05FFA88F1042089
:1014D000009307F047FC009B1888CAF80080B9E623
:1014E0009342D4BFC4EB0303C4EB020394E6032886
:1014F00027D12C4B1B88092B91D0002E8FD0274D44
:101500002B68002B8BD04A20214607F02BFC244B64
:101510002C601888ECE6214607F024FC204B2C6058
:101520001888E5E640207F218DE80C0007F01AFCC2
:10153000019B009A188858451CD002287FF48AAE77
:1015400076E704287FF46BAF002E3FF468AF2146A6
:10155000402007F007FC62E78142D4BFC8EB0101DD
:10156000C8EB00019FE79342D4BFC6EB0303C6EB71
:1015700002037EE6B8F80010DAF800E0B7F8008061
:101580008E45FFF665AF5DE72988B7F800E0206873
:101590000026C1EB0E03B146E9E500BF389CFF1FF2
:1015A000D29DFF1F769DFF1F08B5114B1B88022B94
:1015B00009D0052B07D0032B15D0042B0BD00D4BD6
:1015C00001221A7008BD7F21412007F0CBFB094B97
:1015D00001221A7008BD7F21092007F0C3FB054BCB
:1015E00001221A7008BD4021092007F0BBFBE6E785
:1015F000329CFF1FF09BFF1F38B5244B1B881D2B0F
:1016000040D0234B1B88012B25D0224A224B148823
:101610001B68224AA342128828DB21490988934289
:10162000D4BFC4EB0303C4EB0203121B914224DAC0
:1016300001FB0333541C93FBF4F41A4B1A4D1B8823
:10164000052B06D02B689C4203D0E1B2052007F0A1
:1016500089FB2C6038BD154B154A1B681488154A48
:10166000C3F53B630833A3421288D6DA0C490988D4
:10167000121B91424FF00003DADB03FB01F393FBF3
:10168000F2F4DAE7064B1C88D7E700BFC29DFF1FC4
:10169000309DFF1FAC9DFF1F8C9BFF1FC09DFF1F38
:1016A000C69DFF1F329CFF1F849BFF1F3C9DFF1F99
:1016B000309CFF1FAE9DFF1F38B5124D124C2B887A
:1016C000052B12D022684AB9022B0ED0033B012B06
:1016D00013D90E4A00231370236038BD0021052062
:1016E00007F040FB2B88022B04D10021412007F09A
:1016F00039FBEEE7052BE9D1F7E70021092007F0D8
:1017000031FBE6E7329CFF1F849BFF1FF09BFF1F0E
:1017100008B5284B1B78ABB115200BF02FFA264AE1
:10172000264B128818601D2A15D0254A1288DAB176
:10173000012A2BD0234B1B78002B3AD0BDE8084060
:10174000FFF7BABF11200CF05DF91B4A1B4B128842
:1017500018601D2AE9D11C4B1B88002BEAD01B4BBB
:101760001B78002BE6D008E0174A1288002AE1D047
:10177000174A1B6812889A42DCDC124B1B780BB9A3
:10178000FFF712FFBDE80840FFF736BF0F200CF04F
:1017900039F90D4B0F4A1B88106033B10E4BC0F561
:1017A0003B601B8808309842E7DA064B1B78002B19
:1017B000C4D108BDA69DFF1FC29DFF1F8C9BFF1FAC
:1017C000309DFF1FF09BFF1F329CFF1F749DFF1F6A
:1017D000AC9DFF1F3C9DFF1F309CFF1F38B51020A4
:1017E0000CF010F9C830B0F5FA7FC0F2EE80B0F519
:1017F0007A6F0146A8BF4FF47A6101F51673B3F50D
:101800007A6FA8BF4FF47A639BB289B28E4A8F4C2D
:1018100011802220238007F029FC21888C4D8D4CDB
:10182000242007F023FC0E200BF0A8F940F6FF71EE
:10183000C8308842A8BF084620EAE07000F5FA6286
:1018400083B28A42A8BF0A460220194622802B8012
:1018500007F00CFC2188042007F008FC17200CF08E
:10186000D1F8044616200CF0CDF8A042B8BF2046AF
:1018700000F1C801B1F5FA7FC0F2A280B1F57A6F2C
:10188000A8BF4FF47A6101F54873B3F57A6FA8BF2A
:101890004FF47A639BB289B26F4A704C11800A2070
:1018A000238007F0E3FB21880C2007F0DFFB0F20EB
:1018B0000CF0A8F8C0F53F610431B1F5AF6F7CDBE7
:1018C000B1F5FA6FA8BF4FF4FA6189B2644BC0F565
:1018D0004360B0F5AF6F19806CDBB0F5FA6FA8BF4D
:1018E0004FF4FA6083B25F4CA420238007F0BEFB64
:1018F000A620218807F0BAFB0B200BF05BFE002826
:1019000068D011200CF07EF800F1C801B1F52F7FEE
:101910006EDA40F214534FF42F71534A1180534C36
:101920000620238007F0A2FB2188082007F09EFBF9
:1019300000244FF4AF75E1B24D4809F05DF9013470
:101940008542A8BF05460C2CF5D101200CF05AF8B1
:10195000044600200CF056F8323CA0F13203454911
:101960006FF4957000FB03F300FB04F081FB03426E
:1019700081FB0041DB17C017C3EB6223C0EB612082
:1019800003F5AF7200F5AF739342A8BF13469D42B3
:10199000A8BF1D46A5F11401312938DC40F26C7353
:1019A00032213548354A018013602A20BDE838408D
:1019B00007F05CBB4FF4AF6395E74FF4AF6185E789
:1019C00040F214534FF4FA7166E740F24C434FF47F
:1019D000FA711BE715200BF0D1F800F59671B1F5FF
:1019E0002F7F96DB41F25C2399421FDD194694E775
:1019F00041F25C239942F9DC1B4A00F5487089B238
:101A0000B0F52F7F118019DA4FF42F7387E740F27A
:101A10003A72A5F5B9751A4B02FB05F583FB052350
:101A2000ED17A5EB631389B23233BAE70E4A00F51E
:101A3000617089B2B0F52F7F1180E5DB8342A8BFCA
:101A400003469BB26BE700BF389DFF1F349DFF1F0D
:101A50002C9CFF1FE89DFF1F8C9DFF1FC49BFF1F39
:101A6000309CFF1FAE9DFF1FAC9DFF1FC09DFF1F41
:101A7000209CFF1F67BBCF46E09DFF1F9489FF1F7F
:101A8000B5814E1B2DE9F84F0C200BF043F80C20CC
:101A90000BF0F8FCA14914200BF004FDA049A1486B
:101AA00008F03CFD022103200BF092FD02210420EE
:101AB0000BF08EFD022105200BF08AFD022106208D
:101AC0000BF086FD01210A200BF082FD0121092087
:101AD0000BF07EFD01210D200BF07AFD0121282065
:101AE0000BF076FD012114200BF072FD02210B207A
:101AF0000BF06EFD01210C200BF06AFD0C20002183
:101B00000BF052FD04200BF055FD70B305200BF0D7
:101B100051FD044680B300242046834D287005F013
:101B2000B3FE2B78EBB9204607F0CAFA7F4B804909
:101B30001B88804D0988804A2970A3F5AF7140F257
:101B40003A7303FB01F382FB0312DB177B4E7C48E5
:101B5000A3EB621332335A21336009F089F890B94C
:101B6000FEE7BDE8F84F08F0E9BB06200BF022FDC8
:101B70000028CBD10124D0E703200BF01BFDB0FAE5
:101B800080F04009C9E76F4A6F481268DFF800B279
:101B900000230121FEF788FC0B200BF00BFD011E3A
:101BA0000CBF012300238BF8003002D111200BF071
:101BB0000FFDDFF8A091654FDFF8D881644E002358
:101BC000C9F800303B60C8F800304FF0040A14E058
:101BD0000AF0D4FF3B68184438600AF0010080F036
:101BE000010004F03DFB3388002B14BF4B20DC20A8
:101BF0000BF016FDBAF1010A1BD00F200BF002FF0B
:101C0000D8F8003003440E20C8F800300AF0B6FFC0
:101C1000D9F800309BF800200344C9F800301520A3
:101C2000002AD5D111200BF0EDFE3B681844386036
:101C3000D3E7D8F80030D9F8002046493868DFF8F3
:101C400058E1DFF858C1002BB8BF0333002AB8BFF2
:101C5000033292100A604049404A098812880028DD
:101C6000B8BF03309B10801038605F1A1944CEF85B
:101C70000070CCF80010DFF828E1394F3949C8F876
:101C80000030C2EB000C0244CEF800C03A600B609A
:101C90000CB1FFF7A3FD33885BB94FF4FA7004F081
:101CA000EFFA04F0D9FA06F001F94FF4AF600BF047
:101CB000B7FC2D4B012404201C600BF07BFC10B9F9
:101CC0002A4B28701C702A4B1B881C2B1CD0294CBB
:101CD00004F1C80523200AF051FF44F8040F012045
:101CE0000BF09EFCA542F5D1234A244B10781870C6
:101CF00007F0F0F804F0ACFA45F6BF52204921484D
:101D0000BDE8F84F0AF0F2BC1F4B18880028DED05F
:101D10001E4BC0B2197807F025F8D8E7001B3746EC
:101D200040420F006890FF1FB69BFF1FE09DFF1F02
:101D3000C49DFF1F009CFF1FB5814E1B9489FF1F90
:101D4000209CFF1F2889FF1F549DFF1F789BFF1FAA
:101D5000829DFF1F909BFF1FA489FF1F2C89FF1FDF
:101D6000049CFF1FFC9DFF1FBC9DFF1FA09BFF1F2E
:101D7000C29DFF1F389CFF1F409DFF1F269DFF1F18
:101D8000A5050000D89DFF1F089CFF1FCE9BFF1FCD
:101D9000A69DFF1FB09DFF1FB49DFF1F289DFF1F25
:101DA000109EFF1F2DE9F04F8BB007ADC04F2C46A2
:101DB0000AAE611BC9B2BF4808F01EFF3B888342D0
:101DC00094BF0020012004F8010BA642F1D1BA48CB
:101DD000BA4A9DF81C70BA4907709DF81E00B94DAB
:101DE00010709DF820209DF82430B74EB74C0A7033
:101DF0009DF82210297000253370257073B90029D1
:101E000040F01A81B2491AB10B78002B40F00882D9
:101E1000002800F0DB810223237005E0002A40F057
:101E2000BB800523AA492370DFF8F8B2DFF8F882F7
:101E30009DF81D209DF82100DFF8F092DFF8F0A258
:101E4000A44DA54FA54E0B709DF81FC09DF8231003
:101E50009DF827309DF826E08BF8002088F80000D8
:101E60009DF82520297001203A70337089F800C050
:101E70008AF800E00BF0C6FD994A9A4B1168884237
:101E8000CCBF012200221A7040F38A80964B1B8837
:101E9000182B00F28580954AB2F800E00C3B0093C5
:101EA000BEF1000F40F08580914A9BF800C092F887
:101EB00000B098F8008099F800209AF8009094F803
:101EC00000A02C78ABEB4C0BC2EB0B0BA8EB880EF5
:101ED000DE44C9EB897BC9EB8B09DFF81CB2F14406
:101EE00097F800E0BBF800B009EB44093478CE4421
:101EF00004FB0BEE4FF00C097E4C19FB0AEEC4F804
:101F000000E0B8F1000F0BD036784EB17A4E36882B
:101F1000042E0CBF0EF1020E0EF1040EC4F800E008
:101F2000764E774CDFF80CB23688DBF800B02488A8
:101F3000DFF804A2DFF80492BAF800A0B9F8009024
:101F4000009BC6EBC6065E44033CDFF8F4B104EB2D
:101F50004404DBF800B00EEB84045444C9EBC90917
:101F6000DFF8E0A1D944DFF8E0B15AF826605BF869
:101F700029900C3C1C44A3194B44BCF1000F29D000
:101F80002C783CB3002A5BD1B8FA88F85D4C4FEA54
:101F9000581884F8008024E0062323704C4943E756
:101FA000524AB2F800E000230093BEF1000F3FF464
:101FB0007BAFBEF1010F47D0BEF1020F00F0C88029
:101FC0004C4C9BF800C099F8002098F80080D4F899
:101FD00000E096E74B4C002525700AB13A781ABB11
:101FE0000022494C884222704849C4BF484AC2F87E
:101FF00000E00A68934213D0464A474C10680590A7
:102000000598206012680692444C069A24880B605A
:10201000121AA24284BF424A13600BB0BDE8F08F8F
:102020003D483C4A0068EDE7BCF1000FD8D1B8F15B
:10203000000FD5D10122D4E7042323702449F3E60D
:10204000304A00241470CBE7294A9BF800C092F86C
:1020500000E098F8008099F8002094F800B09AF811
:1020600000902C780194AEEB4C0EC2EB0E0EA8EB58
:1020700088047444C9EBC909D944A31EDFF878A0C9
:10208000DFF8C8E0019C97F800B05EF829E0BAF8E4
:1020900000A096F8009003EB44045C4409FB0A4955
:1020A00009F11809134CCE44C4F800E029E700BF39
:1020B000E09DFF1F209CFF1FE29DFF1FE39DFF1F70
:1020C000E49DFF1FE59DFF1FE69DFF1F2D9DFF1F48
:1020D000369DFF1F189EFF1F199EFF1FC89DFF1FE3
:1020E0009489FF1F749DFF1FC29DFF1F889BFF1FC8
:1020F000A689FF1F7C9DFF1FDE9BFF1FB89DFF1F52
:10210000989DFF1FF69DFF1FF79DFF1FE89BFF1F78
:10211000009EFF1F009FFF1F0C9CFF1FD09DFF1FF5
:10212000089EFF1F149EFF1F169EFF1F159EFF1F78
:10213000179EFF1F349CFF1F9A9BFF1FF29BFF1FE0
:10214000F09DFF1F041A010020170100A01D0100CF
:10215000374A9BF800C092F800B0247899F8002024
:1021600098F800800394ABEB4C049AF80090314B44
:1021700095F800A0CDF804A0A8EB880BA41A5C4445
:102180004FF0050B1BFB094B039C97F800A0CDF803
:1021900008A0C9EBC909B3F800A009EB0403BDF816
:1021A0000490029C0BF1050B1EFB09BE96F800B0D3
:1021B000DFF8A490A6440BFB0AEE59F823901E4CBE
:1021C0000EF10C0ECE44C4F800E09AE65FBB0B782B
:1021D000012B2BD9194A23701288002A3FF424AE10
:1021E000174A1288013A92B2062A3FF61DAE154AE6
:1021F0001278002A3FF418AE134A1268012A7FF4BD
:1022000013AE1248124A0068124E82FB0025C21714
:10221000C2EB650202EB4202A0EB8202328003E6CF
:102220000323237000E601232370FDE53B46FBE515
:10223000A689FF1FDE9BFF1F7C9DFF1FA49DFF1F24
:10224000429DFF1F2E9CFF1FBC9DFF1F089EFF1F6E
:10225000ABAAAA2A809DFF1FC81F01002DE9F04FDD
:102260003A4B1B788BB0002B6BD10E200AF086FC0A
:102270000DF084FF01463648364E374DFEF75AF9C9
:102280003348FEF72DF90EF093F980F30C0030601F
:10229000FFF788FD2C68012C7AD0022C00F0A78271
:1022A000032C00F0B5832D4E2D4C33682D4A2E4E55
:1022B0000993099B316812882360591A013A9142A7
:1022C000274F00F28F82294E32689A1A0D2A00F2A7
:1022D0008282274E32689A1A132A00F27782254E9C
:1022E00032689A1A252A1AD9234B1B88002B40F0F2
:1022F0005D81224B1B78002B40F05881FEF7C8FE11
:102300001F4B1B881B3B9BB2022B04D81D4B1B7819
:10231000002B40F04E8103F0C5FF236833601A4D57
:102320002A689B1A502B00F20D82184B1B88012B38
:1023300000F0258206F0AAFD06F0D8FB0BB0BDE840
:10234000F08F07F083FE0BB0BDE8F08FB69BFF1F48
:10235000549DFF1F909DFF1FBC9DFF1F009FFF1FEF
:10236000509DFF1F9089FF1F289CFF1F189CFF1F77
:10237000F89BFF1FFC9BFF1F329DFF1FB09BFF1FA1
:10238000C29DFF1F749DFF1F449DFF1F949DFF1F53
:10239000DFF82093A04AB9F800001378834204D0F4
:1023A000C3B21846137006F0ADFCDFF804839B4AF5
:1023B000B8F800301178994204D0994F3978002943
:1023C00040F0E486974A33681288974E9A42C0F2EA
:1023D000FA80964A1278002A40F0F580DFF8D8A2F9
:1023E000BAF8003023B9924B1B88002B00F0EE8422
:1023F000904A914B11881B88904A0B4412685B10DD
:1024000093428F4A126880F2908400219342B4BFB5
:1024100001230B4604910093ACBF4FF0010B8B4698
:1024200005910E200AF0AAFB864B874A1B681768A5
:1024300003930133A7F25232002B8446029240F3F9
:10244000CC86802BA8BF8023804A814912780191D5
:10245000002A00F0C2800978914200F0BE80B8F8EE
:102460000010DFF84CE2994201F0E1806C49AEF8CF
:102470000030784B4FF0010E81F800E01978DFF85A
:102480003CE2019B8EF800101A70009B002B00F0BC
:102490001781BAF80030002B00F012816E4B1B68D8
:1024A0005A1C002A40F39D86802A00F399866B4CC3
:1024B0006B496C482488098800682144B0EB610F9F
:1024C000C1F22A83A3F148020F2A02D8473BA9F898
:1024D00000300E200AF052FB6FF454731F44874201
:1024E00002DC614B00221A7000200BF08BFA5F4A6D
:1024F0005F4B11685F4C1B888842D4BF00220122C9
:102500002270002B00F008845B4B1C78944240D072
:1025100088423EDD59490C78002C00F01E8758494E
:1025200091F800C0BCF1000F40F01587554F00979F
:10253000554F56480297534F007887F800C0524FC6
:102540004FF0010E87F800C081F800E0002841F04C
:10255000C5804F490978002900F0E1874D49039172
:102560000C460978002940F0D7874B48464F007841
:10257000397001210297217058B1424840490090BA
:10258000002008700099029F0870039901243C7094
:1025900008701A70414B1B88A3F11B02012A40F2FC
:1025A000B9851D2B00F003863D4C7EE6FEF712FD3B
:1025B000A4E63C4B1B78002B3FF4ADAE2B68012BFF
:1025C0007FF4A9AEA9E63168374A069106983749E3
:1025D000106002220B602A6000E71E49DFF8DCE091
:1025E000097800293FF44DAF9EF8000081423FF486
:1025F00048AF03984B2840F3E1871833802BB8F895
:102600000000A8BF802398423FF43BAF28480380D6
:1026100003480123037034E7269DFF1F009CFF1F22
:10262000A09BFF1F2C9CFF1F009FFF1FB09BFF1F45
:102630001E9CFF1FC49BFF1F8C9DFF1FD89BFF1F6D
:102640000C9EFF1F009EFF1F909BFF1FF69DFF1F0C
:10265000E49BFF1FF79DFF1F7C9DFF1F389DFF1F01
:10266000349DFF1FD09BFF1F2C9DFF1F9489FF1FD0
:10267000429DFF1FCA9BFF1F7C9BFF1F179EFF1FD2
:10268000849DFF1FD49DFF1F2E9CFF1F189EFF1FC0
:10269000149EFF1F7D9BFF1F749DFF1FC29DFF1F88
:1026A000509DFF1FC89DFF1FF49BFF1F4C9DFF1FE8
:1026B000C49DFF1F409DFF1FEC9BFF1FE59BFF1F5D
:1026C000029B9C45BFF605AF864B1B88002B3FF451
:1026D00000AFBBF1000F7FF4E1AE834B1B881BB151
:1026E000059B002B7FF4DAAE049B002B3FF4F1AE88
:1026F0007E4B1A78002A7FF4ECAEDFF8649299F8EA
:10270000004001221A70002C40F02D83784B1B787A
:10271000002B02F0C680774B1B78002B02F09A83C7
:10272000754B1B78002B7FF4D4AE744B1B78002BB9
:102730003FF4CFAEB8F8003071490A3BA8F800303A
:102740000A70C6E605F0E8F86E4B1B7873B96E4B5D
:102750001B785BB96D4B1B7843B96D4B1B782BB95C
:102760006C4B1B7813B903F073FD01E003F07CFDA3
:1027700023682B60684B1B88012B7FF4DBAD674A15
:10278000674B116867481A78A1F118032A2101FBE9
:1027900003F10160002A00F0A982634C236899428A
:1027A00000F3528310DA61480278002A40F07C87F7
:1027B0005F4A1068D0F17F0048BF033080100130BD
:1027C0001B1A994242F3BF86216091E2FEF7A0FFF7
:1027D0002368336083E5FEF735F8FEF785FC236850
:1027E000336076E5FDF77AFF3B6833606BE5514A6D
:1027F00034681188A14204DB464B1B78002B00F0A3
:102800005D834D4E4D48336807934D4B079A0068E2
:102810001B88121A9A4200F2A980002B00F0A680B1
:10282000484B1A88002A3FF4BFAE474B47481B6805
:102830000088A342B8BF2346994241F36681444BC6
:102840001960DFF8208188F80020344FFDF746FF3B
:1028500038687F2840F371853E4B7F3883FB003218
:10286000C317C3EB620303EB4303A0EB8300733096
:10287000394B01931B883860002B40F0CA86234BEC
:1028800000931B78002B00F0C683344C2378002B78
:1028900000F0C183DFF8D090DFF8B8A04FF0000B54
:1028A0000CE003F17300C0B298F8001006F082FA51
:1028B00023780BF1010B5B4540F3AD833B6859F87E
:1028C000040F1844A0F17F038AFB0321DA17C2EB3F
:1028D000610202EB42027F28A3EB8203E1DCFDF7F9
:1028E000BBFEE0E71E9CFF1F489DFF1F2C9DFF1FA6
:1028F000149EFF1F159EFF1F169EFF1F179EFF1F92
:10290000A09BFF1F2E9CFF1F849DFF1FD49DFF1FB8
:102910007D9BFF1FB09BFF1F949DFF1F089EFF1F05
:10292000F09BFF1FEC9DFF1FA89BFF1FD59DFF1F66
:10293000849BFF1F2C9CFF1F009FFF1FF49BFF1F0A
:102940001C9CFF1F9E9BFF1F4C9DFF1FE89DFF1FB0
:10295000809BFF1FABAAAA2AD49BFF1F5489FF1F8D
:102960002D9DFF1F129CFF1F2C89FF1F554B564AA0
:102970001B681088554AA342B8BF2346994200F30A
:102980007A82534C12888342A8BF03462360002AF0
:102990007FF457AF9942C8BF134640F37382401A81
:1029A000B0F5804FAABF9B03C3EB8333013093FB89
:1029B000F0F0FDF779FEC0F3C6100DF0DFFB454BDC
:1029C000044618880DF0DAFB4349074620460DF00F
:1029D00029FC014638460DF025FC21460DF01AFB76
:1029E0004FF07E5104460DF0BBFD002841F0718090
:1029F0003A4920460DF0D2FD002840F06986204675
:102A00000DF0FCFDC0B2DFF8F48088F800001CE790
:102A1000334B34681988A14274DD324B1B78002B8C
:102A200070D1DFF8DC9099F800007F2840F33886F9
:102A3000A3F155337F3803F1004383FB0032C31702
:102A4000C3EB620303EB4303A0EB83007330264B1D
:102A500001931B88C0B289F80000002B41F035803B
:102A6000224B00931B78002B00F0A484204C237889
:102A7000002B00F09F841F4FDFF87C804FF0000A8E
:102A80000AE003F17300C0B206F0BCF923780AF142
:102A9000010A534540F38E8457F8043F99F800002B
:102AA0001844A0F17F0388FB0321DA17C2EB61020F
:102AB00002EB42027F28A3EB8203E2DCFDF7CCFDB0
:102AC000E1E700BF4C9DFF1FE89DFF1F9E9BFF1F7E
:102AD000809BFF1FF89DFF1FCDCCCC3D0000FE4228
:102AE0002C9CFF1FB09BFF1FD49BFF1FD49DFF1F7B
:102AF0005489FF1F2C89FF1FABAAAA2A129CFF1F13
:102B0000789DFF1FB34F38687F2800F3C281FDF71F
:102B1000A3FDDFF8249399F800A0824500F02182FC
:102B2000AD4B1B88002B43D1AC4AAD4812680088DE
:102B3000914205DC8242D4BFC1EB0203C1EB00032A
:102B4000411AB1F5804FA6BF9B030131C3EB83331C
:102B500093FBF1F0FDF7A8FDC0F3C6100DF00EFBDE
:102B6000A04B044618880DF009FB9F49804620467B
:102B70000DF058FB014640460DF054FB21460DF088
:102B800049FA4FF07E5104460DF0EAFC002840F06F
:102B90008F87964920460DF001FD002840F095856D
:102BA00020460DF02BFDC0B2DFF8908288F80000BF
:102BB000BAF17F0F40F3BD838D48AAF17F0A80FBF5
:102BC0000A304FEAEA73C3EB600000EB4000AAEB67
:102BD00080007330874B00931B78C0B289F80000E7
:102BE000002B40F01A83844B03931B78002B40F09A
:102BF0004B85824B02931B78002B40F07E87804BE5
:102C00000193029B1B78FBB17E4B1B88012B00F0CC
:102C1000C385022B01F05380032B01F09281042B1A
:102C200001F09D83052B01F03E84062B01F00D86FB
:102C3000072B01F0C187082B02F07880092B02F0E6
:102C40008C810A2B02F0C283009B1B78002B00F0C2
:102C50007684019B6A4C1988002900F0FD8438684D
:102C60007F2840F36383624B7F3883FB0032C317B6
:102C7000C3EB620303EB4303A0EB830073303860C4
:102C8000002940F0AC84009B1B78002B00F075817C
:102C90005D4C2378002B00F07081DFF8A4A1DFF8F1
:102CA0009C814FF0000B0CE003F17300C0B298F868
:102CB000001006F07FF823780BF1010B5B4540F321
:102CC0005C813B685AF8040F494A1844A0F17F031D
:102CD00082FB0321DA17C2EB610202EB42027F287A
:102CE000A3EB8203E0DCFDF7B7FCDFE7474B19609D
:102CF000474B1B68A92202FB03F3002BBCBF03F563
:102D00007F533F339B13543B194481F30C0128201C
:102D10000AF0BAFAFFF70EBB384C3E483549364A3E
:102D2000237003700B70137034E493424FF0000B68
:102D300080F2BC800123CDF800B0CDF814B004932C
:102D4000FFF76FBB344B1B78002B7FF4C2AB039BA8
:102D5000324A243B83F34703D9B25B20136006F069
:102D600001F899F80040032C30D1DFF8D88098F8AA
:102D70000030002B42F0BD81294F3B78002B42F000
:102D8000AB81254C2378002B42F09981254B1B7891
:102D9000002B42F08781244A1380244B1B78002BA0
:102DA00042F04D820C4B7F221A8098F800306BB9AC
:102DB0003B785BB923784BB91D4A7F2107201380EC
:102DC00005F0D0FF7F210B2005F0CCFF194B1F68C9
:102DD000FFF77FBB089EFF1F9E9BFF1F809BFF1F6F
:102DE000E89DFF1FF89DFF1FCDCCCC3D0000FE42AB
:102DF000ABAAAA2AD49DFF1F7D9BFF1F2E9CFF1FFD
:102E0000D49BFF1F429DFF1F5489FF1FA89BFF1FDC
:102E10008C89FF1F849DFF1F179EFF1FC09BFF1FF4
:102E2000169EFF1F159EFF1F229CFF1F189EFF1F4F
:102E3000769DFF1F909BFF1F789DFF1F129CFF1F19
:102E40002C89FF1F149EFF1FBA4A1078002840F0FB
:102E50005983B94A1268D2F17F0248BF033203EBAB
:102E6000A202531CB54A23609942B8BF1160FFF615
:102E70003FAF19463CE7B24B12881960002A7FF435
:102E8000E0AC0B469842D4BFC1EB0003C1EB030397
:102E900085E5AC4B7F3883FB0032C317C3EB62037D
:102EA00003EB4303A0EB8300733032E60123CDF83C
:102EB00010B0CDF800B00593FFF7B3BA01232B6033
:102EC000A14EA24CFFF7F1B9029B1B78FBB1A04BBE
:102ED0001B88012B00F0E284022B00F06F86032B8D
:102EE00001F0A580042B01F05F82052B01F05283D5
:102EF000062B01F0A284072B01F00685082B01F0B8
:102F00004C87092B02F04A800A2B02F02882019B91
:102F10001B88002B00F06C83009B1B783BB9039B44
:102F20001B7823B9029B1B78002B01F00080894B92
:102F30001B78002B00F0288187490B78082B00F2C2
:102F4000238186483A680068854C0133DBB25F1EF6
:102F5000101A44F827000B70824B3468198889F8DE
:102F60000020A142784EBFF61FAB32687E4B08921C
:102F7000089A764C1A60FFF798B9039B1B78002BD0
:102F8000A2D03B68A3F10C007F2840F36C836D480E
:102F90008B3B80FB0320DA17C2EB600000EB4000A4
:102FA000A3EB800303F17300DFF8D081C0B298F87F
:102FB000001005F0FFFE009B1B78002B84D0664CB0
:102FC0002378002B80D0DFF8B8A14FF0000B0CE085
:102FD00003F17300C0B298F8001005F0EBFE2378FF
:102FE0000BF1010B5B457FF76FAF3B685AF8040F9D
:102FF000544A1844A0F18B0382FB0321DA17C2EB79
:1030000061020C3802EB42027F28A3EB8203DFDC73
:10301000FDF722FBDEE74F4B1B78002B40F0EE82E2
:103020003B68524A1278002A45D0A3F10C007F2851
:1030300040F33383434A8B3B82FB0321DA17C2EB15
:10304000610202EB4202A3EB820303F17300C0B200
:1030500098F8001005F0AEFE009B1B7853B33E4C71
:1030600023783BB3DFF81891DFF8D8A04FF0000BBE
:103070000BE003F17300C0B298F8001005F09AFE5F
:1030800023780BF1010B5B4514DD3B6859F8040F05
:103090001844A0F18B038AFB0321DA17C2EB61020B
:1030A0000C3802EB42027F28A3EB8203E1DCFDF740
:1030B000D3FAE0E73B682E4A1278FAB1244A128824
:1030C000012A00F07284022A00F07786032A01F0B8
:1030D0002F80042A01F08C81052A01F0CE82062A75
:1030E00001F0D883072A01F0B484082A01F0CD86C4
:1030F000092A01F098870A2A02F0F980019A1288B9
:10310000002A00F08D821B4A104C137003232B60A1
:10311000FFF7CBB8DFF86C8098F80030002B40F058
:103120001081154F3B78002B40F0F984074C3B7021
:10313000FFF7BBB8D59DFF1F849BFF1FA89BFF1FF8
:10314000809BFF1FABAAAA2A009FFF1F509DFF1F55
:10315000429DFF1F849DFF1F5489FF1FA49BFF1FDB
:103160003089FF1F2C9CFF1FAC9EFF1F7D9BFF1F04
:103170002E9CFF1F789DFF1F9C9BFF1F129CFF1F13
:103180002C89FF1F749DFF1F3A68E5E6DBB21846E5
:10319000137005F0C5FDAC4BAC491A46AC4B184654
:1031A00000230B703B7013700370FFF70BB9DFF84F
:1031B000BC8298F80030002B40F0CF81A54F3B78BF
:1031C000002BB3D0A44BA54C1988A22005F04EFFCC
:1031D00098F800303B70FFF768B80123FFF734B967
:1031E00080249F499F4BA04A09881B8812680B4482
:1031F000B2EB630FBFF66DA99C4B1B78002B40F020
:103200001C82B8F800309A4AA3423FF462A9994B55
:10321000148001221A70FFF75CB9974B01931B8849
:10322000002B42F08A818A4B0393944B0293944C77
:1032300023786BB3DFF85C82DFF848A24FF0000B15
:1032400009E003F17300C0B205F0DCFD23780BF157
:10325000010B5B451CDD58F8043F99F80000184449
:10326000A0F17F038AFB0321DA17C2EB610202EBB4
:1032700042027F28A3EB8203E3DCFDF7EDF9E2E7EE
:103280007E4B029305F0BEFD009B1B78002BCED138
:10329000039B1B78002B3FF4B4AC99F80030A3F1EA
:1032A0000C007F2840F3ED8176488B3B80FB0320A8
:1032B000DA17C2EB600000EB4000A3EB800303F1E0
:1032C0007300C0B205F09EFD009B1B78002B00F040
:1032D000CD816B4C2378002B01F0C082DFF8B481E4
:1032E000DFF8A0A14FF0000B0AE003F17300C0B2B9
:1032F00005F088FD23780BF1010B5B457FF781AC6E
:1033000058F8043F99F800001844A0F18B038AFB99
:103310000321DA17C2EB61020C3802EB42027F286C
:10332000A3EB8203E1DCFDF797F9E0E7FDF794F901
:10333000A5E45046FDF790F94CE4FDF78DF9FFF751
:1033400097BA514A1278002A40F0D581414F434C38
:103350003B70FEF7AABF002008704C49087840B1C6
:10336000394900910978002900F0B581009F0021BA
:1033700039704749097800297FF4F0A8002C40F003
:10338000CE80002840F0CB80384C2F4F94F800E0DE
:103390002F4C0394394C02942D4C2C492070374CFF
:1033A0000097087038702070BEF1000F7FF4E8A815
:1033B000FFF7EFB8264B1B78002B6DD099F8003043
:1033C000A3F10C007F2840F3CC832E4A8B3B82FB79
:1033D0000321DA17C2EB610202EB4202A3EB820384
:1033E00003F17300C0B205F00DFD009B1B78002BAC
:1033F00052D0234C2378002B4ED0264FDFF8848008
:103400004FF0000A09E003F17300C0B205F0FAFCC6
:1034100023780AF1010A53453EDD57F8043F99F835
:1034200000001844A0F18B0388FB0321DA17C2EBDC
:1034300061020C3802EB42027F28A3EB8203E2DC3C
:10344000FDF70AF9E1E700BFD49DFF1F849DFF1F30
:103450007D9BFF1F9C9BFF1FC69DFF1F509DFF1F55
:10346000389DFF1F349DFF1FD09BFF1F749DFF1FC2
:10347000C49DFF1FA09BFF1FD49BFF1F2E9CFF1FFF
:103480005489FF1FABAAAA2AC89DFF1F189EFF1FC1
:10349000149EFF1F2C89FF1FA84B1B78FBB1A84B64
:1034A0001B88012B00F0D486022B00F0CF87032B62
:1034B00001F04A81042B01F0E481052B01F01B840B
:1034C000062B01F0DA84072B01F01F86082B01F090
:1034D000DD86092B01F0C9870A2B01F0A687019B25
:1034E0001B88002B00F0EC82964B1B78002B40F0E1
:1034F000E282954B954A19883468002001231060B8
:103500002B602EE50130C0B2022886BF0021117069
:1035100010701946FFF7ECBB0398002101708C492D
:10352000097800293FF435A88449029109780029D7
:1035300000F0B287029800210170FFF72AB8039BC0
:103540001B78002B7FF485AB029B1B78002B7FF44C
:1035500080AB019B1988FFF782BB7E4A1278002A54
:103560003FF4F4AE7C4F387802F0ECFE7B4B1B78D6
:10357000002B00F0BB8439887E2900F2B784784C98
:10358000DFF80C922368D9F800209B1A0F2B40F229
:103590009680744B01311B8889B239802BB1052B81
:1035A00003D0C9B2052005F0DDFB6F4F226898F803
:1035B0000030C9F800203B70FEF777BE243B002B9B
:1035C000B8F8000040F3788498423EF45AAF9BB2BA
:1035D0006648A8F8003001230370FEF752BFDFF8F9
:1035E0009081C0B298F8001005F0E4FBFFF74BBBE8
:1035F0005F4B3878197805F0DDFB8DE47F214020A2
:1036000005F0B0FB5B495C4A3B680B600021117020
:1036100007E5C0B298F8001005F0CCFBFFF72FB912
:10362000D8B298F8001005F0C5FB3B686BE5534B2A
:10363000DFF860E11978FEF724BF4B2C40F34C8291
:103640001834802CB8F800304D4AA8BF8024A3421B
:103650007FF4DDADFEF73DBF99F8000005F0D2FB29
:103660002188FFF7FCBAFCF7F7FF9DE4029B1B786B
:10367000002B7FF4C9AA039B1B78002B7FF4E9AAD7
:1036800067E7FCF7E9FF1CE63E4B01931B88002B24
:103690007FF4F6AD294B0293FFE5FCF7DDFFD6E49E
:1036A000FCF7DAFFFFF7D3B90132D2B2022A40F2B7
:1036B0005E82002202701946FFF71ABB284C2A4F7F
:1036C00098F800303B70FEF7F0BD7F20FFF76CBA32
:1036D0007F20FFF798B9194F1A4902974FF0000C55
:1036E00081F800C0009F02994FF0010E87F800E0BA
:1036F00081F800C03DE6244F387802F023FE174BD6
:103700001B78002B00F03A8239887E2900F236823D
:10371000134CDFF87C902368D9F800209B1A0F2BFC
:10372000CDD91A4B0131188889B23980002800F0B0
:103730004182C9B2C0B205F015FB36E72E9CFF1FCF
:10374000429DFF1F849DFF1F2C9CFF1F809BFF1F1E
:10375000749DFF1FC89DFF1FC69DFF1F199EFF1F61
:10376000509DFF1F329CFF1F9C9BFF1FA09BFF1FB4
:10377000129CFF1FA49BFF1F5489FF1FF79DFF1F73
:10378000C49DFF1FD49BFF1FCE9BFF1F089CFF1FE4
:10379000049EFF1FE59BFF1FDFF8B4A399F800000C
:1037A000BAF80030E34AE44CC31A82FB031ED9176F
:1037B000C1EB6E0101EB4101A3EB810303EB43037A
:1037C00054F8233018447F2840F3AE847F3882FBBE
:1037D0000032C317C3EB620303EB4303A0EB830088
:1037E0007330DFF870B3C0B205F00CFBBBF80030EB
:1037F000022B7FF629AA99F80010BAF80030CD4ABA
:10380000CB1A82FB030ED817C0EB6E0000EB400012
:10381000A3EB800303EB430304EB830358680844E2
:103820007F2840F320877F3882FB0032C317C3EB29
:10383000620202EB4202A0EB82007330C0B205F0DC
:10384000E1FABBF80030032B7FF6FEA999F80010CF
:10385000BAF80030B74ACB1A82FB030ED817C0EB78
:103860006E0000EB4000A3EB800303EB430304EB8B
:103870008304A06808447F2840F370817F3882FB6E
:103880000032C317C3EB620202EB4202A0EB8200DC
:103890007330C0B205F0B6FAFFF7D6B9DFF8B0A2C0
:1038A0003868BAF80030A34AA34CC31A82FB031E3F
:1038B000D917C1EB6E0101EB4101A3EB810303EBCF
:1038C000430354F8233018447F2840F329847F3879
:1038D00082FB0032C317C3EB620303EB4303A0EB8D
:1038E00083007330DFF87082DFF868B298F8001058
:1038F000C0B205F05FFABBF80030022B7FF607ABD1
:103900003968BAF800308B4ACB1A82FB030ED817FD
:10391000C0EB6E0000EB4000A3EB800303EB43031E
:1039200004EB8303586808447F2840F398867F3867
:1039300082FB0032C317C3EB620202EB4202A0EB30
:1039400082007330C0B298F8001005F033FABBF86B
:103950000030032B7FF6DBAA3968BAF80030754ACD
:10396000CB1A82FB030ED817C0EB6E0000EB4000B1
:10397000A3EB800303EB430304EB8304A068084438
:103980007F2840F3F8807F3882FB0032C317C3EBF7
:10399000620202EB4202A0EB8200733098F8001042
:1039A000C0B205F007FAFFF7B2BADFF8A4A1614987
:1039B000BAF80020604C9A1A81FB020ED017C0EBB7
:1039C0006E0000EB4000A2EB800202EB420254F8D2
:1039D000220018447F2840F32284A0F17F0381FB5A
:1039E0000321DA17C2EB610000EB4000A3EB80007B
:1039F0007330DFF860B198F80010C0B205F0DAF962
:103A0000BBF80030022B50D93968BAF80030494A67
:103A1000CB1A82FB030ED817C0EB6E0000EB400000
:103A2000A3EB800303EB430304EB830358680844D0
:103A30007F2840F385867F3882FB0032C317C3EBB3
:103A4000620202EB4202A0EB82007330C0B298F82F
:103A5000001005F0AFF9BBF80030032B25D938680A
:103A6000BAF80030334AC31A82FB031ED917C1EBE0
:103A70006E0101EB4101A3EB810303EB430304EB74
:103A80008304A36818447F286EDD7F3882FB0032F0
:103A9000C317C3EB620202EB4202A0EB8200733059
:103AA000C0B298F8001005F085F93B68FFF726BB17
:103AB0000120FFF779B80021402005F053F918E5FF
:103AC00099F8000005F09EF90EE505F09BF9FEF768
:103AD000C7BF0120FEF797BF243C002CB8F8003088
:103AE00040F3C585A3423EF4F4ACA4B2134BA8F84E
:103AF000004001221A70FEF7ECBC114B01931B88A9
:103B0000002B7FF4BFABFFF77CB80E498342A8BF00
:103B100003460B60FEF795BE1446FFF76DBB0A4BDC
:103B20000A4C19886A2005F0A1FA98F800303B7019
:103B3000FEF7BBBBABAAAA2A3C1B0100A09BFF1F40
:103B4000D49BFF1F809BFF1FCE9BFF1F509DFF1F1D
:103B5000809DFF1FB49BFF1F129CFF1FFCF77CFD85
:103B600097E6FCF779FD3DE4FCF776FD98E70270F7
:103B70001946FFF7BDB8FCF76FFD0FE7D14B1B7877
:103B8000002B3FF49BAD3B88CF4F002B3FF496AD0D
:103B9000CE4CDFF848932268D9F80010521A0F2A49
:103BA0007FF68DADCA4A013B108899B23980002852
:103BB0007FF4BFADC8B205F049F9F6E4DFF820A301
:103BC0003868BAF80030C34AC34CC31A82FB031EDC
:103BD000D917C1EB6E0101EB4101A3EB810303EBAC
:103BE000430354F8233018447F2840F325847F385A
:103BF00082FB0032C317C3EB620303EB4303A0EB6A
:103C000083007330DFF8DC82DFF8DCB298F8001054
:103C1000C0B205F0CFF8BBF80030022B7FF677A9D1
:103C20003968BAF80030AB4ACB1A82FB030ED817BA
:103C3000C0EB6E0000EB4000A3EB800303EB4303FB
:103C400004EB8303586808447F2840F30E867F38CE
:103C500082FB0032C317C3EB620303EB4303A0EB09
:103C600083007330C0B298F8001005F0A3F8BBF8D9
:103C70000030032B7FF64BA93868BAF80030954A1C
:103C8000C31A82FB031ED917C1EB6E0101EB410180
:103C9000A3EB810303EB430304EB8304A368184401
:103CA0007F287FF768AF7F3882FB0032C317C3EBF2
:103CB000620303EB4303A0EB830073306EE6DFF88F
:103CC00020A299F80000BAF80030824A824CC31A48
:103CD00082FB031ED917C1EB6E0101EB4101A3EB7F
:103CE000810303EB430354F8233018447F2840F347
:103CF000A7837F3882FB0032C317C3EB620303EB59
:103D00004303A0EB83007330DFF8DCB1C0B205F0F1
:103D100079F8BBF80030022B7EF696AF99F80010C8
:103D2000BAF800306B4ACB1A82FB030ED817C0EBEF
:103D30006E0000EB4000A3EB800303EB430304EBB6
:103D40008303586808447F2840F393857F3882FBBB
:103D50000032C317C3EB620303EB4303A0EB830002
:103D60007330C0B205F04EF8BBF80030032B7EF67E
:103D70006BAF99F80010BAF80030564ACB1A82FBA4
:103D8000030ED817C0EB6E0000EB4000A3EB8003DE
:103D900003EB430304EB8304A06808447F287FF708
:103DA000DDAE7F3882FB0032C317C3EB620303EB47
:103DB0004303A0EB830073306BE5DFF824A1454992
:103DC000BAF80020444C9A1A81FB020ED017C0EBBF
:103DD0006E0000EB4000A2EB800202EB420254F8BE
:103DE000220018447F2840F32E83A0F17F0381FB3B
:103DF0000321DA17C2EB610000EB4000A3EB800067
:103E00007330DFF8E4B098F80010C0B204F0D2FFCD
:103E1000BBF80030022B7FF648AE3968BAF80030A4
:103E20002C4ACB1A82FB030ED817C0EB6E0000EBB6
:103E30004000A3EB800303EB430304EB83035868C8
:103E400008447F2840F319857F3882FB0032C3176E
:103E5000C3EB620303EB4303A0EB83007330C0B2F8
:103E600098F8001004F0A6FFBBF80030032B7FF693
:103E70001CAE3868BAF80030164AC31A82FB031E1B
:103E8000D917C1EB6E0101EB4101A3EB810303EBF9
:103E9000430304EB8304A36818447F287FF764AED0
:103EA0007F3882FB0032C317C3EB620303EB43038B
:103EB000A0EB83007330F3E501283EF4E2AA01236E
:103EC000FFF786BB189EFF1FCE9BFF1F509DFF1F55
:103ED000089CFF1FABAAAA2A5C1C0100049EFF1FBE
:103EE000809DFF1F129CFF1FB49BFF1FCE4B1B78B2
:103EF000002B3FF4E3AB3B88CC48002B3FF4DEAB18
:103F0000CB4CDFF83C932268D9F80010521A0F2AE4
:103F10007FF6D5ABC74A013B128899B20180002ACF
:103F20003FF443AB052A7FF43CABFFF73EBB4FF4B5
:103F30007A43013BFDD199F8000004F063FFFEF7DE
:103F4000F6BFDFF800A399F80000BAF80030BA4ACB
:103F5000BA4CC31A82FB031ED917C1EB6E0101EBE9
:103F60004101A3EB810303EB430354F823301844CE
:103F70007F2840F3E8817F3882FB0032C317C3EB10
:103F8000620202EB4202A0EB82007330DFF8B8B2AB
:103F9000C0B204F037FFBBF80030022B7EF654AEFF
:103FA00099F80000BAF80030A34AC31A82FB032133
:103FB000DA17C2EB610202EB4202A3EB820303EBCE
:103FC000430304EB83035B6818447F2840F31F849A
:103FD0007F380C2290FBF2F302FB13007330C0B267
:103FE00004F010FFBBF80030032B7EF62DAE99F8DD
:103FF0000000BAF80030904AC31A82FB0321DA1796
:10400000C2EB610202EB4202A3EB820303EB430328
:1040100004EB8304A36818447F287FF79FAD7F38A3
:104020000C2290FBF2F302FB1300733031E4DFF853
:1040300014A23868BAF800307F4A804CC31A82FB59
:10404000031ED917C1EB6E0101EB4101A3EB810304
:1040500003EB430354F8233018447F2840F3708166
:104060007F3882FB0032C317C3EB620202EB4202CD
:10407000A0EB82007330DFF8D481DFF8CCB198F880
:104080000010C0B204F096FEBBF80030022B7EF6A2
:104090003EAF3868BAF80030674AC31A82FB032182
:1040A000DA17C2EB610202EB4202A3EB820303EBDD
:1040B000430304EB83035B6818447F2840F3AB831E
:1040C0007F380C2290FBF2F302FB13007330C0B276
:1040D00098F8001004F06EFEBBF80030032B7EF65B
:1040E00016AF3868BAF80030534AC31A82FB03216E
:1040F000DA17C2EB610202EB4202A3EB820303EB8D
:10410000430304EB8304A36818447F287FF733AD8F
:104110007F380C2290FBF2F302FB130073303DE476
:10412000FCF79AFAFFF7DEBBFCF796FAFFF759BBEC
:10413000DFF810A14049BAF80020404C9A1A81FBE0
:10414000020ED017C0EB6E0000EB4000A2EB800225
:1041500002EB420254F8220018447F2840F3F68014
:10416000A0F17F0381FB0321DA17C2EB610101EBB0
:104170004101A3EB81007330DFF8CCB098F8001058
:10418000C0B204F017FEBBF80030022B7FF68DACF6
:104190003868BAF80030284AC31A82FB0321DA17BC
:1041A000C2EB610202EB4202A3EB820303EB430387
:1041B00004EB83035B6818447F2840F338837F381F
:1041C0000C2290FBF2F302FB13007330C0B298F89C
:1041D000001004F0EFFDBBF80030032B7FF665AC58
:1041E0003868BAF80030144AC31A82FB0321DA1780
:1041F000C2EB610202EB4202A3EB820303EB430337
:1042000004EB8304A36818447F287FF7ADAC7F38A4
:104210000C2290FBF2F302FB1300733040E4FCF736
:104220001BFAFFF7E6BB00BF189EFF1FC69DFF1FCE
:10423000509DFF1F329CFF1FABAAAA2AEC1C010055
:10424000049EFF1F809DFF1FB49BFF1F129CFF1F3A
:10425000DFF838A399F80000BAF80030C34AC44C1C
:10426000C31A82FB0317D917C1EB670101EB4101A8
:10427000A3EB810303EB430354F8233018447F2856
:104280006ADD7F3882FB0032C317C3EB620202EBA8
:104290004202A0EB82007330DFF8F4B2C0B204F047
:1042A000B1FDBBF80030022B7FF619A999F8000088
:1042B000BAF80030AD4AC31A82FB0321DA17C2EB09
:1042C000610202EB4202A3EB820303EB430304EB24
:1042D00083035B6818447F2840F3AC827F380C224C
:1042E00090FBF2F302FB13007330C0B204F08AFDBE
:1042F000BBF80030032B7FF6F2A899F80000BAF85B
:1043000000309A4AC31A82FB0321DA17C2EB61021A
:1043100002EB4202A3EB820303EB430304EB8304AF
:10432000A36818447F2814DD7F380C2290FBF2F339
:1043300002FB13007330C0B204F064FDFFF7CFB886
:10434000FCF78AF997E6FCF787F91FE6FCF784F992
:1043500012E7FCF781F9EEE7FCF77EF99CE7DFF85E
:104360002CA299F80000BAF80030804A814CC31A98
:1043700082FB031ED917C1EB6E0101EB4101A3EBD8
:10438000810303EB430354F8233018447F28DADD1C
:104390007F3882FB0032C317C3EB620303EB430396
:1043A000A0EB83007330F1E5DFF8E0A13868BAF8DC
:1043B00000306E4A6F4CC31A82FB031ED917C1EB43
:1043C0006E0101EB4101A3EB810303EB430354F8BE
:1043D000233018447F28B3DD7F3882FB0032C317B7
:1043E000C3EB620303EB4303A0EB8300733042E6AD
:1043F000DFF898A15D49BAF800205E4C9A1A81FB5B
:10440000020ED017C0EB6E0000EB4000A2EB800262
:1044100002EB420254F8220018447F2896DDA0F1F6
:104420007F0381FB0321DA17C2EB610000EB400040
:10443000A3EB800073309FE6FCF70EF9FFF7E2BBB9
:10444000FCF70AF960E4FCF707F9DAE4DFF83CA1CD
:1044500099F80000BAF80030444A474CC31A82FB6E
:104460000317D917C1EB670101EB4101A3EB8103EE
:1044700003EB430354F8233018447F287FF76CAFD5
:104480007F3882FB0032C317C3EB620303EB4303A5
:10449000A0EB83007330FFE6384800903848394974
:1044A0000390FEF76DB8DFF8E4A099F80000BAF8C1
:1044B00000302E4A344CC31A82FB0321DA17C2EBB8
:1044C000610202EB4202A3EB820303EB430354F8C5
:1044D000233018447F2840F3A7817F380C2290FBBB
:1044E000F2F302FB13007330DFF8A4B0C0B204F0A3
:1044F00089FCBBF80030022B19D999F80000BAF8F2
:1045000000300C22C11A91FBF2F302FB131302FBE1
:1045100003435B6818447F2840F385847F3890FB11
:10452000F2F302FB13007330C0B204F06BFCBBF873
:104530000030032B7EF688ABBAF8003099F8000003
:104540000C22C11A91FBF2F302FB131302FB03448A
:10455000A36818447F287FF701AB7F3890FBF2F304
:1045600002FB13007330FFF794B900BFABAAAA2A6D
:104570003C1B0100A81E01005C1C0100D49DFF1F14
:104580007D9BFF1F849DFF1F00200100809DFF1F5A
:10459000B49BFF1FDFF864A33868BAF80030CE4A36
:1045A000CE4CC31A82FB0321DA17C2EB610202EB85
:1045B0004202A3EB820303EB430354F82330184475
:1045C0007F2840F32E817F380C2290FBF2F302FB10
:1045D00013007330DFF82883DFF828B398F8001051
:1045E000C0B204F0E7FBBBF80030022B1AD93868E0
:1045F000BAF800300C22C11A91FBF2F302FB13133C
:1046000002FB03435B6818447F2840F3C3837F3871
:1046100090FBF2F302FB13007330C0B298F8001065
:1046200004F0C8FBBBF80030032B7EF670ACBAF880
:10463000003038680C22C11A91FBF2F302FB13130D
:1046400002FB0344A36818447F287FF794AA7F38AD
:1046500090FBF2F302FB13007330FFF79FB9FBF7F7
:10466000FBFFFFF76FB9FBF7F7FFFFF7E7B8012B89
:104670003DF42FAF0124FFF739BADFF880A2964945
:10468000BAF80020954C9A1A81FB0210D117C1EBA1
:10469000600101EB4101A2EB810202EB420254F8FE
:1046A000220018447F2840F3B980A0F17F030C203A
:1046B00093FBF0F200FB12307330DFF848B298F849
:1046C0000010C0B204F076FBBBF80030022B1AD900
:1046D0003868BAF800300C22C11A91FBF2F302FBE1
:1046E000131302FB03435B6818447F2840F34F8396
:1046F0007F3890FBF2F302FB13007330C0B298F8DE
:10470000001004F057FBBBF80030032B7FF6CDA957
:10471000BAF8003038680C22C11A91FBF2F302FBA0
:10472000131302FB0344A36818447F287FF71CAAD5
:104730007F3890FBF2F302FB13007330FFF7B0B940
:10474000FBF78AFFFFF782B9DFF8B0A199F8000004
:10475000BAF80030604A624CC31A82FB0321DA17B0
:10476000C2EB610202EB4202A3EB820303EB4303C1
:1047700054F8233018447F2846DD7F380C2290FB04
:10478000F2F302FB13007330DFF878B1C0B204F02B
:1047900039FBBBF80030022B19D999F80000BAF8A0
:1047A00000300C22C11A91FBF2F302FB131302FB3F
:1047B00003435B6818447F2840F38B807F3890FB6D
:1047C000F2F302FB13007330C0B204F01BFBBBF822
:1047D0000030032B7EF683AEBAF8003099F8000063
:1047E0000C22C11A91FBF2F302FB131302FB0344E8
:1047F000A36818447F287FF7ACAD7F3890FBF2F3B5
:1048000002FB1300733096E5FBF726FFBCE7FBF7CE
:1048100023FFFFF7E4BBFBF71FFF58E4FBF71CFF88
:104820004BE7FBF719FFD5E6FBF716FF5CE6FBF756
:1048300013FFCBE4FBF710FF57E5DFF8C0A03868A3
:10484000BAF80030244A274CABE6DFF8B0A099F85C
:104850000000BAF80030204A224C2CE6029B1B785C
:10486000002B7EF4D1A9FEF7F4B9FBF7F5FEFFF7B4
:10487000F9B9FBF7F1FEFFF774BAFBF7EDFEFFF7AE
:10488000EEBADFF878A099F80000BAF80030124AC2
:10489000154C61E7DFF864A00F49BAF80020114C0D
:1048A000F1E6124B1B78002B00F0C182104B1B78F5
:1048B000002B7DF40EAE0F4B1B78002B3DF409AEA0
:1048C000B8F800300C490A33A8F800300A70FDF738
:1048D00000BEFBF7C1FE77E7ABAAAA2A00200100C1
:1048E000EC1C0100181E0100A81E0100159EFF1FF0
:1048F000169EFF1F179EFF1FA09BFF1F809DFF1F7F
:10490000129CFF1FB49BFF1FA44C2388002B40F078
:10491000BE83DFF8A0B2A249A24A0988D7F8008076
:10492000B2F800E0A048C1EB080C0C229CFBF2F1AD
:1049300002FB11C14FF0900C0CFB0EFE02FB01E1DB
:104940006FF00B0E405880440EFB03807F2840F32D
:104950000285A0F17F0393FBF2F002FB103073306D
:10496000924BC0B2197804F025FABBF800202388D6
:104970001344022B23DD8A4A8A4B11883868B3F826
:1049800000C0DFF824E2411A0C2291FBF2F302FB93
:104990001311902303FB0CF302FB013373445B6898
:1049A00018447F2840F3AD857F3890FBF2F302FB7B
:1049B000130073307D4BC0B2197804F0FBF9BBF8DB
:1049C000002023881344032B23DD754A754B11887F
:1049D0003868B3F800C0DFF8D0E1411A0C2291FB2F
:1049E000F2F302FB1311902303FB0CF302FB0133E0
:1049F00073449B6818447F2840F35D857F3890FBA3
:104A0000F2F302FB13007330684BC0B2197804F064
:104A1000D1F9BBF8002023881344042B7EF777AA32
:104A2000634B1B88012B7EF472AA3A68A2F10C003A
:104A30007F2840F38F828B3A0C2092FBF0F300FB2F
:104A400013207330594BC0B2197804F0B3F9FEF754
:104A50005EBA524C2288002A00F0D7825449DFF80F
:104A600054B10988BBF800000331884227DD4C4867
:104A70004C490088B1F800E0DFF82CC1181A0C216D
:104A800090FBF1F901FB19004FF0900909FB0EFEB4
:104A900001FB00E06FF00B0E5CF8000003440EFB1E
:104AA00002307F2840F3B7847F3890FBF1F301FB9D
:104AB00013007330C0B298F8001004F07BF9BBF813
:104AC000002023881344022B23DD354B354A3868F8
:104AD0001B88B2F800C0DFF8D0E0C31A0C2193FBAA
:104AE000F1F201FB1232902303FB0CF301FB0233C2
:104AF00073445B6818447F2840F3E4847F3890FB5C
:104B0000F1F301FB13007330C0B298F8001004F009
:104B100051F9BBF8002023881344032B23DD204BDD
:104B2000204A38681B88B2F800C0DFF87CE0C31A5E
:104B30000C2193FBF1F201FB1232902303FB0CF3E7
:104B400001FB023373449B6818447F2840F3C184FF
:104B50007F3890FBF1F301FB13007330C0B298F87B
:104B6000001004F027F9BBF8002023881344042B1D
:104B70007EF79BAF0E4B1B88012B7EF496AF3A68F5
:104B8000A2F10C007F287EF7EFAF8B3A0C2092FB4E
:104B9000F0F300FB13207330FEF782BF149CFF1F5D
:104BA000809DFF1F2E9DFF1F90170100129CFF1F6D
:104BB000EE9BFF1FB49BFF1FCE4C2388002B40F0C1
:104BC0002782DFF864B3CC49CC4A098899F8000001
:104BD000B2F800E0DFF85483C1EB000C0C229CFB20
:104BE000F2F102FB11C14FF0900C0CFB0EFE02FB28
:104BF00001E16FF00B0E58F8011008440EFB0300A2
:104C00007F2840F30484A0F17F0393FBF2F002FBC2
:104C100010307330C0B204F0F5F8BBF800202388E0
:104C20001344022B22DDB44AB44B118899F80000DA
:104C3000B3F800C0DFF8F4E2411A0C2291FBF2F362
:104C400002FB1311902303FB0CF302FB01337344AB
:104C50005B6818447F2840F3E5837F3890FBF2F3CC
:104C600002FB13007330C0B204F0CCF8BBF8002094
:104C700023881344032B22DD9F4AA04B118899F807
:104C80000000B3F800C0DFF8A4E2411A0C2291FB47
:104C9000F2F302FB1311902303FB0CF302FB01332D
:104CA00073449B6818447F2840F302847F3890FB4C
:104CB000F2F302FB13007330C0B204F0A3F8BBF8A8
:104CC000002023881344042B7DF7BEAF8C4B1B8838
:104CD000012B7DF4B9AF99F80020A2F10C007F28D8
:104CE0007EF73CAF8B3A0C2092FBF0F300FB1320D5
:104CF0007330FEF7CEBDDFF800A299F80000BAF8D5
:104D00000030804CC11A0C2291FBF2F302FB13130A
:104D100002FB03F3E35818447F287FF775AD7F3813
:104D200090FBF2F302FB130073302DE5764B1B88EA
:104D3000182B12D099F800201344A3F118007F28F3
:104D400040F3DC830C20973B93FBF0F200FB123323
:104D500003F17300C0B204F055F86C4A6C4B127842
:104D600033F81230182B3DF46FAF99F8002013443C
:104D7000A3F118007F287EF7F1AE0C20973B93FB40
:104D8000F0F200FB123303F17300FEF782BDFBF774
:104D900063FCB3E4FBF760FC3FE45B4B1A88182A22
:104DA00013D03B681344A3F118007F2840F37D83A0
:104DB0000C20973B93FBF0F200FB123303F17300DE
:104DC000544BC0B2197803F0F5FF504B50491A7894
:104DD000022A94BF013200221A701A7831F81200A8
:104DE000182810D10424022A02F10100C2B288BF9F
:104DF000002231F81200182804D1013CF3D11A70B6
:104E0000FEF785B81A703B680344A3F118007F28A9
:104E100040F3A0800C20973B93FBF0F200FB123391
:104E200003F173000EE6FBF717FCFFF77DBB3A4B6F
:104E30001B78002B7DF486AF384B1B78002B3DF49C
:104E400048ABB8F8003036490133A8F800300A7092
:104E5000FDF73FBB304B1B78002B7DF43AAB2F4B5B
:104E60001B78002B3DF435ABB8F800302C49013BE2
:104E7000A8F800300A70FDF72CBBDFF87CA099F889
:104E80000000BAF80030274C3CE71F4A1288182A65
:104E900012D01344A3F118007F2840F3C0820C20E5
:104EA000973B93FBF0F200FB123303F17300C0B2A7
:104EB00098F8001003F07EFF144B15491A78022A67
:104EC00094BF013200221A701A7831F812001828A3
:104ED0002FD10424022A02F10100C2B288BF0022AD
:104EE00031F81200182823D1013CF3D11A703B6825
:104EF000FEF704B9149CFF1F809DFF1F2E9DFF1F0E
:104F0000EE9BFF1F00200100BE9BFF1F139CFF1F95
:104F10009C9DFF1F129CFF1F169EFF1F179EFF1FC9
:104F2000A09BFF1F181E0100B49BFF1F90170100DC
:104F30001A703B680344A3F118007F287EF714AE73
:104F40000C20973B93FBF0F200FB123303F173004C
:104F5000FEF7A6BDFBF780FB74E5BF4B1B88182B43
:104F600012D099F800201344A3F118007F2840F3D1
:104F7000AD820C20973B93FBF0F200FB123303F160
:104F80007300C0B203F03EFFB44AB54B127833F859
:104F90001230182B7FF4E9AEFDF756BEAE4B1A88DF
:104FA000182A13D03B681344A3F118007F2840F35C
:104FB00086820C20973B93FBF0F200FB123303F147
:104FC0007300A84BC0B2197803F0F4FEA34BA449B8
:104FD0001A78022A94BF013200221A701A7831F826
:104FE000120018287FF40FAF0424022A02F10102F4
:104FF00094BFD2B2002231F8120018287FF402AF19
:10500000013CF2D11A70FDF782BFDFF87CB22EE5C9
:10501000954ADFF874B21288BBF80010033291424F
:105020007FF7FBADCFE58C4A1288182A12D01344C3
:10503000A3F118007F2840F35E820C20973B93FB7E
:10504000F0F200FB123303F17300C0B298F80010C5
:1050500003F0B0FE814B82491A78022A94BF0132D4
:1050600000221A701A7831F8120018287FF461AF04
:105070000424022A02F1010294BFD2B2002231F8C4
:10508000120018287FF454AF013CF2D12EE7764A83
:10509000DFF8F4B11288BBF80010033291427FF7B9
:1050A00064AC38E4714B01227F2107201A8003F0A1
:1050B00059FE7F210B2003F055FEFDF76EBE6C4BB1
:1050C00004227F2107201A8003F04CFE00210B20D0
:1050D00003F048FEFDF75ABE654B02227F210720F0
:1050E0001A8003F03FFE7F210B2003F03BFEFDF70B
:1050F00048BE5F4B002107201C8003F033FE7F2158
:105100000B2003F02FFEFDF737BE5A4C2388002BEF
:1051100040F0E681DFF870B1574999F80000574A2E
:1051200009881788DFF858E1411A0C2291FBF2FC3C
:1051300002FB1C114FF0900C0CFB07F702FB0171F6
:105140006FF00B075EF80110014407FB03107F2886
:1051500040F3C3817F3890FBF2F302FB13007330FE
:10516000C0B203F04FFEBBF8002023881344022B8B
:1051700021DD414B414A99F800001B88B2F800E05C
:105180003F4FC31A0C2193FBF1F201FB1232902323
:1051900003FB0EF301FB02333B445B6818447F289A
:1051A00040F3C8817F3890FBF1F301FB13007330AB
:1051B000C0B203F027FEBBF8002023881344032B62
:1051C00021DD2D4B2D4A99F800001B88B2F800E034
:1051D0002B4FC31A0C2193FBF1F201FB12329023E7
:1051E00003FB0EF301FB02333B449B6818447F280A
:1051F00040F39D817F3890FBF1F301FB1300733086
:10520000C0B203F0FFFDBBF8002023881344042B39
:105210007EF765A9144B1B88012B7EF460A999F8D1
:105220000020A2F10C007F287FF793A88B3A0C2076
:1052300092FBF0F300FB13207330FFF77CB8114BA7
:1052400000227F2107201A8003F08CFD7F210B2094
:1052500003F088FDFDF7A9BDC69BFF1F139CFF1F30
:10526000149DFF1F129CFF1FEE9BFF1F229CFF1F20
:10527000769DFF1F149CFF1F809DFF1F2E9DFF1F0B
:10528000901701009E9BFF1FB49BFF1FB04B1B8814
:10529000182B12D099F800201344A3F118007F288E
:1052A00040F33C810C20973B93FBF0F200FB123360
:1052B00003F17300C0B203F0A5FDA64AA64B127815
:1052C00033F81230182B3EF40AA999F80020134441
:1052D000A3F118007F287FF73CA80C20973B93FB95
:1052E000F0F200FB123303F17300FFF724B89B4A7E
:1052F0001288182A12D01344A3F118007F2840F313
:1053000007810C20973B93FBF0F200FB123303F173
:105310007300C0B298F8001003F04CFD8D4B90491B
:105320001A78022A94BF013200221A701A7831F8D2
:10533000120018287FF4FDAD0424022A02F10102B4
:1053400094BFD2B2002231F8120018287FF4F0ADD9
:10535000013CF2D1CAE5FBF77FF9FFF701BB7F4BB8
:105360001A88182A13D03B681344A3F118007F2829
:1053700040F3DA800C20973B93FBF0F200FB1233F2
:1053800003F17300774BC0B2197803F013FD714B32
:1053900073491A78022A94BF013200221A701A78CF
:1053A00031F8120018287FF42EAD0424022A02F1ED
:1053B000010294BFD2B2002231F8120018287FF403
:1053C00021AD013CF2D11A70FDF7A1BD634B1B88E2
:1053D000182B12D099F800201344A3F118007F284D
:1053E00040F393800C20973B93FBF0F200FB1233C9
:1053F00003F17300C0B203F005FD564A584B127812
:1054000033F81230182B7FF4B0ACFDF71DBCFBF75E
:1054100023F9FFF7FFBBFBF71FF9FFF74BBBFBF7C8
:105420001BF944E5FBF718F91DE44C4B1B88182BBE
:1054300011D099F800201344A3F118007F286ADDE9
:105440000C20973B93FBF0F200FB123303F1730047
:10545000C0B203F0D7FC3F4A414B127833F8123008
:10546000182B7FF432AFFEF73AB83F4B1B88182B4E
:1054700011D099F800201344A3F118007F2850DDC3
:105480000C20973B93FBF0F200FB123303F1730007
:10549000C0B203F0B7FC2F4A344B127833F8123005
:1054A000182B7FF412AFFEF71AB8FBF7D5F887E494
:1054B000FBF7D2F800E4FBF7CFF8FFF7A5BAFBF74C
:1054C000CBF87EE5FBF7C8F8FFF71EBBFBF7C4F887
:1054D00057E5FBF7C1F8FFF741BBFBF7BDF83FE627
:1054E000234ADFF898B01288BBF8001003329142CB
:1054F0007FF739AE10E6FBF7AFF8A6E5FBF7ACF89F
:1055000028E4FBF7A9F8FFF755BAFBF7A5F871E710
:10551000FBF7A2F8FDE6FBF79FF899E7FBF79CF88D
:10552000C8E6FBF799F8B3E7FBF796F82AE7FBF72D
:1055300093F865E6FBF790F83AE60E4B03930E4BB3
:105540000293FDF79FBE23601946FDF7D1BB00BF54
:10555000BE9BFF1F139CFF1F9C9DFF1FC89BFF1F2F
:105560001C9DFF1F129CFF1FC69BFF1F149DFF1F4A
:10557000EE9BFF1F7D9BFF1F2E9CFF1FB49BFF1FF9
:1055800038B507F097FB0B4805F0CEFA00234FF033
:105590007E5201210848FAF769FF084B084A094979
:1055A000802400251C7118461D60BDE838400BF0B2
:1055B00045B800BF209CFF1F549DFF1FD89DFF1FB3
:1055C0001C89FF1FFD05000010B50446A420636878
:1055D000198803F04BFDE368A6201988BDE8104048
:1055E00003F044BD43682A20198803F03FBD00BF83
:1055F00010B5044622206368198803F037FDE3687C
:1056000024201988BDE8104003F030BD10B50446D1
:105610000A206368198803F029FDE3680C201988C3
:10562000BDE8104003F022BD10B5044606206368B3
:10563000198803F01BFDE36808201988BDE81040B5
:1056400003F014BD10B5044602206368198803F006
:105650000DFDE36804201988BDE8104003F006BD85
:1056600070B50E4C84B01225042201230646039027
:10567000029320468DE824001423102106F058FCE4
:1056800006220923029303960195204600921423D3
:10569000102106F04DFC04B070BD00BF489EFF1FF6
:1056A00070B5AE4CB4F90030032B00F0E880002B4D
:1056B0004DD0022B6CD0052B00F09880012B00F010
:1056C000C080042B00D070BD00244FF4AF75E1B250
:1056D000A34805F091FA01348542A8BF05460C2C79
:1056E000F5D1012008F08EF90446002008F08AF96F
:1056F000323CA0F132039B496FF4957000FB03F339
:1057000000FB04F081FB034281FB0041DB17C01763
:10571000C3EB6223C0EB612003F5AF7200F5AF73FA
:105720009342A8BF13469D42A8BF1D46A5F1140190
:10573000312900F3E28040F26C7332218A488B4AAF
:105740000180BDE870402A20136003F08FBC0E205A
:1057500007F014FA40F6FF71C8308842A8BF084627
:1057600020EAE07000F5FA6283B28A42804D814EF1
:10577000A8BF0A460220194633802A8003F076FC2F
:105780002988042003F072FCB4F90030022B92D176
:10579000172008F037F90546162008F033F9A8421B
:1057A000B8BF284600F1C801B1F5FA7FC0F2BF804A
:1057B000B1F57A6FA8BF4FF47A6101F54873B3F57C
:1057C0007A6FA8BF4FF47A639BB289B26A4A6B4D75
:1057D00011800A202B8003F049FC29880C2003F05B
:1057E00045FCB4F90030052B7FF468AF0F2008F0BA
:1057F00009F9C0F53F630433B3F5AF6FC0F28F8092
:10580000B3F5FA6FA8BF4FF4FA6399B25C4BC0F5D9
:105810004360B0F5AF6F19807EDBB0F5FA6FA8BFBB
:105820004FF4FA6083B2574DA4202B8003F01EFC86
:105830002988A62003F01AFCB4F90030012B7FF46C
:1058400040AF0B2007F0B6FE00283CD0112008F036
:10585000D9F800F1C801B1F52F7F3CDB41F25C23A0
:10586000994278DC484A00F5487089B2B0F52F7F3C
:1058700011806DDB8342A8BF03469BB231E010204C
:1058800008F0C0F8C830B0F5FA7F4BDBB0F57A6F9E
:105890000146A8BF4FF47A6101F51673B3F57A6F2C
:1058A000A8BF4FF47A639BB289B2384A384D118051
:1058B00022202B8003F0DAFB2988242003F0D6FB7A
:1058C000B4F90030F3E6152007F058F900F59671A9
:1058D000B1F52F7F30DA40F214534FF42F712A4A7A
:1058E00011802C4D06202B8003F0C0FB2988082056
:1058F00003F0BCFBB4F90030E3E640F23A72A5F5E0
:10590000B975254B02FB05F583FB0523ED17A5EBC8
:10591000631389B2323311E74FF4AF6383E74FF477
:10592000AF6173E740F24C434FF4FA71BDE740F2C8
:1059300014534FF4FA7149E741F25C2399420ADCAF
:10594000114A00F5617089B2B0F52F7F118091DAAC
:105950004FF42F73C5E71946C1E700BF229EFF1F12
:10596000209CFF1F67BBCF46E09DFF1F9489FF1F50
:10597000E89DFF1F2C9CFF1F8C9DFF1FC49BFF1FDA
:10598000309CFF1FAE9DFF1FAC9DFF1F389DFF1F6A
:10599000349DFF1FC09DFF1FB5814E1B2DE9F041B7
:1059A000224D82B0012602B284B2009228460196AE
:1059B0007823192106F002FA04F10C0212B28DE8E4
:1059C00044002846A7197823192104F1020806F09B
:1059D000F5F93FB20FFA88F819233A4628461946D6
:1059E0000196CDF8008006F0E9F978233A4628467A
:1059F0001946CDF80080019604F10A070B3406F031
:105A0000DDF93FB224B278233A46284619468DE89C
:105A1000500006F0D3F9192300943A46019628461F
:105A2000194606F0CBF902B0BDE8F081489EFF1F91
:105A300030B583B000230C4605B2009326225B23C9
:105A40001C210C4805F00AFF29460123262209489B
:105A500005F014FA002C24B205DB2146012326228E
:105A6000044805F00BFA044A044B15801C8003B06F
:105A700030BD00BF489EFF1FAA89FF1FAC89FF1FD2
:105A800070B59F4C237882B01BB19E4B4FF6FF72CE
:105A90001A809D4BB3F90030C3B99C4A994B1068EA
:105AA000B3F9002080F30C005B2303FB00F000132C
:105AB0001C30824243D04FF0FF31FFF7B9FF9448CA
:105AC00005F030FF0023237002B070BD012B1BD006
:105AD000022B53D0032B38D0042B00F08D80052BE4
:105AE000F0D10F2007F08EFFC0F53B600830B0F515
:105AF000AF6F41DBB0F5FA6FA8BF4FF4FA60A0F5C5
:105B0000AF625B2383482EE0834B1A68B2F52F7F88
:105B100032DB41F25C239342A8BF1346A3F52F73F7
:105B20005B227E4802FB03F380FB0320DB17C3EB01
:105B3000A0201C30734BB3F900308342BBD1784BAB
:105B4000B3F900300133B6D1BCE7764B1B68B3F52F
:105B5000FA7F11DBB3F57A6FA8BF4FF47A6372480E
:105B6000A3F5FA725B2303FB02F380FB0320DB1730
:105B7000C3EB20201C30DDE71C20DBE76B4B1B68F0
:105B8000B3F5FA7F2EDBB3F57A6FA8BF4FF47A63D3
:105B9000A3F5FA7264485B2303FB02F380FB032046
:105BA000DB17C3EB20201C30614B1B68B3F5FA7F79
:105BB0001ADBB3F57A6FA8BF4FF47A63A3F5FA72D4
:105BC00059495B2303FB02F381FB0321DB17C3EB82
:105BD00021211C314B4BB3F90030834206D0FFF733
:105BE00027FF6CE71C20DFE71C21F3E74C4BB3F9E0
:105BF00000308B42F3D165E7272200258DE8240091
:105C000076231C2142484B4E06F0D8F816E0B0F53A
:105C1000AF7FA8BF4FF4AF70323803FB00F386FBB1
:105C20000321DB17C3EB61111C3109B201231D44B1
:105C30002722374805F022F90C2D09D0E9B23E4859
:105C400004F0DAFF31284FF05B03E0DC1C21EDE7C4
:105C5000012007F0D7FE6FF495733238374A03FB03
:105C600000F082FB0023C017C0EB632303F5AF7382
:105C7000312B42DDB3F5AF7FA8BF4FF4AF735B228A
:105C8000323B2C4D02FB03F385FB0325DB17C3EBF3
:105C900065151C35002007F0B5FE6FF4957332389A
:105CA000264A03FB00F082FB0023C017C0EB6323EE
:105CB00003F5AF73312B1EDDB3F5AF7FA8BF4FF4F3
:105CC000AF735B22323B1B4902FB03F381FB0321D1
:105CD000DB17C3EB61111C310A4BB3F90030AB4247
:105CE00001D028467BE70E4BB3F900308B423FF4DE
:105CF000E6AE284673E71C21EEE71C25CAE700BF85
:105D00001C9EFF1FAA89FF1F229EFF1F909DFF1F41
:105D1000489EFF1F37800B6D8C9BFF1FD30585416D
:105D2000AC89FF1FD09BFF1F011FB812D89BFF1F1C
:105D30000C9EFF1F4B48371B209CFF1F67BBCF46A5
:105D40002DE9F041044682B056482768E56805F021
:105D5000DDFC1120FFF722FE012619234FF0280851
:105D6000194624224F480196CDF8008006F026F807
:105D70007823194624224B480196CDF8008006F07E
:105D80001DF83146474806F0AFFB0222192145486D
:105D900006F0A6FB38460BF013FA39460246414896
:105DA00006F038FD3F4806F04BFD142200213D4827
:105DB00006F096FB03223C493A4806F02BFD394891
:105DC00006F03EFD23220021364806F089FB03221F
:105DD0003649344806F01EFD324806F031FD7DB1EB
:105DE0002F20FFF7DBFD322200212E4806F078FB42
:105DF00003222F492B4806F00DFD2A4806F020FD0E
:105E000001232C4A18461370FFF72AFC2189638965
:105E100062685B1A5C2B128832DD521A02EB420276
:105E2000C2EB4212013392FBF3F31B33224A1D48AB
:105E3000138001261A221BB28DE844001946142251
:105E400005F0BCFFCDB1218A638AE2685B1A5C2B46
:105E500012881DDC511A5C2202FB01F292FBF3F363
:105E60001B33164A0F481380012438221BB28DE8D9
:105E700014001946322205F0A1FF02B0BDE8F081FE
:105E8000511A5C2202FB01F292FBF3F31B33CDE7C4
:105E9000521A02EB4202C2EB4212334492FBF3F37A
:105EA0001B33DEE7489EFF1FD8200100DC200100E5
:105EB000E0200100C19EFF1F1E9EFF1F209EFF1FAE
:105EC0002DE9F0411E4682B014461AB3052A054654
:105ED00000F09C80099B6F4A00EBC305012C6F8981
:105EE00029896868A7EB010382FB03E21A444FEAA1
:105EF000E373C3EBA213028829D0042C69D0664A4D
:105F0000022CB2F9001060D0082C65D0012002B03C
:105F1000BDE8F081614D624A2B681268CB1A93424A
:105F20000F466FD95F4A338811785F48012918BF3F
:105F300001241470089A06321BB212B28DE81400C4
:105F40001946BDF9202005F039FF2F60DEE79BB22E
:105F5000D31A994203DC9F423946A8BF1946089AD2
:105F60000180B6F90030BDF920804F48971D4FF0F1
:105F7000000E3FB2194642460097CDF804E005F006
:105F80001DFF29896A896B68521A1B885C2AA3EB5A
:105F9000010377DD03EB43030132C3EB431393FBB0
:105FA000F2F303F11B0213B201203280194642467C
:105FB000019000973C4805F001FF3A4B00221A700F
:105FC000354A022CB2F900109ED14B1C1BB2138033
:105FD00004E012FA83F3BCE700231380994295D0C2
:105FE000089AB6F9003030480632012412B2009205
:105FF00019460194BDF9202005F0E0FE204602B0CC
:10600000BDE8F081204602B0BDE8F08107240026FB
:106010005A2323228DE850001A21234805F09CFEC4
:106020000121214806F060FA01211F4806F062FABA
:10603000232235211C4806F053FA22461B491A48F0
:1060400006F0E8FB184806F0FBFB174805F06AFC71
:106050004FF4FA6007F0E4FAFFF722FB5A232322F9
:106060001A218DE85000104805F076FE0E4805F024
:1060700059FC2846FFF764FE0D4B01221A70FFF70A
:10608000FFFC43E75C2101FB03F393FBF2F21B32BD
:1060900089E700BFC94216B2269EFF1FAC9EFF1FB4
:1060A000F42F0100C19EFF1F489EFF1FE420010046
:1060B0001C9EFF1F2DE9F04F5A4E5B4DB6F9007044
:1060C0004C7855F8277085B08146984604B10C7815
:1060D000DFF874A11AB99AF80030002B39D0534D6B
:1060E000002338462B808AF80030FFF729FE504AFB
:1060F000504BB5F90000012111704FF6FF721A8064
:1061000060B301285ED00120322322460190009323
:106110004946494B3846FFF7D3FE00240346B5F9FC
:106120000020022A39DD00222A80B6F900203D49EC
:10613000002A3BDB052AC4BF00220A80B8F1000F09
:1061400039D1002C0CBF18464FF0FF3005B0BDE828
:10615000F08F364DB5F900000028D2D1DFF8ECB051
:10616000364ADBF800301268C3EB0903934227D9A3
:10617000334B1A78012A18BF01201870FFF770FA04
:106180000123CBF80090012C2AD0042C35D0022C0E
:106190003AD0082C3ED00024C1E7C6D1FA68002AC4
:1061A000C1D0B6F900201F49002AC3DA05220A80AF
:1061B000B8F1000FC5D00393FFF762FC039BC0E763
:1061C0000346E0E74FF0000E142322468DE8084016
:1061D00049461C4B38467446FFF772FE03469EE75D
:1061E00032888AF80040013232807A6982B1002414
:1061F000384603939047039B91E732880121013A87
:1062000032808AF80010F0E701222A8000248CE70F
:10621000144684E77A69002129804FF0FF34002A70
:10622000E6D182E7229EFF1FB089FF1F269EFF1F37
:106230001C9EFF1FAA89FF1F209EFF1FF42F010035
:10624000C19EFF1F1E9EFF1F249EFF1FAC9EFF1FAF
:1062500001210D2007F0A8B900210D2007F0A4B9F5
:1062600001460D2007F0A0B908B50D2007F0A2F9EE
:10627000B0FA80F149090D20BDE8084007F094B953
:1062800010B5002144080D2007F08EF9204607F0D4
:10629000C7F90D20012107F087F92046BDE810401D
:1062A00007F0BEB9214A224B10881B68984210B5EE
:1062B00035DA204A1288141A9A42A8BF1A46B4F551
:1062C000157F22DA121A40F2532303FB02F393FBE9
:1062D000F4F105310A2006F0D7FF174B197801B306
:1062E000164B17491B6840F2271283F3070302FB82
:1062F00003F381FB03211944DB17C3EBA111053123
:106300000920BDE8104006F0BFBF131A4FF4157204
:10631000611C02FB03F393FBF1F10531DAE7002185
:10632000D8E70920BDE8104006F0AEBF2C9CFF1F47
:10633000809BFF1FE89DFF1FF09BFF1F849BFF1F9B
:10634000090402817F2838B5A8BF7F200F4C4FF485
:10635000167202FB00F284FB02311144D21705468B
:10636000C2EBA1110A2006F08FFF7F3D4FF4967318
:1063700003FB05F384FB03211944DB17A3EBA111F5
:106380000920BDE8384006F07FBF00BF0904028144
:10639000C368B3F9003030B583EAE374A4EBE37467
:1063A000002BA0B218DB012300E0134603EB8302AD
:1063B00052009442F9DA0A4D90FBF3F285FB03E4B4
:1063C00003FB1200DB173032D3EBA40380B201F8D9
:1063D000012BF1D10B7030BD2D230B700131E2E7A1
:1063E0006766666638B5094D8224204602F058FE7D
:1063F00035F8021B00B28842204601D002F036FE7A
:106400000234A4B28A2CF0D138BD00BF1C9DFF1FFE
:10641000024B8020198802F029BE00BFC89BFF1FD5
:1064200038B5094D7824204602F03AFE35F8021BB3
:1064300000B28842204601D002F018FE0234A4B215
:10644000802CF0D138BD00BF149DFF1F024B762079
:10645000198802F00BBE00BFC69BFF1F38B5094D5F
:106460004624204602F01CFE35F8021B00B288428A
:10647000204601D002F0FAFD0234A4B24E2CF0D135
:1064800038BD00BF9C9DFF1F024B4420198802F0BD
:10649000EDBD00BFBE9BFF1F024B4E20198802F0CE
:1064A000E5BD00BFD49BFF1F024B9A20198802F064
:1064B000DDBD00BF149CFF1F024B9820198802F01D
:1064C000D5BD00BFEE9BFF1F024B8C20198802F048
:1064D000CDBD00BF2E9DFF1F024B9C20198802F0EE
:1064E000C5BD00BFB49BFF1F024BA020198802F05E
:1064F000BDBD00BFA49DFF1F024B9620198802F06E
:10650000B5BD00BF809DFF1F024B8A20198802F095
:10651000ADBD00BF429DFF1F08B5034B1020198879
:1065200002F0A4FD012008BD409DFF1F024B10207A
:10653000198802F09BBD00BF409DFF1F024B2C201D
:10654000198802F093BD00BFB29BFF1F024B1E20B3
:10655000198802F08BBD00BFCC9BFF1FC3680E20C3
:10656000198802F083BD00BF024B2820198802F071
:106570007DBD00BF989DFF1F024B6220198802F06D
:1065800075BD00BFDE9BFF1F024B6420198802F01F
:106590006DBD00BF949DFF1F024B5A20198802F069
:1065A00065BD00BF949BFF1F024B1620198802F0A7
:1065B0005DBD00BF9E9BFF1F024B2E20198802F07D
:1065C00055BD00BF1C9CFF1F024B3020198802F0F4
:1065D0004DBD00BFF89DFF1F024B9E20198802F0A1
:1065E00045BD00BF9089FF1F024B1820198802F09B
:1065F0003DBD00BF329CFF1F024BA220198802F054
:1066000035BD00BFC69DFF1F024B1A20198802F03E
:106610002DBD00BFDC9BFF1F024B1C20198802F020
:1066200025BD00BFD69BFF1F024B6620198802F0D4
:106630001DBD00BFD29DFF1F024B7220198802F0C2
:1066400015BD00BFF49DFF1F024B2020198802F0EA
:106650000DBD00BFD09DFF1F024B3220198802F0F4
:1066600005BD00BFC29DFF1F024B6820198802F0C4
:10667000FDBC00BF089CFF1F024B6C20198802F074
:10668000F5BC00BF889BFF1F024B5220198802F007
:10669000EDBC00BF2E89FF1F024B5020198802F06D
:1066A000E5BC00BF2089FF1F024B5420198802F06F
:1066B000DDBC00BFA489FF1F024B5C20198802F0DB
:1066C000D5BC00BFA889FF1F024B5E20198802F0CD
:1066D000CDBC00BF2C89FF1F024B6020198802F03F
:1066E000C5BC00BF309DFF1F024B5620198802F029
:1066F000BDBC00BF109CFF1F244B1B880B2B43D835
:10670000DFE803F00B10151A1F24292E33383D063D
:10671000084604221E490AF011BE084604221D49FB
:106720000AF00CBE084604221B490AF007BE0846C0
:1067300004221A490AF002BE0846042218490AF047
:10674000FDBD0846042217490AF0F8BD0846042298
:1067500015490AF0F3BD0846042214490AF0EEBDBB
:106760000846042212490AF0E9BD084604221149EC
:106770000AF0E4BD084604220F490AF0DFBD0846CE
:1067800004220E490AF0DABD704700BF809DFF1F4A
:106790009028010050260100042501004429010031
:1067A000082501002C2901000C25010010250100FD
:1067B00074270100142501009C2801001825010000
:1067C000064B074A10B41C88064B0846002C14BF21
:1067D00011461946042210BC0AF0B0BDEC9BFF1F05
:1067E0001C25010020250100064B074A10B41C8817
:1067F000064B0846002C14BF11461946042210BC53
:106800000AF09CBD1E9CFF1F1C25010020250100D5
:10681000064B074A10B41C88064B0846002C14BFD0
:1068200011461946042210BC0AF088BD329DFF1F94
:106830001C25010020250100064B074A10B41C88C6
:10684000064B0846002C14BF11461946042210BC02
:106850000AF074BD489DFF1F1C2501002025010082
:10686000064B074A10B41C88064B0846002C14BF80
:1068700011461946042210BC0AF060BD829DFF1F1C
:106880001C25010020250100064B074A10B41C8876
:10689000064B0846002C14BF11461946042210BCB2
:1068A0000AF04CBD229CFF1F1C2501002025010081
:1068B0001B4B1B880A2B0AD8DFE803F00A0E1216BE
:1068C0001A1E22262A2E0600164B186808607047EA
:1068D000154B186808607047144B186808607047BB
:1068E000134B186808607047124B186808607047AF
:1068F000114B186808607047104B186808607047A3
:106900000F4B1868086070470E4B18680860704796
:106910000D4B1868086070470C4B1868086070478A
:10692000429DFF1F4825010020250100242501006C
:10693000282501002C250100302501003425010007
:10694000382501003C2501004025010044250100B7
:10695000F0B52B4E2B4FDFF8C4E005460FCE87B0C5
:106960006C460FC496E803003B68274A274F44F85B
:10697000040B40F6CC308342C8BF3A46BEF80060F4
:106980002180012E11889278ADF80D108DF80F201E
:106990002AD032D340F6CA02022E18BF00229A42F1
:1069A00026DAA3F698031A491A4AC3EB031381FBAC
:1069B00003011944DB17C3EB6123243382FB03215A
:1069C000DA17C2EBA10202EB8201A3EB41033033E1
:1069D00030328DF813308DF8112069462846162282
:1069E0000AF0ACFC07B0F0BD40F698029A42D8DB42
:1069F000094B1868CDF81100EFE740F6FC02CEE72E
:106A00005C250100889DFF1F502501004C250100D9
:106A10003B773B986766666654250100249DFF1FFF
:106A2000F8B5174C174E2278174D33782F888E46BD
:106A3000003218BF012201467046FFF73BFB0023DE
:106A400098423370237015DB14BF012000202B887F
:106A50009F420ED040F23A72A3F5AF730B490C4C33
:106A600002FB03F381FB0312DB17A3EB6213323348
:106A70002360F8BD0749012218460A702270E6E734
:106A8000A08AFF1F399EFF1FE09DFF1FB5814E1B8F
:106A90009489FF1FC09EFF1F014B187802F07EBA39
:106AA000A89EFF1F014B187802F092BA4C90FF1F6E
:106AB000134BB3F9003030B583EAE374A4EBE3740D
:106AC000002BA0B218DB012300E0134603EB830286
:106AD00052009442F9DA0B4D90FBF3F285FB03E48C
:106AE00003FB1200DB173032D3EBA40380B201F8B2
:106AF000012BF1D10B7030BD2D230B700131E2E77A
:106B00004C90FF1F67666666144BB3F9003070B592
:106B100083EAE375A5EBE375002BACB21ADB012326
:106B200000E0034603EB830040008542F9DA0C4E97
:106B300094FBF3F086FB03E503FB1044DB173030D6
:106B4000D3EBA503A4B201F8010BF1D105480B70FA
:106B5000106070BD2D230B700131E0E7949BFF1F87
:106B60006766666674250100134BB3F9003030B5D3
:106B700083EAE374A4EBE374002BA0B218DB0123D7
:106B800000E0134603EB830252009442F9DA0B4D06
:106B900090FBF3F285FB03E403FB1200DB173032BA
:106BA000D3EBA40380B201F8012BF1D10B7030BDFF
:106BB0002D230B700131E2E79089FF1F676666663F
:106BC000134BB3F9003030B583EAE374A4EBE374FC
:106BD000002BA0B218DB012300E0134603EB830275
:106BE00052009442F9DA0B4D90FBF3F285FB03E47B
:106BF00003FB1200DB173032D3EBA40380B201F8A1
:106C0000012BF1D10B7030BD2D230B700131E2E768
:106C1000C69DFF1F67666666134BB3F9003030B53B
:106C200083EAE374A4EBE374002BA0B218DB012326
:106C300000E0134603EB830252009442F9DA0B4D55
:106C400090FBF3F285FB03E403FB1200DB17303209
:106C5000D3EBA40380B201F8012BF1D10B7030BD4E
:106C60002D230B700131E2E72E89FF1F67666666F0
:106C7000134BB3F9003030B583EAE374A4EBE3744B
:106C8000002BA0B218DB012300E0134603EB8302C4
:106C900052009442F9DA0B4D90FBF3F285FB03E4CA
:106CA00003FB1200DB173032D3EBA40380B201F8F0
:106CB000012BF1D10B7030BD2D230B700131E2E7B8
:106CC0002089FF1F67666666134BB3F9003030B545
:106CD00083EAE374A4EBE374002BA0B218DB012376
:106CE00000E0134603EB830252009442F9DA0B4DA5
:106CF00090FBF3F285FB03E403FB1200DB17303259
:106D0000D3EBA40380B201F8012BF1D10B7030BD9D
:106D10002D230B700131E2E7A489FF1F67666666C9
:106D2000134BB3F9003030B583EAE374A4EBE3749A
:106D3000002BA0B218DB012300E0134603EB830213
:106D400052009442F9DA0B4D90FBF3F285FB03E419
:106D500003FB1200DB173032D3EBA40380B201F83F
:106D6000012BF1D10B7030BD2D230B700131E2E707
:106D7000A889FF1F67666666134BB3F9003030B50C
:106D800083EAE374A4EBE374002BA0B218DB0123C5
:106D900000E0134603EB830252009442F9DA0B4DF4
:106DA00090FBF3F285FB03E403FB1200DB173032A8
:106DB000D3EBA40380B201F8012BF1D10B7030BDED
:106DC0002D230B700131E2E72C89FF1F6766666691
:106DD00008B5702002F064F9044B1988884204D089
:106DE0007020BDE8084002F041B908BD249DFF1F96
:106DF00008B5742002F054F9044B1988884204D075
:106E00007420BDE8084002F031B908BDB89DFF1FED
:106E1000054B1B880846042213B904490AF08EBAB0
:106E200003490AF08BBA00BFD49BFF1F7C250100E9
:106E3000782501000E4B1B88032B17D8DFE803F0E1
:106E4000110C0702084604220A490AF077BA0846DC
:106E5000042209490AF072BA0846042207490AF0D6
:106E60006DBA0846042206490AF068BA704700BFA6
:106E70002E9DFF1F8C25010088250100842501001F
:106E80008025010010B40A4B0A4C0A4693E803001F
:106E900083B0238802AC04E9030004EB83031046AB
:106EA00053F8081C052203B010BC0AF047BA00BF13
:106EB0007C210100949DFF1F30B40A4B0A4D0C4603
:106EC00093E8070084B02B8804AD05E9070005EBC3
:106ED0008303204653F80C1C042204B030BC0AF093
:106EE0002DBA00BF84210100249DFF1FF0B40C4D7A
:106EF0000C4F0E460FCD8CB001AC0FC40FCD0FC49C
:106F000095E807003B8884E807000CAA02EB83039E
:106F1000304653F82C1C04220CB0F0BC0AF00EBA18
:106F200090210100769DFF1FF0B40B4D0B4F0E46D4
:106F30000FCD86B06C460FC495E803003B8884E80B
:106F4000030006AA02EB8303304653F8181C042200
:106F500006B0F0BC0AF0F2B9CC210100329CFF1F50
:106F6000F0B40A4D0A4F0E460FCD86B001AC0FC4E7
:106F70002A683B88226006AA02EB8303304653F856
:106F8000141C0C2206B0F0BC0AF0D8B9E4210100B0
:106F9000D69BFF1FF0B40B4D0B4F0E460FCD86B0A6
:106FA0006C460FC495E803003B8884E8030006AAFA
:106FB00002EB8303304653F8181C042206B0F0BCE1
:106FC0000AF0BCB9F8210100B89DFF1F164B1B88C1
:106FD0000BB31BB283EAE370A0EBE370002B30B578
:106FE00084B21DDB012300E0134603EB8302520051
:106FF0009042F9DA0D4894FBF3F280FB03E503FBC2
:107000001244DB173032D3EBA503A4B201F8012BF5
:10701000F1D10B7030BD0846042205490AF08EB943
:107020002D230B700131DDE7089CFF1F6766666644
:107030009025010030B40A4B0A4D0C4693E8070036
:1070400084B02B8804AD05E9070005EB83032046D7
:1070500053F80C1C042204B030BC0AF06FB900BF16
:1070600010220100889BFF1F054B1B881BB9054B95
:107070001868086070470846042203490AF05EB9A0
:10708000149CFF1F202501001C250100164B1B88A6
:107090000BB31BB230B583EAE374A4EBE374002BAB
:1070A000A0B21CDB012300E0134603EB8302520075
:1070B0009442F9DA0D4D90FBF3F285FB03E403FBF8
:1070C0001200DB173032D3EBA40380B201F8012B9E
:1070D000F1D10B7030BD064B1868086070472D2346
:1070E0000B700131DEE700BFCC9BFF1F6766666651
:1070F00020250100164B1B880BB31BB230B583EA69
:10710000E374A4EBE374002BA0B21CDB012300E0CA
:10711000134603EB830252009442F9DA0D4D90FBC3
:10712000F3F285FB03E403FB1200DB173032D3EBF1
:10713000A40380B201F8012BF1D10B7030BD064BD6
:107140001868086070472D230B700131DEE700BF1F
:10715000869DFF1F6766666620250100164B1B880B
:107160000BB31BB230B583EAE374A4EBE374002BDA
:10717000A0B21CDB012300E0134603EB83025200A4
:107180009442F9DA0D4D90FBF3F285FB03E403FB27
:107190001200DB173032D3EBA40380B201F8012BCD
:1071A000F1D10B7030BD064B1868086070472D2375
:1071B0000B700131DEE700BF9E9BFF1F67666666AE
:1071C00094250100174B1B881BB31BB270B583EAD3
:1071D000E375A5EBE375002BACB21EDB012300E0E9
:1071E000034603EB830040008542F9DA0E4E94FB20
:1071F000F3F086FB03E503FB1044DB173030D3EBE1
:10720000A503A4B201F8010BF1D108480B7010607E
:1072100070BD074B1868086070472D230B70013153
:10722000DCE700BF1C9CFF1F6766666698250100AF
:1072300020250100164B1B880BB31BB230B583EA27
:10724000E374A4EBE374002BA0B21CDB012300E089
:10725000134603EB830252009442F9DA0D4D90FB82
:10726000F3F285FB03E403FB1200DB173032D3EBB0
:10727000A40380B201F8012BF1D10B7030BD064B95
:107280001868086070472D230B700131DEE700BFDE
:10729000F89DFF1F6766666620250100164B1B8858
:1072A0000BB31BB230B583EAE374A4EBE374002B99
:1072B000A0B21CDB012300E0134603EB8302520063
:1072C0009442F9DA0D4D90FBF3F285FB03E403FBE6
:1072D0001200DB173032D3EBA40380B201F8012B8C
:1072E000F1D10B7030BD064B1868086070472D2334
:1072F0000B700131DEE700BFD29DFF1F6766666637
:1073000020250100164B1B880BB31BB230B583EA56
:10731000E374A4EBE374002BA0B21CDB012300E0B8
:10732000134603EB830252009442F9DA0D4D90FBB1
:10733000F3F285FB03E403FB1200DB173032D3EBDF
:10734000A40380B201F8012BF1D10B7030BD064BC4
:107350001868086070472D230B700131DEE700BF0D
:10736000F49DFF1F6766666620250100174B1B888A
:107370001BB31BB270B583EAE375A5EBE375002B75
:10738000ACB21EDB012300E0034603EB83004000A8
:107390008542F9DA0E4E94FBF3F086FB03E503FB1E
:1073A0001044DB173030D3EBA503A4B201F8010B76
:1073B000F1D108480B70106070BD074B1868086069
:1073C00070472D230B700131DCE700BFD09DFF1FFC
:1073D000676666669825010020250100074B1B881B
:1073E000022B06D0012B0CBF054B064B186808601A
:1073F0007047054B18680860704700BF309DFF1F3D
:10740000A0250100A42501009C250100054B1B8837
:107410001BB1054B186808607047044B186808607A
:10742000704700BF109CFF1FAC250100A82501007C
:10743000184B1A8852B3184A128830B50A80B3F92B
:107440000030002B83EAE374A4EBE374BCBF2D236C
:107450008B70A0B2ACBF02310331012300E01346B0
:1074600003EB830252009442F9DA0C4D90FBF3F2E5
:1074700085FB03E403FB1200DB173032D3EBA403DC
:1074800080B201F8012BF1D10B7030BD044B1868AC
:1074900008607047DC9BFF1FB025010067666666C9
:1074A0002025010070B53C4D2B780646002B35D1C8
:1074B0001C4673780BB9204670BDFAF773FC374A47
:1074C000374B3848127831781B78007802EB430349
:1074D0004A1E03EB80030E2AEDD801A050F822F0DB
:1074E000497500006B750000B77400004975000015
:1074F000B7740000B7740000B7740000377500005F
:10750000B7740000B7740000B7740000B7740000CF
:10751000B7740000B774000033750000AE21224834
:1075200003F0A4FE204804F0F1F800232B7001249E
:10753000BFE706F087FBAF211B4803F097FE1B4A0D
:10754000012313702B70B6E783B919480388042907
:107550004FF6FF7103F1FF320CBF01230B461344BA
:1075600003F07F03013303800FE073B1013B114A45
:1075700032F813304BB10E4E0F481049104A338089
:107580000123002606700B701370084A02210123A4
:1075900011702B70204670BDA08AFF1F189EFF1F20
:1075A000199EFF1FC89DFF1F489EFF1FC09EFF1F03
:1075B000C49DFF1F049DFF1F009CFF1FA09BFF1F7A
:1075C000C39EFF1F10B5064B064C1A8820460121AA
:1075D00001F03AFD21884220BDE8104001F046BD8F
:1075E000EC9BFF1FBC9BFF1F10B5064B064C1A8877
:1075F0002046022101F028FD21884220BDE81040EC
:1076000001F034BD1E9CFF1FBC9BFF1F10B5064B35
:10761000064C1A882046042101F016FD21884220DC
:10762000BDE8104001F022BD329DFF1FBC9BFF1F33
:1076300010B5064B064C1A882046062101F004FDC1
:1076400021884220BDE8104001F010BD489DFF1F79
:10765000BC9BFF1F10B5064B064C1A882046002124
:1076600001F0F2FC21884220BDE8104001F0FEBC90
:10767000829DFF1FBC9BFF1F08B5122001F010FD6B
:10768000054B1988884206D0122001F0EFFCBDE8B6
:10769000084001F003BC08BD769DFF1F08B55820C7
:1076A00001F0FEFC054B1988884206D0582001F0F5
:1076B000DDFCBDE8084001F0F1BB08BD869DFF1F61
:1076C00008B5142001F0ECFC054B1988884206D05F
:1076D000142001F0CBFCBDE8084001F0DFBB08BD81
:1076E000229CFF1FF0B480EAE075A5EBE07500284E
:1076F000ACB21FDB1DBF2B230B704E1C0E460123AB
:1077000000E0134603EB830252009542F9DA0B4F77
:1077100094FBF3F287FB030503FB1244DB173032C3
:10772000D3EBA503A4B206F8012BF1D133700846C0
:10773000F0BC70472D230B704E1CE0E76766666651
:10774000174B18880C2813D0192815D01A2817D0D1
:107750001B2819D01C281BD01D281DD01E2803D083
:107760000C3800B2FFF7BEBF0E4A106808607047C1
:107770000D4A1068086070470C4A1068086070472E
:107780000B4A1068086070470A4A10680860704722
:10779000094A106808607047084A10680860704716
:1077A000C29DFF1FD0250100B8250100BC250100A6
:1077B000C0250100C4250100C8250100CC25010019
:1077C000034B1888A0EB8000400000B2FFF78ABF8F
:1077D000A89EFF1F024BB3F90000FFF783BF00BF55
:1077E000DE9BFF1F024B1888033800B2FFF77ABFF9
:1077F000989DFF1F024B18880C3800B2FFF772BF2C
:107800009A9BFF1F024B1888183800B2FFF76ABF17
:10781000C89BFF1F024B1888183800B2FFF762BFE1
:10782000C69BFF1F024B1888183800B2FFF75ABFDB
:10783000BE9BFF1FC3681888183800B2FFF752BFFD
:10784000054B1B881BB9054B186808607047084634
:107850000422034909F072BDA49DFF1F20250100E9
:107860001C250100054B1B881BB9054B18680860D7
:10787000704708460422034909F060BDEE9BFF1FD4
:10788000202501001C25010030B5134C85B00125D1
:107890002B463C2202212046009503F05DFD204648
:1078A00003F034FF00224021802320460191009301
:1078B00011460A4B029504F0D7FB204604F032F83B
:1078C00007480849084A0023036083800B608B80C7
:1078D0001360938005B030BD489EFF1FD02B010080
:1078E000289EFF1F409EFF1FB09EFF1F10B500EB9C
:1078F000C00000F10F02D2B293B284B09C1E981C5B
:107900003D2303918DE819003921024804F010FB52
:1079100004B010BD489EFF1F014B01221A70704732
:10792000399EFF1FF0B56B4B6B4C6C4F6C4E6D4D21
:1079300085B004228DE80C00029320466A4B402259
:10794000802103F011FB2046684A6949694C08F020
:1079500075FE6949694A8F61694FCF61694F9761C7
:10796000694B6A4FD7616A4F9F616A4FDF616A4F07
:10797000B7616A4FF7616A4FAF616A4FEF616A4F53
:10798000A7616A486A4FE7616A4F87616A496B4F2E
:10799000C7616B4F8F616B4A6B4FCF616B4F9761C4
:1079A0006B4B6C4FD7616C4F6C4E9F616C4FDF61BE
:1079B0006C4F6D4DB7616D4FF7616D4F6D4CAF61A1
:1079C0006D4FEF616D4F6E48A7616E4FE7616E4F6F
:1079D0006E4987616E4FC7616E4F6F4A8F616F4FFF
:1079E000CF616F4F6F4B97616F4FD7616F4F9F6143
:1079F0006F4E704FDF61704FB761704D704FF76120
:107A0000704FAF61704C714FEF61714FA76171485A
:107A1000714FE761714F87617149724FC761724F52
:107A20008F61724A724FCF61724F9761724B734F81
:107A3000D761734F9F61734E734FDF61734FB761AF
:107A4000734D744FF761744FAF61744C744FEF61B5
:107A5000744F7548A761754FE761754F7549876128
:107A6000754FC761754F764A8F61764FCF61764FFC
:107A7000764B9761764FD761764F774E9F61774F00
:107A8000DF61774F774DB761774FF761774F784C6C
:107A9000AF61784FEF6178487849794F794DA761A8
:107AA000E561794F794D7A4CDFF808E2794A7A4BF3
:107AB0008761C5618C61794E794F7A4D7A4CC1F8F6
:107AC0001CE07A487A499761D5619C61D861B160C0
:107AD00005B0F0BD40420F00489EFF1FF577000043
:107AE000088CFF1FCC8EFF1F6890FF1F1C89FF1F93
:107AF000C1AF0000108AFF1FEC89FF1FA88EFF1F77
:107B00005D650000E5770000188EFF1F69650000C5
:107B1000C1670000C5750000E9670000E975000055
:107B2000116800000D760000D5770000988CFF1FCB
:107B30007965000039680000288DFF1F317600004C
:107B4000856E0000748CFF1F89650000616800006D
:107B5000048DFF1F55760000C1770000E08CFF1FE9
:107B6000996A0000B16A0000848EFF1FA56A0000B8
:107B7000B96E00009C8BFF1FD16D0000ED6E000000
:107B8000388FFF1F79760000F5700000508CFF1FC2
:107B90009D760000096B0000588BFF1F996500005F
:107BA00089680000A48FFF1FC17600005D7100008E
:107BB0002C8CFF1FA9650000C57100004C8DFF1FB4
:107BC000B965000035720000E48BFF1FC965000035
:107BD000696B0000C88AFF1FD9650000296F00008B
:107BE000348AFF1FE9650000C16B0000BC8CFF1FD9
:107BF000F965000031740000608EFF1F0966000007
:107C0000616F00002890FF1F196600009D72000040
:107C1000F48DFF1F2966000005730000EC8AFF1F2A
:107C200039660000956F00005C8FFF1FF16D00004A
:107C30006D7300003C8EFF1F496600004177000015
:107C4000108BFF1F59660000CD6F0000A48AFF1F34
:107C50006966000035700000F88FFF1F796600002C
:107C6000196C0000C08BFF1F89660000716C00005A
:107C70007C8AFF1F99660000348BFF1FF08EFF1F68
:107C8000C96C0000A9660000216D0000B966000003
:107C9000796D0000588AFF1FC889FF1F1C90FF1FC5
:107CA000DD730000D96600000D740000E966000075
:107CB0003D820000C9660000F0B5461C83B00D4649
:107CC0000127032336B22AB2044631468DE88800E4
:107CD0002448ADB204F0C2F80C23AA1C12B20093DF
:107CE0000197052321B21F4804F0B8F81E4A1F4B24
:107CF00012881B68BA422AD023D3022A10D11C4C06
:107D0000A3F6CA0384FB03241C44DB17C3EB24142F
:107D10000A2CA8BF0A2424EAE474A2B223B202E027
:107D200000231A461C460D35AA1A01200093019023
:107D300012B2314603230B4804F00EF8204603B07C
:107D4000F0BD0C4CA3F6FC0384FB0324DDE7084CD8
:107D5000A3F6980384FB03241C44DB17C3EBE40461
:107D6000D6E700BF489EFF1F249DFF1F889DFF1F71
:107D7000898888881F85EB512DE9F0438FB283B045
:107D8000DFF84C80BD1D461D2DB204B236B24FF057
:107D900001090AB22346314640460095CDF80490C9
:107DA00004F00CF82A463346214640468DE820026E
:107DB00004F004F807F10C020095334612B2214694
:107DC000CDF80490404603F0F9FF03B0BDE8F0831E
:107DD000489EFF1F2DE9F043804685B0002956D10B
:107DE0000121304804F080FB2F4998F8062098F8CC
:107DF000083011F80290994522DA4FEA89064D467B
:107E00000C24D8F80C3027489B595F6822B2002117
:107E100004F066FB384609F0D3F93946024621489A
:107E200004F0F8FC1F4804F00BFD98F80830013509
:107E30000934AB42A4B206F1040601DD422CE0D1C4
:107E4000B9F1000F13D109F1060999450CDA3C2369
:107E500001213B22039102930093019239233F2297
:107E60003A21104804F064F805B0BDE8F0830F2310
:107E700001213B22039102930093019239230C22AA
:107E80003A21084804F054F898F80830DBE700215C
:107E90003423009301913F230C22024803F05CFF3E
:107EA0009EE700BF489EFF1F409EFF1F10B5104C6D
:107EB0000121204604F01EFB2046012104F014FBA2
:107EC00020463422552104F00BFB204602220949AA
:107ED00004F0A0FC20460522074904F09BFC204644
:107EE00004F0AEFC2046BDE8104003F01BBD00BF0F
:107EF000489EFF1FD4250100D825010070B50D460E
:107F0000064609F05DF900EB40008400002D36D0F4
:107F1000284609F055F900EB4000400023185B109B
:107F200003F16001091A282209B21748C3F160045D
:107F300004F0D6FA0121144804F0D6FA284609F0D4
:107F40003FF929460246104804F064FC0E4804F04C
:107F500077FC02210C4804F0C7FA21B221220A481A
:107F600004F0BEFA304609F02BF9314602460648C5
:107F700004F050FC0448BDE8704004F061BC64109B
:107F8000C4F16004E5E700BF489EFF1F184B70B5C1
:107F9000B3F9003083EAE374A4EBE374002B82B0FE
:107FA000A1B21EDB68466D46012300E0134603EBD9
:107FB000830252009442F9DA0E4E91FBF3F286FBF3
:107FC00003E403FB1211DB173032D3EBA40389B2B5
:107FD00005F8012BF1D119462B70FFF78FFF02B086
:107FE00070BD2D238DF800300DF101056846DBE7EB
:107FF000409DFF1F6766666610B50D4B1B5C51F810
:108000002340237884B013B1012004B010BD04AA2A
:1080100001A942F8103D2046A3699847A38A9B070F
:10802000F2D401A80099FFF769FF012004B010BD48
:10803000289EFF1F2DE9F04F2F4DDFF8CCB0DFF861
:10804000C4A0DFF8C8900FCD91B003AC0FC40FCD22
:108050000FC40FCD0FC42B6823600025A8462F4600
:108060002E4600E09846BAF8003024495BF82320F9
:1080700028461123F8F702FB00EBC00400EB840054
:1080800089FB00340444C017C0EB6434C4F13C00E5
:10809000C6F13C0207F14101012600B208F141039B
:1080A00000901BB2019612B209B2154803F086FE89
:1080B00008EB060305F211153C2B2646ADB24746E8
:1080C000D0D134226B210E4804F00AFA00210C486A
:1080D00004F00AFA0B4B1B8810AA02EB830353F837
:1080E000344C204609F06CF802460548214611B090
:1080F000BDE8F04F04F08EBB1C220100141C0100EF
:10810000489EFF1FB29BFF1FD0190100090002808B
:1081100010B5424C424882B003F0F8FA2378C3B954
:1081200006213F4804F0E0F92378012B37D90A22D1
:10813000022B11463A486BD004F0D2F93949032298
:10814000374804F067FB364802B0BDE8104004F041
:1081500077BB354B1A7801210523002A35D10191CF
:10816000009311462E4803F079FE304B1A78002A0E
:1081700036D0052301220192009300220A212848CB
:1081800003F0EAFD2A4B1A78002A35D10121052394
:10819000019100931421224803F060FEC0E7254CB2
:1081A0002388092B32D9632B8CBF0A211F210A2275
:1081B0001B4804F095F92188194804F091FB1848F0
:1081C00002B0BDE8104004F03BBB002201910093D7
:1081D0001146134803F0C0FD144B1A78002AC8D189
:1081E00005230121019100930A210D4803F036FE79
:1081F0000F4B1A78002AC9D001220523019200935F
:1082000000221421064803F0A7FD89E73021CEE7BC
:1082100004F066F90322084992E700BFC39EFF1FDE
:10822000489EFF1FE4250100189EFF1F199EFF1F97
:10823000C89DFF1FC49DFF1FE0250100F8B56D4DCF
:10824000287840B96C4B1B6899425CD36B4A012378
:1082500013702B70F8BD0C4600266948664F03F07A
:1082600055FA04F6AC53324665483B6031212E7016
:1082700004F036F901216248624D04F03BF93146C1
:108280005F4804F031F905225F495D4804F0C2FA05
:108290005B4804F0D5FA0C221021594804F020F96B
:1082A0000B225A49564804F0B5FA05225849544859
:1082B00004F0B0FA524804F0C3FA564B50481C6818
:1082C000A4F69803C3EB031385FB03251D4410217B
:1082D000DB172022C3EB652504F002F940F6CC330E
:1082E0009C4205F124054FF022014FF004000BDC05
:1082F000FFF7E2FC484B1C88064674B3012C46D0BD
:10830000022C41D00120F8BDFFF736FD0922434978
:108310003B4804F07FFA2A221021394804F0E0F8A3
:108320003F4C374884FB0534EB17C3EBA4042146CC
:1083300004F0D6FA01223B49314804F06BFA04EB11
:108340008401A5EB41012E4804F0CAFA0122364906
:108350002B4804F05FFA0120F8BD34491022284868
:1083600004F058FA264804F06BFA2A221021244817
:1083700004F0B6F83146224804F0B2FA07222C493C
:108380001F4804F047FACBE70C222A49E7E70C2202
:1083900029491B4804F03EFA194804F051FA2A22F0
:1083A0001021174804F09CF8314615481C4E04F083
:1083B00097FA07221E49124804F02CFA86FB05366C
:1083C000EB17C3EBA60631460D4804F089FA2246A6
:1083D00014490B4804F01EFA06EB8601A5EB410197
:1083E000074804F07DFA22460F49054804F012FAC6
:1083F0002046F8BDA08AFF1F309EFF1FC09EFF1FB2
:10840000489EFF1F3B773B98E8250100F0250100BF
:10841000D8250100889DFF1F249DFF1FFC2501001A
:108420006766666684310100FC30010008260100A1
:108430001C26010034260100242601002DE9F0410C
:10844000754C2278002A05460F4614BF4FF00108EC
:108450004FF000084ED1714E3368CB1AB3F5FA6F66
:1084600004D86B78A3B94046BDE8F0816C4B6D48E9
:108470006D49DFF8D0E11A70012303700988237079
:1084800026208EF8002000F0F1FD6B78002BEAD05A
:108490003760F9F787FC654A654B6649127828789A
:1084A0001B78097802EB4303421E03EB81030E2A7B
:1084B000D9D801A151F822F0A985000075850000E6
:1084C00067840000A98500006784000067840000BD
:1084D000678400005D850000678400000F85000050
:1084E00067840000678400006784000067840000E0
:1084F0000B850000AF215048484E02F0B7FEFFF751
:1085000007FE002337602370ABE705F09BFB4A486A
:1085100003F0FCF80221484803F0E6FF0F22232174
:10852000454803F0DDFF05224449434804F072F951
:10853000414804F085F91E2223213F4803F0D0FF73
:1085400005223F493C4804F065F93B4804F078F9BE
:10855000394803F0E7F900F0ADFC84E7394D2B789A
:10856000012B50D9304B2620198800F07FFD0023C5
:108570002B7078E7002B3FF476AF013B324A32F89C
:108580001330002B3FF46FAF274C304825492D4A5C
:1085900023804FF001080023037081F8008082F8E7
:1085A0000080FFF7B5FD5EE793B1013B264A32F844
:1085B000131019B31C4B254D1A4C224A1980002662
:1085C000012326202E702370137000F04FFD15E05C
:1085D000154C1E4922880B7004284FF6FF7002F1DB
:1085E000FF310CBF012202460A440E4E154D02F027
:1085F0007F0201320121228031702B70FFF788FD4C
:108600004FF001082FE70649064A012300200870B1
:1086100013702370A6E700BFA08AFF1FBC9EFF1F38
:10862000C09EFF1FA09BFF1FC49DFF1F189EFF1F22
:10863000199EFF1FC89DFF1F489EFF1F4426010073
:108640004C260100C39EFF1F049DFF1F009CFF1FBF
:108650002DE9F04F05468BB00F46AD480121164677
:1086600003F048FFAA8812F0010440F0B080DFF860
:10867000CC8298F80030002B7DD1AB79A54AD15C33
:10868000A1B9DFF8BCA279781AF8039041B3397820
:108690000139072900F2B780DFE811F0F100540139
:1086A000B5006C01B500B500B500E9007C78002C80
:1086B00000F0CA800139EC68387854F82170FC6801
:1086C000411EB4F80080072900F2A780DFE811F00E
:1086D00074015901A5006C01A500A500A5009F002B
:1086E000DFF854A2DAF80020B21AB2F5967F75D9F5
:1086F000894A107801281ABF012010701170874A2A
:1087000018BF0146D05CC0EB0900C0B2FFF7EEF81D
:108710000124CAF80060AB889B0770D57B78002BDA
:108720006DD0F9F73FFB7E4B7E4A7F481B7812786D
:1087300039780078022515FB02330A2903EB800300
:1087400000F04E810C295AD1002B58D003F11900AA
:10875000764E774A013B0021400080B226F8131084
:108760000123157088F8003000F080FC714B032263
:1087700020461A702FE0664802F0C8FF01216448C5
:1087800003F0B2FE62482246214603F0A9FEAB8800
:10879000580725D42C68204608F012FD21460246D1
:1087A0005B4804F037F85A4804F04AF809220123DC
:1087B0008DE80C0000217F23554803F0FFFA0021CB
:1087C0002846FFF707FB002388F8003055E7AB6821
:1087D0003146384698470BB0BDE8F08F0846FAE7B7
:1087E0002B6804A8984704A808F0EAFC04A90246EC
:1087F000474804F00FF8464804F022F8D6E7204630
:108800000BB0BDE8F08F00240AF8039083E7002145
:10881000D1543846FB699847FC68A4F800800027CB
:1088200025223C238DE8840041211822384803F09A
:1088300093FAE968A879FFF7DFFB374A3E4B1770D8
:108840001E600BB0BDE8F08F3B490A68B21AB2F562
:10885000967FD4D9304F0E603E78012E00F0B48060
:10886000E968184601233B70FFF7C6FBB3E7304ABF
:10887000E9791170012288F800200024C4E72A7ADF
:10888000013A4A45BFDD09F10104E4B2A145BAD07D
:10889000224E16F803B0CBEB0900C0B20021FFF75F
:1088A00025F82B7A052BD9461BD9CBEB0402042AD9
:1088B00040F3AE80A4F1040BBBF1000FC0F2B08016
:1088C000063B5B45A8BF5B465FFA83F9AA7913486C
:1088D000B15C994205D000F8029001212846FFF7CB
:1088E00079FAC9EB0400C0B201210B4EFEF7FEFF7E
:1088F00000213423019100930548317040230B225D
:108900003F21A14603F028FA0124AB797CE700BFA0
:10891000489EFF1FB09EFF1FC19EFF1F409EFF1F6E
:10892000189EFF1F199EFF1FC89DFF1F049DFF1F5C
:10893000C09EFF1FC39EFF1FAC9EFF1FA08AFF1F8C
:10894000289EFF1F0FFA89F1E868604C50F82160FB
:108950002168049134785E4904980860002C71D035
:10896000012C7FF450AF5B4A317A88F800401170D7
:10897000002449E7B9F1000F50D009F1FF34E4B207
:1089800084E7B98A01F0040189B200293FF440AFBD
:108990003B6A03929847039A00283FF43DAFAB79B6
:1089A000FC680021D15438E77B8A43453CD908F163
:1089B00001081FFA88F830E73B8A43453BD208F1AB
:1089C000FF381FFA88F828E725238DE81800424869
:1089D0003C703C231822412103F0BEF93046FAE6F0
:1089E000002B3FF40CAF3D4A3D4E1188394A03F14C
:1089F0001900013B400080B226F81310012388F8CB
:108A00000030157000F032FB364B20461D70E2E658
:108A1000002A3FF755AF04F1FF3B4DE74C46F3E624
:108A20004FF000094B4651E7BB8ADA077FF5F5AEF8
:108A3000B7F81080F1E6BB8AD9077FF5EEAEB7F83C
:108A40001280EAE62849C85CC0EB090009F1010E72
:108A5000C0B201214FF0340B02F803E0FEF746FFED
:108A6000B6681D48019440230B223F210124CDF814
:108A700000B003F071F940230B223F211648CDF8D6
:108A800000B0019403F0EAF92146134803F02CFDED
:108A9000304608F095FBA0EB800000F15F0109B2C1
:108AA0000F220D4803F01CFD304608F089FB3146CB
:108AB0000246094803F0AEFE074803F0C1FEE9682C
:108AC000A879FFF799FAAB799EE600BF009FFF1FD8
:108AD000AC9EFF1FC09EFF1F489EFF1FC49DFF1F2F
:108AE000049DFF1FC39EFF1F409EFF1F2DE9F047FF
:108AF000DFF808926D4B99F800601B68DFF800A260
:108B000082B0003601934FF0030018BF0126019F89
:108B10009AF8008004F04EFD0546042004F04AFD5A
:108B20000446052004F046FD800040EA4404062087
:108B300004F040FD2C4364B25D4944EAC0000A7869
:108B400080F00F03DBB29A425A4A3CD017600022F1
:108B500059480B7003788DF800808DF8012053B3CD
:108B6000564A12684EF66021BA1A8A4219D8022B68
:108B700059D0012B5FD0062B48D0032B63D0042B98
:108B800069D0052B77D0072B7DD0082B00F0838090
:108B9000092B68D016B14A4802F0C4FE02B0BDE805
:108BA000F087484A484C002301212370037013606A
:108BB000938089F800103A4669464448FFF748FD1B
:108BC0003043C6B2E6E71268BA1A1E2A6BD99AF881
:108BD0000020934222D0394C3D488AF80030012BC6
:108BE000276082EA030207609846B1D0042BAFD118
:108BF00037480068381AB0F5C87FA9D9354C2068C5
:108C0000381A3228A4D927601A46A1E73A4669469D
:108C10003148FFF71DFD3043C6B2BBE7012B4FF0D3
:108C20000002E3D1E4E73A4669462C48FFF710FD1D
:108C30003043C6B2AEE73A4669462948FFF708FD19
:108C40003043C6B2A6E73A4669462648FFF700FD1C
:108C50003043C6B29EE73A4669462348FFF7F8FC20
:108C60003043C6B296E73A4669462048FFF7F0FC23
:108C70003043C6B28EE73A4669461D48FFF7E8FC26
:108C80003043C6B286E73A4669461A48FFF7E0FC29
:108C90003043C6B27EE73A4669461748FFF7D8FC2C
:108CA0003043C6B276E7002252E700BF009FFF1FA5
:108CB000C49EFF1F349EFF1FC09EFF1FB89EFF1F54
:108CC000489EFF1FB09EFF1FC29EFF1F5824010039
:108CD000C89EFF1F3C9EFF1F88240100B023010097
:108CE000B42201005030010040300100A4220100F4
:108CF0000C230100942301001C90FF1FA08AFF1F7A
:108D0000389EFF1F28B11028044BA8BF1020186000
:108D10007047024B01201860704700BFCC9EFF1FB8
:108D200038B50F4D2B78013B01381B02C4B203F458
:108D30007063200443F4404343F00C0300F4FE004E
:108D4000184305F09FFD2868013860F03F00C0B26D
:108D500004F0C6FD2046BDE8384004F0C1BD00BFA8
:108D6000CC9EFF1F70B5124D2B78013B1B0203F404
:108D70007063064643F430430806320400F0FE40B8
:108D800043F00B03034302F4FE0018430C4605F0C6
:108D900079FD2868013860F04F00C0B204F0A0FDF2
:108DA000304604F09DFD2046BDE8704004F098BDBB
:108DB000CC9EFF1F70B5124D2B78013B1B0203F4B4
:108DC0007063064643F410430806320400F0FE4088
:108DD00043F00903034302F4FE0018430C4605F078
:108DE00051FD2868013860F06F00C0B204F078FDD2
:108DF000304604F075FD2046BDE8704004F070BDBB
:108E0000CC9EFF1F38B5104D2B78013B1B0203F49D
:108E10007063044643F41043000443F0090300F474
:108E2000FE00184305F02EFD2868013860F06F0041
:108E3000C0B204F055FD204604F052FD0020BDE80C
:108E4000384004F04DBD00BFCC9EFF1F38B50E4D1D
:108E50002B78013B1B0203F47063044643F4504338
:108E6000000443F00D0300F4FE00184305F00AFD72
:108E70002868013860F02F00C0B204F031FD2046B0
:108E8000BDE8384004F02CBDCC9EFF1F08B5002083
:108E900005F0C2FD0028FAD108BD00BF08B5642165
:108EA0000720FFF75FFF7F210B20BDE80840FFF799
:108EB00059BF00BF10B500217B20FFF753FF0024EE
:108EC000E0B2FFF79FFF0134022004F0A9FB802CE1
:108ED000F6D110BD10B504464FF4406004F0B0FC6C
:108EE00004F008FD2CB1102C044BA8BF10241C600A
:108EF00010BD024B01241C6010BD00BFCC9EFF1FA3
:108F000010B5044641F0E00004F0EAFC04F07F00F4
:108F100004F0E6FCC4F3C610BDE8104004F0E0BC69
:108F200038B5134D2B78044641F6FF72A0F500507A
:108F3000824203F1FF33A8BF02461B0202F5005232
:108F400003F47063100443F4604343F00E0300F431
:108F5000FE005204184302F0FE42104305F092FC5A
:108F6000296801392046C9B2BDE83840FFF7C8BFBB
:108F7000CC9EFF1F38B504460D46F02004F0B0FC2F
:108F800035B1254414F8010B04F0AAFCAC42F9D128
:108F9000F720BDE8384004F0A3BC00BF00B50B4B80
:108FA00083B00246998818680090032AADF804102F
:108FB00002D903B05DF804FB684606218DF8052050
:108FC000FFF7D8FF03B05DF804FB00BFBC30010021
:108FD00000B50B4B024683B0186899880090131FA8
:108FE0004C2BADF8041002D903B05DF804FB6846C1
:108FF00006218DF80520FFF7BDFF03B05DF804FBE7
:10900000C4300100030203F4FE43C0F3C61018434A
:10901000704700BF03784078DB0103F47E5300F013
:109020007F001843704700BF82B002AA114642F881
:10903000040D002012F8013B03F07F03914243EA44
:109040000020F7D102B07047003210B403884FF00F
:10905000010404FA01F418BF012202FA01F123EA23
:1090600004020A43028010BC704700BF70B5CEB244
:109070000C46054603F066FE864203D0314628467C
:1090800003F07AFE0135284603F05CFE240A844290
:1090900005D021462846BDE8704003F06DBE70BD86
:1090A00038B5054603F04EFE4FF0000460F30704A8
:1090B000681C03F047FE60F30F24A0B238BD00BF68
:1090C000F8B504460020FFF7EBFF002C00F06781A5
:1090D0004FF4AF610220FFF7C9FF04204FF47A611B
:1090E000FFF7C4FF0B2004F065FA002840F0C286A9
:1090F0004FF496610620FFF7B9FF4FF4FA6108209C
:10910000FFF7B4FF4FF4FA610A20FFF7AFFF40F614
:10911000B8310C20FFF7AAFF4FF42F612220FFF790
:10912000A5FF40F6AC512420FFF7A0FF7D212A20A7
:10913000FFF79CFF0C210E20FFF798FF0121102064
:10914000FFF794FF02211220FFF790FF0021142067
:10915000FFF78CFF00211620FFF788FF022118205F
:10916000FFF784FF01211A20FFF780FF01211C2057
:10917000FFF77CFF04211E20FFF778FF1421202039
:10918000FFF774FF01212620FFF770FF032128203D
:10919000FFF76CFF04212C20FFF768FF14212E201D
:1091A000FFF764FF00213020FFF760FF0C21322021
:1091B000FFF75CFF00213420FFF758FF0021362025
:1091C000FFF754FF00213820FFF750FF00213A201D
:1091D000FFF74CFF00213C20FFF748FF00213E2015
:1091E000FFF744FF00214020FFF740FF002142200D
:1091F000FFF73CFF1F214420FFF738FF13214620D3
:10920000FFF734FF0E214820FFF730FF11214A20DD
:10921000FFF72CFF0A214C20FFF728FF00214E20EA
:10922000FFF724FF06215020FFF720FF02215220E4
:10923000FFF71CFF0C215420FFF718FF00215620D8
:10924000FFF714FF00215820FFF710FF01215A20DB
:10925000FFF70CFF08215C20FFF708FF0A215E20C2
:10926000FFF704FF00216020FFF700FF04216220C8
:10927000FFF7FCFE01216420FFF7F8FE00216620C5
:10928000FFF7F4FE0B216820FFF7F0FE7F216A2034
:10929000FFF7ECFE00216C20FFF7E8FE00216E20B6
:1092A000FFF7E4FE00217020FFF7E0FE00217220AE
:1092B000FFF7DCFE00217420FFF7D8FE1F21762087
:1092C000FFF7D4FE13217820FFF7D0FE0E217A207D
:1092D000FFF7CCFE11217C20FFF7C8FE0A217E207B
:1092E000FFF7C4FE1F218020FFF7C0FE132182205C
:1092F000FFF7BCFE0E218420FFF7B8FE1121862067
:10930000FFF7B4FE0A218820FFF7B0FE00218A2073
:10931000FFF7ACFE00218C20FFF7A8FE002196206D
:10932000FFF7A4FE00219820FFF7A0FE00219A205D
:10933000FFF79CFE05219C20FFF798FE06219E204A
:10934000FFF794FE0021A020FFF790FE7F21A220CE
:10935000FFF78CFE40F2A461A420FFF787FE4FF4D4
:10936000E161A620FFF782FE0021A820FFF77EFE24
:109370000021AA20FFF77AFE29210020FFF776FEC0
:109380000220FFF78DFEB0F5805F034616D34FF441
:10939000AF610220FFF76AFE4FF4AF630EE04FF6B5
:1093A000FF7398423FF494AE292840F0858502204F
:1093B000FFF776FEB0F5805F0346E8D2D24A04207C
:1093C0001380FFF76DFEB0F5805F034680F03D85AA
:1093D000CE4A06201380FFF763FEA0F52F739BB2E1
:1093E000B3F57A6F024606D940F628210620FFF72A
:1093F0003DFE40F62822C64B08201A80FFF750FE9B
:10940000A0F52F739BB2B3F57A6F024606D940F6EA
:10941000E4410820FFF72AFE40F6E442BD4B0A2053
:109420001A80FFF73DFEA0F5FA739BB240F6AC51EF
:109430008B42024606D94FF4FA610A20FFF716FE66
:109440004FF4FA62B44B0C201A80FFF729FEA0F506
:10945000FA739BB240F6AC518B42024606D940F6F5
:10946000B8310C20FFF702FE40F6B832AB4B0E20AD
:109470001A80FFF715FE1828034600F2DF84A84A79
:1094800010201380FFF70CFE431E9BB20F2B0246E9
:1094900004D901211020FFF7E9FD0122A14B122080
:1094A0001A80FFF7FDFD0A28034600F2C0849E4A99
:1094B00014201380FFF7F4FD0128034604D900218E
:1094C0001420FFF7D3FD0023984A16201380FFF7DE
:1094D000E7FD7F28034600F2A384954A18201380F5
:1094E000FFF7DEFD0528034600F29384914A1A2017
:1094F0001380FFF7D5FD0C28034600F283848E4AC3
:109500001C201380FFF7CCFD0428034600F273846F
:109510008A4A1E201380FFF7C3FD0928034600F284
:109520006384874A20201380FFF7BAFD462803464C
:1095300000F25384834A22201380FFF7B1FDA0F587
:10954000FA739BB240F6AC518B42024606D94FF4F7
:109550002F612220FFF78AFD4FF42F627A4B2420DF
:109560001A80FFF79DFDA0F5FA739BB240F6AC544C
:10957000A342024604D921462420FFF777FD224664
:10958000724B26201A80FFF78BFD7F28034600F2DE
:109590001D846F4A28201380FFF782FD06280346AA
:1095A00000F20D846B4A2A201380FFF779FDA0F1A9
:1095B00032039BB2B3F5967F024604D97D212A205F
:1095C000FFF754FD7D22644B2C201A80FFF768FDC5
:1095D0000C28034600F2ED83604A2E201380FFF72B
:1095E0005FFD1E28034600F2DE835D4A30201380B3
:1095F000FFF756FD0928034600F2CF83594A32206F
:109600001380FFF74DFD1E28034600F2C083564A23
:1096100034201380FFF744FD7F28034600F2B18316
:10962000524C36202380FFF73BFD7F28034600F293
:10963000A28338206380FFF733FD7F28034600F2C2
:1096400094833A20A380FFF72BFD7F28034600F286
:1096500086833C20E380FFF723FD7F28034600F24A
:1096600078833E202381FFF71BFD7F28034600F20D
:109670006A8340206381FFF713FD7F28034600F2D1
:109680005C834220A381FFF70BFD394D28804420E5
:10969000FFF706FD3028034600F24983354A46208D
:1096A0001380FFF7FDFC3028034600F23A83324C6A
:1096B00048202380FFF7F4FC3028034600F22B8378
:1096C0004A206380FFF7ECFC3028034600F21D833C
:1096D0004C20A380FFF7E4FC3028034600F20F8300
:1096E0004E20E380FFF7DCFC0128034604D900216B
:1096F0004E20FFF7BBFC0023204A50201380FFF7C9
:10970000CFFC431E3CE000BF2C9CFF1FE89DFF1FC9
:10971000AC9DFF1FC09DFF1F8C9DFF1FC49BFF1FA3
:109720009A9BFF1F409DFF1F769DFF1F229CFF1FDE
:109730009E9BFF1F329CFF1FDC9BFF1FD69BFF1FC2
:10974000CC9BFF1FD09DFF1F389DFF1F349DFF1F27
:10975000C49DFF1F989DFF1FE09DFF1FB29BFF1F31
:109760001C9CFF1FF89DFF1FC29DFF1F049DFF1F34
:10977000BC9BFF1FBE9BFF1F9C9DFF1FD49BFF1F19
:109780009BB20B2B024604D906215020FFF76EFC3A
:109790000622CF4B52201A80FFF782FC0428034692
:1097A00000F2A782CB4A54201380FFF779FC431EB6
:1097B0009BB21D2B024604D90C215420FFF756FC06
:1097C0000C22C54B56201A80FFF76AFC012803467D
:1097D00004D900215620FFF749FC0023BF4A582036
:1097E0001380FFF75DFC7F28034600F27C82BC4AB1
:1097F0005A201380FFF754FC431E9BB2092B0246EC
:1098000004D901215A20FFF731FC0122B54B5C201D
:109810001A80FFF745FC431E9BB2102B024604D969
:1098200008215C20FFF722FC0822AF4B5E201A8043
:10983000FFF736FC431E9BB21D2B024604D90A21BA
:109840005E20FFF713FC0A22A84B60201A80FFF766
:1098500027FC0228034600F24082A54A64201380B8
:10986000FFF71EFC0128034604D901216420FFF7FD
:10987000FDFB01239F4A62201380FFF711FCC31EEA
:109880009BB2012B024604D904216220FFF7EEFBB4
:109890000422994B66201A80FFF702FC7F280346BA
:1098A00000F21582954A68201380FFF7F9FB7F28A4
:1098B000034600F20682924A6A201380FFF7F0FB0B
:1098C0007F28034600F2F7818E4A6C201380FFF751
:1098D000E7FB0228034600F2E8818B4A6E201380E2
:1098E000FFF7DEFB1928034600F2D981874A702072
:1098F0001380FFF7D5FB0228034600F2CA81844A91
:1099000072201380FFF7CCFB0628034600F2BB81D0
:10991000804A74201380FFF7C3FB0528034600F23A
:10992000AC817D4A8A201380FFF7BAFB0A280346E0
:1099300000F29D81794A8C201380FFF7B1FB042847
:10994000034600F28E81764A98201380FFF7A8FB29
:109950000128034604D900219820FFF787FB002344
:10996000704A9A201380FFF79BFB0128034604D915
:1099700000219A20FFF77AFB00236B4A9620138080
:10998000FFF78EFB0B28034600F26581674A9C2097
:109990001380FFF785FB831E9BB2032B024604D97D
:1099A00005219C20FFF762FB0522614B76201A807F
:1099B000FFF776FB3028034600F247815D4A7820A6
:1099C0001380FFF76DFB3028034600F238815A4CB4
:1099D0007A202380FFF764FB3028034600F22981B8
:1099E0007C206380FFF75CFB3028034600F21B817C
:1099F0007E20A380FFF754FB3028034600F20D8140
:109A00008020E380FFF74CFB3028034600F2FF8004
:109A10004A4A82201380FFF743FB3028034600F2B6
:109A2000F080474C84202380FFF73AFB3028034620
:109A300000F2E18086206380FFF732FB3028034686
:109A400000F2D3808820A380FFF72AFB302803464A
:109A500000F2C580A020E380FFF722FB0128034627
:109A600004D90021A020FFF701FB0023354A9E20E6
:109A70001380FFF715FBC31E9BB20C2B024604D9C3
:109A800006219E20FFF7F2FA06222F4BA2201A8011
:109A9000FFF706FB431E9BB27E2B024604D97F21B3
:109AA000A220FFF7E3FA7F22284BA4201A80FFF7B9
:109AB000F7FAA0F5AF639BB2B3F5167F024647D91C
:109AC00040F2A461A420FFF7D1FA40F2A4623FE083
:109AD0002089FF1F2E89FF1FA489FF1F109CFF1FD5
:109AE000869DFF1F949BFF1FA889FF1F2C89FF1FC6
:109AF000309DFF1F949DFF1FDE9BFF1FD29DFF1F08
:109B0000089CFF1FCE9BFF1F889BFF1F1A9EFF1FF5
:109B1000249DFF1FF49DFF1FB89DFF1F429DFF1F47
:109B20002E9DFF1FEE9BFF1F149CFF1F809DFF1F9C
:109B3000B49BFF1FC69BFF1F149DFF1FC89BFF1FE9
:109B40001C9DFF1FA49DFF1F9089FF1FC69DFF1F27
:109B5000CE4BA6201A80FFF7A3FAA0F5AF639BB205
:109B6000B3F5167F024606D94FF4E161A620FFF750
:109B70007DFA4FF4E162C64BA8201A80FFF790FAF5
:109B80000628034600F27081C24AAA201380FFF71C
:109B900087FA032800F262812B88DFF818E3BE4FB2
:109BA000BE4ABF4DBF4EC04CC04903F0010CAEF8D9
:109BB00000C0C3F3400EA7F800E0C3F3800717808E
:109BC000C3F3C007BA4A2F70C3F30017C3F340159D
:109BD000C3F38013378025800B801080F8BD0A21E5
:109BE0008820FFF743FA0A2334E711218620FFF784
:109BF0003DFA112326E70E218420FFF737FA0E23C2
:109C000018E713218220FFF731FA132309E71F21F8
:109C10008020FFF72BFA1F23FAE60A217E20FFF7A8
:109C200025FA0A23ECE611217C20FFF71FFA112305
:109C3000DEE60E217A20FFF719FA0E23D0E6132173
:109C40007820FFF713FA1323C1E61F217620FFF7D0
:109C50000DFA1F23B2E600219620FFF707FA002332
:109C600094E600218C20FFF701FA00236BE6002127
:109C70008A20FFF7FBF900235CE600217420FFF740
:109C8000F5F900234DE600217220FFF7EFF90023DC
:109C90003EE600217020FFF7E9F900232FE60021BE
:109CA0006E20FFF7E3F9002320E600216C20FFF788
:109CB000DDF9002311E67F216A20FFF7D7F97F2322
:109CC00002E60B216820FFF7D1F90B23F3E5002111
:109CD0006620FFF7CBF90023E4E500216020FFF7C1
:109CE000C5F90023B9E500215820FFF7BFF900238B
:109CF0007DE502215220FFF7B9F9022352E50A213E
:109D00004C20FFF7B3F90A23EAE411214A20FFF7B8
:109D1000ADF91123DCE40E214820FFF7A7F90E234B
:109D2000CEE413214620FFF7A1F91323BFE41F213E
:109D30004420FFF79BF91F23B0E400214020FFF7E8
:109D400095F900239DE400213E20FFF78FF90023C1
:109D50008FE400213C20FFF789F9002381E40021F2
:109D60003A20FFF783F9002373E400213820FFF73E
:109D70007DF9002365E400213620FFF777F9002301
:109D800057E400213420FFF771F9002348E40C2147
:109D90003220FFF76BF90C2339E400213020FFF764
:109DA00065F900232AE414212E20FFF75FF914231C
:109DB0001BE404212C20FFF759F904230CE40321B0
:109DC0002820FFF753F90323FFF7ECBB01212620DE
:109DD000FFF74CF90123FFF7DCBB14212020FFF72C
:109DE00045F91423FFF7A6BB04211E20FFF73EF917
:109DF0000423FFF796BB01211C20FFF737F901234D
:109E0000FFF786BB01211A20FFF730F90123FFF786
:109E100076BB02211820FFF729F90223FFF766BB62
:109E200000211620FFF722F90023FFF756BB02217D
:109E30001220FFF71BF90223FFF739BB0C210E207C
:109E4000FFF714F90C23FFF71ABB4FF47A610420D3
:109E5000FFF70CF94FF47A63FFF7BABAAA20002192
:109E6000FFF704F9002097E60021A820FFF7FEF88D
:109E7000002389E640F628210620FFF7F7F840F690
:109E8000E4410820FFF7F2F8FFF73CB9309CFF1FD0
:109E9000AE9DFF1F969BFF1FEC9BFF1F1E9CFF1F8D
:109EA000279DFF1F329DFF1F969DFF1F489DFF1F8F
:109EB000F29BFF1F829DFF1F17287FF609A9192813
:109EC0007FF678A91B287FF695A91C283FF4AAA93C
:109ED0001E287FF6AFA91F283FF4B4A920283FF41D
:109EE000CDA921283FF4D6A922283FF4DBA92328B5
:109EF0003FF4E4A924283FF415AA25283FF41AAA20
:109F000026283FF41BAA27283FF420AA28287FF4FC
:109F100033AAFFF729BA00BFF8B5BD2006F0C8FB89
:109F2000204B214A054603CB1368C5F803001A0CE1
:109F3000AC20C5F807102B80AA70FFF763F82E46F7
:109F4000002426F80B0FA0B2FFF7AAF8FFF75AF883
:109F50000234AC2C26F8020FF5D16C1E05F1B806C0
:109F60004FF0FF3014F8013F082758400F4B40F3E3
:109F700000017A1E0B4012F0FF0783EA5000F5D172
:109F8000B442EFD1C043FFF74FF83A46C5F8B900E5
:109F9000BD21284604F0C4FC2846BDE8F84006F080
:109FA0008FBB00BFD0300100CC3001002083B8ED62
:109FB000F0B50E4B0E4C054693E8070085B02468BB
:109FC0002E88AD7801AB83E80700270C18460022E5
:109FD0000B21ADF804408DF80670ADF80C608DF8DB
:109FE0000E5004F09DFC05B0F0BD00BFDC30010058
:109FF000CC300100F0B5124B124D1E68124F0FCD40
:10A0000087B06C460FC495E8030044F8040B386829
:10A010003B79CDF80D00320C292021808DF80220EB
:10A020008DF81130ADF80060FEF7ECFF0022ADF8BE
:10A030000B001221684604F073FC07B0F0BD00BFAE
:10A04000CC300100E8300100D8250100002004F0E8
:10A05000E3BC00BF02F02EBE70B5124C82B00025EA
:10A06000402306462946204600930195802320225E
:10A0700001F072FE20222946204602F031FA2046E5
:10A08000012102F037FA304607F09AF831460246CD
:10A09000204602F0BFFB204602B0BDE8704001F050
:10A0A00041BC00BF489EFF1FF0B5BC2983B075D9E5
:10A0B0000546441E00F1B8064FF0FF3014F8012F9A
:10A0C00008275040404A40F300017B1E0A4013F02D
:10A0D000FF0782EA5000F5D1B442EFD1C043FEF74A
:10A0E000A3FF0146D5F8B9000190019A914202D030
:10A0F000B2F17F2F0BD105F10B00FEF78BFFAC28DF
:10A100000BD03248FFF7A8FF002003B0F0BD304865
:10A11000FFF7A2FF384603B0F0BD05F10D00FEF7D2
:10A1200079FF292840D1002440F6AC5613E00428DA
:10A130001AD0062821D008281FD00A2828D00C2899
:10A1400022D1A1F5FA7292B2B24201D8FEF78EFF87
:10A150000234AC2C0ED004F10D002844FEF75AFF57
:10A16000022C0146A0B2E2D1B1F5805FEED30234F9
:10A17000AC2CF0D1012003B0F0BDA1F52F7292B24A
:10A18000B2F57A6FE4D8E1E7222801D0242811D172
:10A19000A1F5FA7292B2B242DAD8D7E70D48FFF7CA
:10A1A0005BFF002003B0F0BD0B48FFF755FF002018
:10A1B00003B0F0BD2A28C9D1A1F1320292B2B2F5A2
:10A1C000967FC5D8C2E700BF2083B8ED2C310100CF
:10A1D00018310100003101004031010003290CD980
:10A1E00070B5461C82B005460C46304603222A490B
:10A1F00007F054F810B102B070BD70470B2C05D9B0
:10A2000005222649281D07F049F840B12448FFF7E8
:10A2100023FF244802B0BDE87040FFF7C9BE05F136
:10A220000901032201A807F089F801A803221E49A9
:10A2300007F034F8D8B103221C4901A807F02EF822
:10A2400008B301A803221A4907F028F8B0B9194841
:10A25000FFF702FFA11E89B23046FFF725FF002855
:10A26000C9D0154802B0BDE87040FFF7F5BE1348ED
:10A27000FFF7F2FEFFF750FE1148F3E71148FFF732
:10A28000EBFE1148C6E71148FFF7E6FE02B0BDE855
:10A290007040FFF7AFBE00BFCC300100E8250100E1
:10A2A000583101006C31010070310100983101001A
:10A2B000B0310100B4310100C83101007431010036
:10A2C00088310100DC310100F03101009C310100D6
:10A2D0002DE9F043174D2B6883B081460F46904619
:10A2E000F3B1154E34880A1992B2184611463280DD
:10A2F00006F05CFD28603A464946204402F06CFDB9
:10A30000B8F1000F09D031882868FFF767FF286887
:10A3100006F0D6F900232B60338003B0BDE8F0834C
:10A32000054E01930846318006F0C2F9019B286072
:10A330001C46E0E7D49EFF1FD09EFF1F10B51F4CA8
:10A340004FF4FA70FBF79CFF204601F0DFF9002282
:10A350001146204602F0C4F82046012102F0CAF856
:10A360002046002102F0C0F80B221549204602F0D9
:10A3700051FA204602F064FA0F221249204602F0F8
:10A3800049FA204602F05CFA0F490722204602F003
:10A3900041FA204602F054FA204601F0C3FA0B4B72
:10A3A0000B4A1A604FF4FA70FBF76AFFFFF722FEC0
:10A3B0000848BDE81040FFF74FBE00BF489EFF1F92
:10A3C000F431010000320100103201008CA0FF1FA7
:10A3D000D1A20000183201000020704790F8392007
:10A3E00090F83800101A704790F8383090F83920FB
:10A3F0009A4205D95A1C034480F83820187E7047C9
:10A400004FF0FF30704700BF90F8383090F8392097
:10A410009A4286BF1B18187E4FF0FF30704700BF6E
:10A42000704700BF38B50546B0F85E0090B195F8AA
:10A430005D301446C3F1210294420CD805F13B0073
:10A440001844224602F0C8FC95F85D30234485F894
:10A450005D30204638BD012014462871EEE700BF6C
:10A46000B0F85E306BB190F85D30202B07D8C21881
:10A47000013380F85D30012082F83B1070470123E2
:10A4800003710020704700BF0023426980F8383014
:10A4900080F8393080F85C3080F85D3080F85E30CC
:10A4A00080F85F3006CA30B40D68046943662A43F9
:10A4B00083660A60A370426990F861301649146897
:10A4C00013441D7A5B7B01EBC5051B026D6803F429
:10A4D000E06343F064032B6090F8623013449D7C8A
:10A4E000DB7D01EBC5011B02496803F4E06343F027
:10A4F00064030B6021685368194205D00369272261
:10A500005A70036904229A71036920225A710369FF
:10A5100080229A7030BC70474C3D010043690CCBDF
:10A5200012681A420CD0094B99420AD9084B994239
:10A53000036994BF1A220D225A70036904229A718A
:10A540007047036927225A70F7E700BF7F1A060099
:10A550003F420F0010B50269D378DBB2D90604463A
:10A560003DD510215806D17038D503F0040303F00F
:10A57000FF02002B51D03D49626E00230B7084F81E
:10A580005D30002A5BD0904794F85D30002B56D0A8
:10A590002369D0229A70236994F83B201A712369A9
:10A5A000012284F85C200222DA7010BD304B84F85E
:10A5B00060009C424AD02F4B9C4252D094F83910F4
:10A5C00013791F29DBB207D82848007820B160181A
:10A5D000013184F8391003760223D37010BD590677
:10A5E000C3D4917801F0100101F0FF000029DDD003
:10A5F00013F001031ED194F85C1094F85D008842BA
:10A6000081BF4B1C091984F85C3091F83B30137101
:10A610002369D0229A702269DEE7236984F8392001
:10A62000C0229A702369114A1979012111700222FE
:10A63000DA7010BDC023937022691379CCE7012230
:10A64000002384F85D2084F83B30A1E7626994F828
:10A650006130094913440322187A02F043FD22694C
:10A66000ACE7626994F861300449F3E7D89EFF1FB4
:10A670006890FF1FD490FF1FDDA60000E9A6000030
:10A680000369DB7803F0200373B190F86030013385
:10A69000DBB2012B80F860301AD9426990F8613042
:10A6A0001344187A02F09ABD70B5426903F0FF05B1
:10A6B00090F8613013440446187A02F08FFDA36EBF
:10A6C0005BB184F8385094F83900BDE87040184701
:10A6D00090F85F30002BE0D0704770BD0148FFF765
:10A6E000CFBF00BF6890FF1F0148FFF7C9BF00BF81
:10A6F000D490FF1F2DE9F047374FDFF8E0903B681B
:10A70000026982B006460093DDF800800021A02592
:10A71000D3789B065BD53B680193019BC8EB030391
:10A720000F2BF5D949B1102BF2D00020907033696E
:10A7300080229A7002B0BDE8F087726996F86130A5
:10A7400013440521187A02F043FF726996F86130CC
:10A750001344012193F812A0504602F039FF092456
:10A760000021504602F020FF2B46013BFDD1012184
:10A77000504602F019FF2B46013BFDD1013CEFD1C1
:10A78000706996F8611001444FF4A0720C7A4B7B0B
:10A7900009EBC4011B02496803F4E06343F064035E
:10A7A0000B6096F862300344997CDB7D09EBC101B4
:10A7B0001B02496803F4E06343F064030B60013A51
:10A7C000FDD13269D3789B064FF00101A3D401205B
:10A7D00002B0BDE8F08700BF009FFF1F4C3D0100A5
:10A7E000F0B503691222DA700269937803F020034E
:10A7F00085B004460D46002B5ED0B42393703C49CF
:10A8000022690B680093009E05E00B680193019B91
:10A810009B1B042B42D8D37803F0200303F0FF00E6
:10A82000002BF2D094F85D30002B31D04FF0000EA9
:10A830004FF0020C04EB0E0393F83B3013710B68DE
:10A840000393039F206907E09B060DD50B680293D5
:10A85000029BDB1B052B28D8C378DBB203F0020276
:10A8600002F0FF06002AEFD080F803C02669F378D3
:10A87000DBB2DF0632462DD49F062BD5DB0731D461
:10A880000EF1010E94F85D305FFA8EFE7345D1D85B
:10A8900000201DBB002384F85E3004E09070236923
:10A8A00080229A70042005B0F0BD86702369802252
:10A8B00004209A7005B0F0BD03F0FF06FFF71AFF01
:10A8C00010B9042005B0F0BD236984F85F60B022A0
:10A8D0009A7094E78023B3700420DAE72669802316
:10A8E000B370D7E7BEF1000F0CBF02200320F6E7DC
:10A8F000009FFF1F2DE9F04106690025122780F80F
:10A90000385080F83950F770D0F810C09CF802E049
:10A910000EF0200E88B00446884615461E46BEF14D
:10A92000000F49D0B4238CF80230784B21691A68A3
:10A930000092DDF800E006E01A6801920198CEEB83
:10A940000000042830D8C87800F0200000F0FF078D
:10A950000028F1D04FEA480242F00102D2B20A7157
:10A960001A680292DDF808E0206906E01A6803928E
:10A970000399CEEB010105292AD8C17801F0020123
:10A9800001F0FF070029F1D04FF0020C80F803C05E
:10A990002269D17811F0110722D12DBB002E0CBFF6
:10A9A000A0238023937003E08F70236980229A7024
:10A9B000384608B0BDE8F0810EF0FF07FFF79AFEB9
:10A9C0000028F5D0236984F85F70B0229A70ACE754
:10A9D00087702369802238469A7008B0BDE8F081FC
:10A9E000802393700027E3E7012D75D0A02191709B
:10A9F00021690A79BE4667464FF0A80C1A6804928E
:10AA0000049805E01A680592059A121A052A4AD890
:10AA1000CA7802F0020202F0FF08002AF2D0CF70DA
:10AA20002169CA78D2B212F0100F08465AD19206A4
:10AA300058D5013DEDB2012D49D0BEF11F0F3BD9D4
:10AA40000A79012DDAD11A680692069D05E01A6886
:10AA50000792079A521B052A46D8C27802F00202D2
:10AA600002F0FF01002AF2D00223C3702269D378DA
:10AA7000DBB2D9063AD49B0634D5B023BEF11F0F02
:10AA800093703FD8226904EB0E0312791A760EF107
:10AA9000010E5FFA8EFE16B1236980229A7084F847
:10AAA00039E0774684E781F80280236980229A7032
:10AAB000774684F839E07BE704EB0E0291F80480D6
:10AAC00082F818800EF1010E5FFA8EFEB9E781F868
:10AAD00002C021690846B0E7A82191702069BE46EE
:10AAE0000279B0E7774663E78170DEE71021A023A3
:10AAF000D170013BFDD12269937803F0F7037746CB
:10AB0000937055E723691B79C5E700BF009FFF1FBE
:10AB10000148FFF71FBD00BF6890FF1F0148FFF706
:10AB200019BD00BFD490FF1F704700BF38B5144C4B
:10AB3000037801225B000546204684F83B3084F808
:10AB40005E2084F85D20FFF78BFC20460021FFF794
:10AB500047FE0B4C2978012320461A46FFF7CAFE10
:10AB60000128F6D194F8383094F839209A4205D962
:10AB7000E218013384F83830107E38BDFF2038BD2C
:10AB80006890FF1F38B51B4C037801225B00054617
:10AB9000204684F83B3084F85E2084F85D20FFF77F
:10ABA0005FFC20460021FFF71BFE124C297820464F
:10ABB00001230222FFF79EFE0228F6D194F83820E6
:10ABC00094F839108A420FD2531CDBB2A018994274
:10ABD00084F83830007E0AD9234402321B7E84F880
:10ABE000382040EA032038BD4FF6FF7038BD40F4EE
:10ABF0007F4038BD6890FF1F0C2901D900207047A5
:10AC00000231490001F0FE01FFF7BCBF70B50C4CEA
:10AC10000378164601255B00204684F83B3084F813
:10AC20005E5084F85D50FFF71BFC31462046FFF76D
:10AC300017FC29462046BDE87040FFF7D1BD00BF94
:10AC40006890FF1FF8B505460F4616464124214679
:10AC50003A462846FFF7DAFF611C0234C9B2324691
:10AC60002846E4B2FFF7D2FF592CF0D1F8BD00BF5F
:10AC700038B504460D463548FFF706FC63228021AF
:10AC800020462570FFF7C2FF012002F0C9FC2046D4
:10AC900000225E21FFF7BAFF20465D21FFF746FF45
:10ACA000242801D0002038BD204606220C21FFF7C1
:10ACB000C9FF204601222B21FFF7A8FF20460122D1
:10ACC0002C21FFF7A3FF20460E222D21FFF79EFF28
:10ACD000204600222E21FFF799FF204601222F2136
:10ACE000FFF794FF204605223021FFF78FFF204613
:10ACF00001223121FFF78AFF204600223221FFF78F
:10AD000085FF204600223321FFF780FF20460022E6
:10AD10003421FFF77BFF204600223521FFF776FF25
:10AD2000204600225B21FFF771FF204610225C21A4
:10AD3000FFF76CFF204620225D21FFF767FF2046CA
:10AD40008F225E21FFF762FF012038BD6890FF1F50
:10AD500010B4047F4160022CC26002D010BC01F02C
:10AD6000D7BB836810BC184790E80C00F0B41C688F
:10AD700059682568164F174E29432160164D17490B
:10AD80001760D66015611160417A154A5C180A3166
:10AD900094F8244053F8215002EBC40149680D6037
:10ADA000017A5C1803EB8101247ECD6902EBC401BA
:10ADB00049680D60817A581803EB810390F83000E0
:10ADC000596B02EBC002F0BC53681960704700BFBA
:10ADD00001401F00011000380110007800001F80A2
:10ADE0004C3D0100704700BFF0B50C1EBDF814606B
:10ADF00034DBB0F906701919B942C4BF3B1B1BB252
:10AE0000002BA6461CDD002A1146B8BFD11D02F05A
:10AE10000705CC10826A012007FB04E1A840012E3F
:10AE20000A44C0B21ED00CD3022E09D1013B12FA43
:10AE300083F3013A12F8011F41409A421170F9D18F
:10AE4000F0BDC043013B12FA83F3C0B2013A12F8DD
:10AE5000011F014093421170F9D1F0BD23441BB290
:10AE60000024C6E7013B12FA83F3013A12F8011FEE
:10AE700001439A421170F9D1F0BD00BFF8B50D1E23
:10AE80000EDB14461F46064601F03AFBA84207DDDA
:10AE9000002C05DB304601F037FBA04201DCF8BD99
:10AEA000F8BD304601F02AFB022853D003284BD0CE
:10AEB000012806D16540F3886C406540013B5D1B6D
:10AEC0002DB2012F03D02AD3022F14D0F8BD002CAD
:10AED0002246B6F90630B06AB8BFE21D42F3CF028F
:10AEE00002FB035504F00704435D012101FA04F459
:10AEF0001C434455F8BD002C2246B6F90630B06A12
:10AF0000B8BFE21D42F3CF0202FB035504F0070471
:10AF1000435D012101FA04F45C404455F8BD002C66
:10AF20002246B6F90630B06AB8BFE21D42F3CF023E
:10AF300002FB035504F00704435D012101FA04F408
:10AF400023EA04044455F8BD3389013B591B2546C7
:10AF50000CB2B6E7F18832890139013A4D1B141B56
:10AF60002DB224B2ADE700BF2DE9F041079E9DF957
:10AF70001880089D04461F4600F0C0FF0D4B0E4888
:10AF80000E4984F83380FF22002F08BF1F4684F843
:10AF90002F20002384F8302084F8312084F83220D8
:10AFA0002060A665E565676261652362A36220464D
:10AFB000BDE8F0816890FF1FA43201000110013844
:10AFC00010B50446806A034B236008B105F078FB96
:10AFD000204610BDA4320100F8B5436ADBB190F8F9
:10AFE0002C200125AA4083F83B2083F85E5083F88B
:10AFF0005D500446406A03680E461B68002198476E
:10B00000606A036831461B6898472946606ABDE854
:10B01000F840FFF7E5BBC26BC56C1368046A23EA0E
:10B02000050313604CB122684FF00043D3625163B3
:10B03000D36A002BFCDA936BF8BD836B466B082553
:10B04000802410E03768426C3A4332601F68826C9B
:10B050003A431A601A68876C013D22EA07024FEAF8
:10B0600054041A6007D02142ECD13268476C22EABE
:10B0700007023260EAE7F8BD70B50446406A0D4643
:10B0800000282BD0A16DFFF749FA002D20460CBFF8
:10B09000A621A721FFF7A0FF606A20B1E16DBDE8FE
:10B0A0007040FFF73BBA216C226D0868236A0243A7
:10B0B0000A6093B1DA7A82B1D00703D5224A99693E
:10B0C0001160DA7A910703D5204AD9691160DA7ADA
:10B0D000520702D51E4A1B6A136070BD236A002BFB
:10B0E0002BD0D97A626DE1B172B6D97ACE0706D586
:10B0F0001848D9680668314099610160D97A880793
:10B1000006D51548196906683140D9610160D97AB8
:10B110004E0705D51148596906683140196201602A
:10B1200062B61B68D968914207D00D4818600D4976
:10B13000DA6042F0804018611960226C216D13685A
:10B1400023EA01031360A0E700E100E004E100E06E
:10B1500008E100E080E100E084E100E088E100E057
:10B1600001403F0000003F80436A2DE9F041054661
:10B170000E469046002B3ED090F82C100124A140A2
:10B1800083F83B1083F85E4083F85D40406A0368B3
:10B1900000211B6808F1FF379847FFB2B8F1000F94
:10B1A00023D03744A046013E686A16F8011F0368A1
:10B1B0001B6898470134B742E4B216D0202CF3D173
:10B1C0000121686AFFF70CFB95F82C206B6A52008E
:10B1D00083F83B2083F85E8083F85D80686A0368AB
:10B1E00000211B6898470124DEE7686A0121BDE859
:10B1F000F041FFF7F5BAC26BC16C136823EA010393
:10B2000006EB080413604FF00048A6420ED02B6AEC
:10B2100016F801EB63B11A68C2F82C80C2F834E06A
:10B22000D36A002BFCDAA642936BF0D1BDE8F08123
:10B23000AB6BD5F834C008208021DCF800206F6C9F
:10B240001EEA010F14BF3A43BA43CCF800201A6833
:10B25000AF6C3A431A601A68AF6C013822EA0702F1
:10B260004FEA51011A60E8D1CFE700BF70B504463C
:10B27000406A0D46002828D0A16DFFF74FF92046FF
:10B280002946FFF7A9FE606A20B1E16DBDE8704074
:10B29000FFF744B9216C226D0868236A02430A60F3
:10B2A00093B1DA7A82B1D00703D5234A9969116044
:10B2B000DA7A910703D5214AD9691160DA7A5207FF
:10B2C00002D51F4A1B6A136070BD236A002B2BD066
:10B2D000D97A626DE1B172B6D97ACE0706D519482E
:10B2E000D9680668314099610160D97A880706D526
:10B2F0001548196906683140D9610160D97A4E074D
:10B3000005D512485969066831401962016062B674
:10B310001B68D968914207D00D4818600D49DA6062
:10B3200042F0804018611960226C216D136823EA95
:10B3300001031360A3E700BF00E100E004E100E0C7
:10B3400008E100E080E100E084E100E088E100E065
:10B3500001403F0000003F802DE9F041044686B0E7
:10B36000806A9DF830801E460F461546B4F90830B5
:10B37000002800F04281DA1D48BF03F10E02B4F943
:10B380000630D21003FB02F2002105F0BDFCB4F937
:10B390000820202A00F39280B4F90610A34B012064
:10B3A000203A733902EBD27201EBD1714FF0200ECB
:10B3B000029073208DE8014042F34F0241F34F01A8
:10B3C000204600F051FE606A84F82D70002800F0DD
:10B3D0004D81002D40F08A80B4F90830202B14BF35
:10B3E0003D253C2584F82C50B8F1000F40F08580B5
:10B3F00006B394F93300002818DBC0B2012102F033
:10B40000E7F8012194F8330002F0CEF8012002F0B1
:10B4100007F9002194F8330002F0C6F80A2002F080
:10B42000FFF8012194F8330002F0BEF8606A0028AA
:10B4300000F08280A16DFFF771F804227C4920465C
:10B44000FFF792FE217A0139C9B22046FFF7C4FD09
:10B45000784904222046FFF787FE94F92D30012B0E
:10B4600014BF142110212046FFF7B6FD04227249B3
:10B470002046FFF779FEB4F90630802B00F0928069
:10B48000602B00F0A680D9212046FFF7A5FD94F996
:10B490002D30012B14BFF12122212046FFF79CFD06
:10B4A000204606226549FFF75FFE606A50B3E16DF2
:10B4B000FFF734F8012006B0BDE8F081B4F90610BA
:10B4C0005F4B0120403A52394FF0400E029002EBA0
:10B4D000D272522001EBD1718DE8014042F34F024C
:10B4E00041F34F01204600F0BFFD6CE76DB284F8D8
:10B4F0002C50B8F1000F3FF47BAFFEF7C5FF002ED4
:10B5000094D076E7216C226D0868236A02430A60B2
:10B5100073B1DA7A62B1D00703D54A4A99691160EA
:10B52000DA7A91077CD4520702D5474A1B6A136026
:10B53000012006B0BDE8F081236A002B2BD0D97A18
:10B54000626DE1B172B6D97ACF0706D53F48D968A6
:10B550000568294099610160D97A8E0706D53C4873
:10B56000196905682940D9610160D97A4D0705D567
:10B5700038485969056829401962016062B61B683C
:10B58000D968914207D0344818603449DA6042F0F3
:10B59000804018611960226C216D136823EA010351
:10B5A00013604AE7B4F90830202B00F08680402B66
:10B5B0007FF469AF2A4920460322FFF7D5FD94F9AD
:10B5C0002D30012B14BFCF219F212046FFF704FD12
:10B5D00059E7B4F90830102B7FF455AF21492046C4
:10B5E0000322FFF7C1FD94F92D30012B14BFAF21C9
:10B5F00010212046FFF7F0FC45E7DA1D48BF03F1B4
:10B600000E02B4F90630D21003FB02F21046059286
:10B6100005F04EF8A06200283FF44DAF059AB3E65E
:10B62000114AD9691160DA7A7DE700BFFC32010066
:10B63000DC340100E0340100E4340100E8340100AE
:10B64000F034010000E100E008E100E080E100E00A
:10B6500084E100E088E100E001403F0000003F801D
:10B66000F8320100B037010004E100E0012194F854
:10B670003100244F01F0ACFF94F83200012101F0B9
:10B68000A7FF94F9312094F9323057F83220E26361
:10B6900057F83330206A23640125E56425651A686C
:10B6A0002A431A6078B1B8F1000F3FF428AFFFF7D2
:10B6B0005BFB002E3FF4BAAE9BE604221249204603
:10B6C000FFF752FDDFE6294694F82F0001F080FFD6
:10B6D000294694F8300001F07BFF94F92F2094F96B
:10B6E000303057F83220626357F833306564A56410
:10B6F0001A68A36322F001021A60002E3FF496AE8E
:10B7000077E600BF4C3D0100F4320100B0F908209B
:10B71000D31D48BF02F10E03B0F90620806ADB108A
:10B7200002FB03F2002105F0EFBA00BFF0B50029DB
:10B73000BDF814502EDBB0F90660B1422ADA002AB7
:10B7400059DBB0F9087014461C44BC42C4BFBB1A94
:10B750001BB2002B1EDDD2B2D408D0F828E016FBB5
:10B76000041112F00702DBB20EEB010421D0C2F18A
:10B770000807FAB2374F9342BF5C0CD2C3EB020CFE
:10B78000FF2646FA0CF6012D07EA06073FD005D33F
:10B79000022D36D0F0BD012D39D030D21EF8016017
:10B7A00026EA07070EF801709342F3D3B0F90610AA
:10B7B0000C449A1AD2B2072A10D9022D36D0002D85
:10B7C00014BFFF26002613462670083BB0F906106A
:10B7D000DBB2072B0C44F7D802F00702002AD9D0BD
:10B7E0001D4B012D9B5C1DD017D3022DD2D1227889
:10B7F00053402370F0BD13441BB20022A1E7022D79
:10B8000025D11EF8016077400EF80170CCE71EF8D4
:10B81000016037430EF80170C6E7227822EA03037D
:10B820002370F0BD227813432370F0BD11462378B6
:10B83000DB4323700839B0F90630C9B207291C442C
:10B84000F5D812F00702A5D0034B9B5CCFE7344438
:10B85000AFE700BF943201008432010070B4C47DB0
:10B86000BDF80C50022C18D0032C1FD0012C0BD08B
:10B87000002A03DBB0F90840944201DC70BC704739
:10B88000039570BCFFF7B0BAC4880395013CA41AB5
:10B890000A4621B270BCFFF749BF0689C488013E41
:10B8A000641AB21AE41A12B221B2E1E704890395CC
:10B8B000E41A641A114622B270BCFFF737BF00BF0A
:10B8C00070B4C57DBDF80C60022D1AD0032D12D0C6
:10B8D000012D03D0039670BCFFF728BFC488E41A7B
:10B8E000A41A0A4621B2002A03DBB0F908409442A8
:10B8F00013DC70BC70470489013C641A114622B203
:10B90000F1E7C48805890396013CAD1AED1A621A65
:10B9100011B22AB270BCFFF709BF039670BCFFF7E3
:10B9200063BA00BF2DE9F8430446406A002863D09B
:10B93000A16DFEF7F3FD052274492046FFF714FCC4
:10B94000A1790139C9B22046FFF746FBB4F90820B6
:10B95000E588A66AD31D48BF02F10E03DB10626AB8
:10B9600015FB03F51FFA85F8002A7BD094F82C30DC
:10B970000125AB4082F83B3082F85E5082F85D5082
:10B98000606A036840211B6808F1FF379847BFB21F
:10B99000B8F1000F23D03744A846013E606A16F87C
:10B9A000011F03681B6898470135B742EDB216D0F6
:10B9B000202DF3D10121606AFEF712FF94F82C20AC
:10B9C000636A520083F83B2083F85E8083F85D80D1
:10B9D000606A036840211B6898470125DEE7012162
:10B9E000606AFEF7FDFE606A002800F08D80E16D60
:10B9F000BDE8F843FEF792BD236A002B2BD0D97A1D
:10BA0000626DE1B172B6D97ACE0706D54048D968E1
:10BA10000568294099610160D97A8D0706D53D48AE
:10BA2000196905682940D9610160D97A480705D5A7
:10BA300039485969056829401962016062B61B6876
:10BA4000D968914207D0354818603549DA6042F02C
:10BA5000804018611960226C216D136823EA01038C
:10BA6000136068E7E26BE36C1168276A0B4306EB2F
:10BA7000080913604FF0004E4E450DD016F801CB6B
:10BA80002FB33A68C2F82CE0C2F834C0D36A002B56
:10BA9000FCDA4E45936BF1D1226C236D11680B4398
:10BAA000136097B1FB7A83B1D90703D51D4BBA69EF
:10BAB0001A60FB7A9A0703D51B4BFA691A60FB7A66
:10BAC0005B0702D5194B3A6A1A60BDE8F883A36B8D
:10BAD000D4F8348008208021D8F80020656C1CEA56
:10BAE000010F14BF2A43AA43C8F800201A68A56CA6
:10BAF0002A431A601A68A56C013822EA05024FEA47
:10BB000051011A60E8D1B7E7276AC5E78C32010016
:10BB100080E100E084E100E088E100E001403F00D6
:10BB200000003F8000E100E004E100E008E100E007
:10BB30002DE9F04F85B09946BDF93870BDF83CA0AD
:10BB4000BB1AC1EB090B002BB8BF5B42BBF1000F66
:10BB5000B8BFCBF1000B5B450D46164600938046FF
:10BB600048DC4D453A4633464CDC194613460A46F6
:10BB7000C5EB09019B1A89B2002B0CB2B8BF5B421E
:10BB800004EBD474BE42ACBF4FF0FF3201224D45EE
:10BB9000039102924FEA640429DC9BB201930DE009
:10BBA000D8F80070BF69B847019BE41AA3B21CB271
:10BBB0000135002C2DB211DBA94518DB009B5B453C
:10BBC0002A46534631464046EADCD8F80020534620
:10BBD0009769294632464046B847E5E7029A164437
:10BBE000039AA94502EB030436B224B2E6DA05B0A3
:10BBF000BDE8F08F4A462B46B94635464D451746B7
:10BC00001E46B2DD304629463E464D460746894629
:10BC1000AEE700BF10B404682469A44610BC6047B6
:10BC200030B40468BDF808500295A46BA44630BC3B
:10BC3000604700BF30B40468BDF808500295E46B5B
:10BC4000A44630BC604700BF70B40468BDF90C6006
:10BC5000BDF8105003960495246CA44670BC604750
:10BC6000704700BF10B582B0B0F90C200191016897
:10BC7000009200220C6CB0F90A301146A04702B0C5
:10BC800010BD00BF704700BF01F003010129C1755D
:10BC900006D0032904D0C28803894281838170477A
:10BCA0000289C38842818381704700BF2DE9F0413A
:10BCB0000568134E6F6986B0B7420446BDF8308000
:10BCC00010D1013B13441BB20093CDF804800B4606
:10BCD000AD6A2046A8472368DB6AB3420AD106B0A2
:10BCE000BDE8F081059304920391B84703A9256844
:10BCF0000EC9E6E7204606B0BDE8F041184700BF90
:10BD000061BC00002DE9F0410568124E6F6986B0F4
:10BD1000B7420446BDF830800FD1013BCDF8048016
:10BD20000B4400921BB2AD6A2046A8472368DB6A29
:10BD3000B3420AD106B0BDE8F081059304920391A5
:10BD4000B84703A925680EC9E7E7204606B0BDE855
:10BD5000F041184761BC00002DE9F04F0568DFF89D
:10BD600058B06F6985B05F450646BDF93890BDF89B
:10BD70003CA00C46904615D11F19BC420CDACDF8F8
:10BD800000A0214601342D6A4B464246304624B27B
:10BD9000A847BC423568F2DBEB6A5B4507D105B0CA
:10BDA000BDE8F08F0393B8473568039BE4E730465E
:10BDB00005B0BDE8F04F184761BC00002DE9F04325
:10BDC00087B099420546BDF93840BDF83C6025D0A2
:10BDD000A24212D00768DFF88080D7F81490C145DE
:10BDE00032D18DE850002846BC6AA0472B68DB6A38
:10BDF000434524D107B0BDE8F083994202DD0846EF
:10BE00001946034628680E96C46B01335B1A1BB2B1
:10BE10002846A44607B0BDE8F0436047A24202DDD1
:10BE2000134622461C4628680E96631C846B9B1A98
:10BE30001BB22846A44607B0BDE8F0436047284639
:10BE400007B0BDE8F0431847059304920391C84733
:10BE500003A92F680EC9C4E761BC00002DE9F04FAB
:10BE6000D0F800E0DFF89090DEF814B083B0CB4556
:10BE70000446BDF93080BDF834A00D4617461E4675
:10BE800031D1CDF800A0DEF824B0294633463A4639
:10BE90002046D8472368CDF800A008F1FF323A4485
:10BEA000D3F824B0294612B233462046D847236837
:10BEB000CDF800A02946D3F820B03A4643462046A4
:10BEC000D8472068CDF800A0711E29444346056A72
:10BED00009B23A462046A8472368DB6A4B4506D19B
:10BEE00003B0BDE8F08FD847D4F800E0C9E720469A
:10BEF00003B0BDE8F04F184761BC0000F0B4002467
:10BF000001264FF6FF75094F07600471C475C4819F
:10BF100004824476C4618675067685824582C18036
:10BF2000028141818281F0BC704700BFBC370100B3
:10BF30002DE9F04F85B00668BDF84450BDF9388052
:10BF4000CDF8008004460195D6F848B00392BDF9BB
:10BF50003C60BDF9407089469A46D84723680195F0
:10BF6000009742465146D3F8488020463346C047A2
:10BF70002068039B0E930F95856C4B463A463146DD
:10BF80002046AC4605B0BDE8F04F60472DE9F04FC4
:10BF900087B01746BDF9404000912546E91D05933D
:10BFA00044BF2B4603F10E010268BDF84860536997
:10BFB0000294C91003912B49BDF9444001968B426C
:10BFC000824645D1002C3CDD029B3C445E1EB6B24D
:10BFD0004FF0000923B2049301364D46029B002B1B
:10BFE00028DD059B002403EB090806E0EDB22B06D3
:10BFF00004F1010411D4A6421CD0A1B211F0070F24
:10C0000023B24FEA4505F1D1002BB8BF0733DB104F
:10C01000013418F803502B06EDD5009BD2F818B068
:10C0200019443A4609B2019B5046D847A642DAF86D
:10C030000020E2D1039B01379944049B3FB2BB42ED
:10C04000CCD1D36A074A934206D107B0BDE8F08F3E
:10C050009847DAF80020B5E7504607B0BDE8F04F42
:10C06000184700BF61BC000070B4BDF90C60BDF999
:10C070001050BDF8144003960495059470BCFFF76A
:10C0800085BF00BF2DE9F04F93B090460591C1697F
:10C090001090BDF870000790BDF874909DF878A0DE
:10C0A0000493002900F0CD800A7A0AC989460499D0
:10C0B0008A1AD2B203EBC203BAF1010FDA780B92FB
:10C0C00093F905201E8893F802B00F9293F9064069
:10C0D00079D913B2099323B20C93109B1A68A94B18
:10C0E0001193194653698B4240F0A6800B9B002B9D
:10C0F00055D01FFA88F300210D93C8462344DDF87C
:10C10000409006910E930F460C46BBF1000F3FD0B6
:10C11000BDF818100C9B03971FFA8AF0CB1813FB7D
:10C1200000F304900E9801440D98034409B21BB229
:10C130000A910893002505E00135EBB264009B45A8
:10C14000E4B222D9039B2B44590703D1731C18F87E
:10C1500006409EB22306EFD5099BBDF81000E918F2
:10C1600011FB00F10598BAF1010F0FFA8AF30144AF
:10C170001CD0079801900093D26909B2174648462F
:10C18000089AB847D9F80020D6E7039F5F44FFB26A
:10C19000069B0B9901330693DBB29942B5D8D36A5B
:10C1A000119A934243D113B0BDE8F08F0F9B191839
:10C1B00093690A9A29441F4609B2079B4846B84723
:10C1C000D9F80020B8E700230C93099385E70A9A71
:10C1D0000D9B0132013B52B213F0FF030A920D9303
:10C1E0006FD1DDF81890079BDDF83C80DDF820A0CA
:10C1F0004B4517D0BAF1010F00F0C8800B9A109D83
:10C20000CDF804900BEB8B014FEACB030A4400936B
:10C210001146DEF81C405346424609B22846A04764
:10C22000D5F800E0DEF82C30119A9342BBD010987C
:10C2300013B0BDE8F04F1847109D284698472A686C
:10C2400054E7109A0598B2F90A308342ABDDB2F98F
:10C250000C304345A7DD062313FB0A03002BA2DDA8
:10C2600008EBCA03002B9EDD537E2BB9049BAF2B3A
:10C2700002D90133DBB20493109BD3F800E0414BA9
:10C2800011931A46DEF81430934240F08E801FFA64
:10C2900088F30E9308339BB2BDF814200593052351
:10C2A0000D9300230A93CDF83C800FFA8AF3DDF852
:10C2B0004080CDF818900B921FFA8AFBCDF820A091
:10C2C00099460A9ABDF810000B9C0E9D052319464D
:10C2D00011FB00232C481146C75C039702FB0B425D
:10C2E00014FA81F312B21BB209920C932C462E461B
:10C2F0001CE0089B0999012B2AB24B4640462DD0E1
:10C30000079F0197CDF80090DEF81CA0D047D8F821
:10C3100000E0039B5B0801340393059BA4B25D44DA
:10C320005E44A342ADB2B6B23FF451AF039BD8070F
:10C33000DFD4079B069A9342EBD0089B012B16D0C3
:10C34000069B0193CDF80090DEF81CA009994B469E
:10C3500032B24046D047D8F800E0DAE7DEF818A05D
:10C36000079B0C9922B2D047D8F800E0D1E7DEF85D
:10C3700018A00C991346404622B2D047D8F800E0E6
:10C38000C7E700BF61BC00000C3801000B99109D8D
:10C39000CDF800900531DEF8204009B2424608236E
:10C3A0002846A047D5F800E03CE7109C2046984777
:10C3B000D4F800E06BE700BFF0B5C36985B0044670
:10C3C0002BB30A2968D00D294AD01A7A914247D353
:10C3D000587A884244D35D688A1A05EBC205AA7868
:10C3E000002A50D0E87800284DD0207E00283AD08E
:10C3F00095F905E0B4F90E00A67DB4F90A7072440F
:10C4000006FB0202BA4262DCB4F9102030E00A29CD
:10C4100056D00D2924D0027E002A4BD0B0F90E0050
:10C42000A57DB4F90A60062212FB0502B2423EDD88
:10C43000228AE38102EBC50212B218462282A78A41
:10C44000668A02950B468DE8C00001462046FFF73C
:10C4500019FEA37DE28903EB430302EB4303E3816F
:10C46000012005B0F0BDA67DB4F90E00B4F910208E
:10C47000B4F814E0678A02960B468DE880400146C6
:10C480002046FFF7FFFD2979E389A27D012001FB0A
:10C490000233E38105B0F0BD0022C2819A7A817D2A
:10C4A000038A01FB02330382012005B0F0BDB4F919
:10C4B0001020C4E7857DB4F91020B0F90E00BEE766
:10C4C000028A817DC38102EBC1030382C8E7002099
:10C4D000E0819B7A228A03FB062212B22282C7E7FE
:10C4E000C1810282704700BF002908BF0121817508
:10C4F000704700BF81824182704700BFC07D704796
:10C50000B0F90A00704700BFB0F90C00704700BFD7
:10C5100010B4EFF3108272B6437F33B9017F012963
:10C5200007D003290FD00123437702B962B610BCAC
:10C530007047124C2168A1B1114943610B688361B6
:10C5400008605861EFE70F4C216881B10E494361E3
:10C550000B688361086058610C4B4FF08051196083
:10C56000E1E7074B4161816120601860DBE7064B22
:10C570004161816120601860EEE700BFEC9EFF1F03
:10C58000E89EFF1FDC9EFF1FE09EFF1F04ED00E002
:10C5900070B5EFF3108272B60C4C206880B10C4E6F
:10C5A00000254369236073B19D6102B962B6457786
:10C5B00083689847EFF3108272B620680028F0D1A4
:10C5C00002B962B670BD3360EFE700BFDC9EFF1FAB
:10C5D000E09EFF1FFFF7DCBF184A30B41468002C40
:10C5E00027D0036821688B420ED2CB1A00218460C9
:10C5F000C1602360E06010600223037530BC7047A7
:10C6000011688B42144608D3A2685B1A0360002AA3
:10C61000F6D18260C460A060EEE7D268C260846038
:10C62000E060C568CB1A0222A8602360027530BCA6
:10C6300070478460C4601060DEE700BFE49EFF1FA7
:10C64000F8B5224E34682CB32368002B3AD1204F22
:10C650001D4604E03468ECB12368002B32D1A36896
:10C6600003B1DD6020693360036825751B68BB4238
:10C6700021D1037F4560022BC46020D0FFF748FF23
:10C680006368002BE6D023602046FFF7A5FF3468DF
:10C69000002CE1D1EFF3108372B60E4A002110682E
:10C6A000116003B962B628B18468FFF795FF204690
:10C6B0000028F9D1F8BD224600219847E0E78368B9
:10C6C0009847DDE7013B2360E4E700BFE49EFF1FDE
:10C6D00051AD0000F49EFF1F024A1368013313603E
:10C6E000FFF7AEBF009FFF1F704700BF0368F0B4A5
:10C6F000FBB1002501249D60DC601B4C1A601C44CA
:10C70000241104F144056A11032692009E60174F1C
:10C710000679174B47F8241002F1604202F5614296
:10C7200005F01F05012000FA05F5E6541560F0BC80
:10C730007047104C236843F40003236000BF0E4B86
:10C740000E4DA4F58734A4F59E7401261E60234681
:10C7500004609C68002CD0D01033AB420360F8D149
:10C76000002303601846E2E7008FFCBF4091FF1FE3
:10C7700044E400E03C80044000700340407103400A
:10C780000168A9B10B4BF0B40B441B110A4E0B4FBF
:10C790000B4D46F8237003F1440202F01F040123FD
:10C7A0005211A340002445F822308C600460F0BC94
:10C7B000704700BF008FFCBF4091FF1FE9C600001B
:10C7C00080E100E0024A034B012111601B68184719
:10C7D0000C7103404091FF1F024A034B012111607D
:10C7E0005B6818471C7103404091FF1F024A034BCE
:10C7F000012111609B6818472C7103404091FF1F75
:10C80000024A034B01211160DB6818473C71034069
:10C810004091FF1FF8B50E4671B17AB10746144634
:10C8200000253B6816F8011B1B6838469847013CF9
:10C830000544F6D12846F8BD0846F8BD1046F8BDB7
:10C8400000B5064A036812885B6883B001A9ADF899
:10C8500004200222984703B05DF804FB0C3D010060
:10C86000F0B507468BB0002A33D0012A08BF0A2250
:10C8700051B3212400E0F4B2B1FBF2F502FB151133
:10C88000C8B2092900F1300198BFC8B20AA988BF0F
:10C890003730214488BFC0B201F8240C661E2946F7
:10C8A000002DE8D133B1013CE4B20AAB23442D2280
:10C8B00003F8242C3B6801AA11195B683846C4F1BF
:10C8C000220298470BB0F0BD30228DF8252021249C
:10C8D000E8E70368C9B21B6898470BB0F0BD00BF1A
:10C8E0000029BABF49422D2300230A22FFF7B8BF0F
:10C8F000374A384913681B06FCD40B6813F08003D1
:10C90000F8D172B634490A78002A5FD0334A3448E5
:10C91000F0B4344C176806682568D4680C303E447F
:10C92000143200681268304F35442C4420440244CD
:10C93000C2F34E022D4E2E482E4D2F4C42F4004293
:10C940003A60376806682D682C4A24680C303E44EB
:10C95000006812682A4F35442C4420440244C2F334
:10C960004E02284E2848294D294C42F400423A6094
:10C97000376806682D68274A24680C303E440068F2
:10C980001268254F35442C4420440244C2F34E0221
:10C99000224E2348234D244C42F400423A6037682B
:10C9A00006682D68214A24680C303E4400681268ED
:10C9B00035442C4420440244C2F34E021C4842F445
:10C9C000004202600B7062B6F0BC704762B67047FE
:10C9D00024B0034024B00B40F99EFF1F38B0034041
:10C9E0003CB0034040B003402CB0034058B003407B
:10C9F0005CB0034060B0034064B003406CB00340DF
:10CA000030B0034038B00B403CB00B4040B00B405E
:10CA100044B00B404CB00B402CB00B4058B00B4016
:10CA20005CB00B4060B00B4064B00B406CB00B408E
:10CA300030B00B4030B42948294A2A4B2A4D602493
:10CA4000E121047011701B78284C082B30D00A2B80
:10CA50002748284937D00C2B0CBF35223D22122302
:10CA60002A60236002600B60234B24491B78244A10
:10CA7000BBB101230B601360224B23491B78234A6F
:10CA8000012B26D9042B0FD9082B1ED9102B94BFAC
:10CA9000862387230B6013601D4B01221A7030BC64
:10CAA00070470B601360E7E784230B601360F3E7C4
:10CAB00000F58E200F490830012213232A602360DD
:10CAC00002600B60D0E73922F7E785230B60136023
:10CAD000E2E780230B601360DEE700BF0040074001
:10CAE000014007405091FF1F08B003400CB00340C5
:10CAF00008B00B400CB00B40FC9EFF1F20B0034061
:10CB000020B00B405191FF1F24B0034024B00B40D4
:10CB1000F99EFF1F0C2830B417D91023984228BF64
:10CB200018461C46104A114D1178181A8C4228706C
:10CB300018D00F4913700B7823B10E490E4A002309
:10CB40000B60136030BCFFF775BF0A2802D90C23B5
:10CB50001C46E7E7082802D90A231C46E2E7082317
:10CB60001C46DFE730BC70475091FF1FF89EFF1F47
:10CB7000F99EFF1F24B0034024B00B4028282FD873
:10CB8000334B2DE9F0411E5CFF2E2BD0314B1B782F
:10CB9000002B2AD132062CD472B62F4D2F4C2F46A3
:10CBA000012326602B7062B672B623681B060CD474
:10CBB0003B781BB9F4E72B78002BF1D062B602F07A
:10CBC0009BF972B623681806F5D5254B1B68002221
:10CBD0002A7062B6234A107843FA00F0BDE8F0816B
:10CBE000002070470020BDE8F081FFF781FE32068B
:10CBF000D2D572B61C4DDFF87C801C4C06F0400785
:10CC0000FFB206F03F06D8F80030DFB123F0100382
:10CC1000C8F8003001232660134A2B7062B672B642
:10CC2000236819060CD413781BB9ECE72B78002B7A
:10CC3000E9D062B602F060F972B623681B06F5D53A
:10CC40000B4BC3E743F01003C8F80030E2E700BF26
:10CC5000103D0100F99EFF1FFB9EFF1F00B0034027
:10CC600010B00340F89EFF1FFA9EFF1F00B00B405C
:10CC700010B00B400CB00B400A4A0B49136843F448
:10CC8000805313600B7843B9084BC0221A70084BCD
:10CC900080F30C0000B218807047044B80221A7099
:10CCA000F5E700BF2C800440FC9EFF1F21C00C4014
:10CCB00000C00C40F0B51B4B1B4E596818689A68B1
:10CCC000DB6885B06C460FC4337899071DD5174AC9
:10CCD000174C1378174913F0700318BF1370164AD6
:10CCE000164B8027177000263320032226706D46CE
:10CCF00008701A7072B6043C45F001052046A8473A
:10CD000062B6237813F0700309D10D4B064901E098
:10CD1000013B02D00A78D207FAD505B0F0BD2370E6
:10CD200005B0F0BD3C3D01000100024000000240A2
:10CD3000040002400B000240070002400A000240CB
:10CD4000410D0300B0F5006F0AD210B5094B1B78F6
:10CD5000DB07044606D504F1A0500078C0B210BD30
:10CD600000207047FFF7A6FF04F1A0500078C0B282
:10CD700010BD00BF01000240B0F5006F17D238B5FA
:10CD80000F4B1B78DA070D46044611D504F1A0506D
:10CD90000378AB420AD00B4A137813F0700318BF24
:10CDA0001370074A05701378DB07FCD538BD704750
:10CDB000FFF780FF04F1A0500378AB42EBD1F5E719
:10CDC000010002400000024008B5F4F75BFEF5F7F1
:10CDD00045FA02F091F8FAE7844641EA000313F0BD
:10CDE00003036DD1403A41D351F8043B40F8043B72
:10CDF00051F8043B40F8043B51F8043B40F8043B35
:10CE000051F8043B40F8043B51F8043B40F8043B24
:10CE100051F8043B40F8043B51F8043B40F8043B14
:10CE200051F8043B40F8043B51F8043B40F8043B04
:10CE300051F8043B40F8043B51F8043B40F8043BF4
:10CE400051F8043B40F8043B51F8043B40F8043BE4
:10CE500051F8043B40F8043B51F8043B40F8043BD4
:10CE600051F8043B40F8043B403ABDD2303211D374
:10CE700051F8043B40F8043B51F8043B40F8043BB4
:10CE800051F8043B40F8043B51F8043B40F8043BA4
:10CE9000103AEDD20C3205D351F8043B40F8043B74
:10CEA000043AF9D2043208D0D2071CBF11F8013B72
:10CEB00000F8013B01D30B8803806046704700BF38
:10CEC000082A13D38B078DD010F003038AD0C3F147
:10CED0000403D21ADB071CBF11F8013B00F8013B29
:10CEE00080D331F8023B20F8023B7BE7043AD9D3E8
:10CEF000013A11F8013B00F8013BF9D20B780370BD
:10CF00004B7843708B7883706046704708B5104C3F
:10CF100008E0236859050DD423681A050FD4236847
:10CF2000DB0411D423685803F3D500F08DFE236889
:10CF30005905F1D502F044F823681A05EFD502F03F
:10CF4000D5F82368DB04EDD500F0F0FCEAE700BF7C
:10CF50003480044008B5FFF7D9FF00BF014B102211
:10CF60001A80704700200540704700BF094908B586
:10CF70000B6830B16A461844A2F58052904202D242
:10CF80000860184608BD03F065FB0C2303604FF0F2
:10CF9000FF3008BD5491FF1FFEE700BFEFF3138081
:10CFA00070B9EFF310836BB9EFF305825AB94FF400
:10CFB0008070EFF311832BB1984228BF1846704759
:10CFC0004FF0FF3070470F2A01D81846F1E7014BA8
:10CFD000D05CEEE7F0E300E0F0B44D1E2E460024F6
:10CFE00000E00134B0FBF2F302FB1300092800F16A
:10CFF00030078ABF3730F8B2C0B206F8010F1846C2
:10D00000002BEED10A1953704CB1107815F8016F4E
:10D0100028700133E01A834202F80169F5DB084603
:10D02000F0BC7047704700BF10B40F4B53F830206E
:10D0300092F880422CB1012369B182F8803010BC93
:10D04000704703EBC0035B681A6841B922F0020223
:10D050001A6010BC704782F8003110BC704742F073
:10D0600003021A6010BC70474C3D01001C4A02EBE1
:10D07000C00301295B6811D004291BD052F830008D
:10D08000002280F8802229B1022920D0032922D051
:10D090001A6070474FF480721A60704752F830007F
:10D0A0004FF4A27280F880121A601A6822F02002EF
:10D0B0001A60704752F830104FF4A272012081F8C4
:10D0C00080021A601A6842F020021A60704740F22B
:10D0D00003121A6070474FF481721A60704700BFE4
:10D0E0004C3D0100212848D8F8B5042A44D8DFE88F
:10D0F00002F0484B4E0345004FF410262B4B03EB38
:10D10000C0030D465C68216811F4E06148D0284BEB
:10D11000284A2949C3F89C2104F140422748C3F812
:10D12000A411A2F59221264FC3F8A0017C2925481D
:10D13000C3F8A871C3F8AC012CD9A2F594237C2BB9
:10D140002AD9A2F596237C2B28D9A2F598237C2BEB
:10D1500029D9A2F59A227C2A27D81B4872B62368BF
:10D1600023F4702343F08072C4F3840116432360D8
:10D1700040F82150266062B6F8BD70474FF4302663
:10D18000BCE74FF40026B9E74FF44026B6E74FF46A
:10D190002026B3E70D48E1E70D48DFE70D48DDE75E
:10D1A000FFF764FFB3E70C48D8E7F8BD4C3D01003A
:10D1B0000082FF1FF188FF1F9988FF1FC588FF1F8E
:10D1C0006D88FF1F4188FF1F3092FF1F5891FF1F7E
:10D1D0009091FF1FE091FF1F1092FF1F1A4B03EB6E
:10D1E000C00010B4426802F14043A3F592217C29AB
:10D1F00023D9A3F594217C290DD9A3F596217C2967
:10D200001FD9A3F598217C2919D9A3F59A237C2B42
:10D2100011D80E4C00E00E4C72B613680D4823F086
:10D220008773C2F3840123F4803343F08073136067
:10D2300044F8210062B610BC7047074CECE7074C7D
:10D24000EAE7074CE8E700BF4C3D01003092FF1FC2
:10D250009091FF1F25D000005891FF1F1092FF1FD3
:10D26000E091FF1F30B4054B054D064C0022102104
:10D270001A602A602060196030BC704714D00340E7
:10D2800004D0034000D00340282838B52ED0002910
:10D2900004464FDD5F4B1B78012505FA03F28A42F5
:10D2A00002D8212837D938BD0338C2B2012A3AD969
:10D2B000202C4AD0192C48D0574A126802FB011280
:10D2C00022FA03F31D2800F29B80DFE800F0928B26
:10D2D000847D9999766F999999999999999999686D
:10D2E000615A53994C99999999999945494B1B7849
:10D2F0000B2B08D90C2B1CBF0C3B19410846BDE871
:10D300003840FFF7B9BCC3F10C0399400846BDE8AB
:10D310003840FFF7B1BC2946FFF786FE2946BDE835
:10D320003840FFF7A3BE3D4A126802FB011222FA01
:10D3300003F3C7E72128B6D80021FFF775FE204682
:10D340000121BDE83840FFF791BE354A126802FB63
:10D35000011222FA03F3B5E73249334A0B604FF466
:10D360005173136038BD3149314A0B604FF451732A
:10D37000136038BD2F49304A0B6040F244431360BC
:10D3800038BD2E492E4A0B6040F24443136038BD2D
:10D390002C492D4A0B6040F24443136038BD2B49A1
:10D3A0002B4A0B6040F24443136038BD29492A4A96
:10D3B0000B6040F24443136038BD2849284A0B6093
:10D3C00040F24443136038BD2649274A0B6040F2BF
:10D3D0004443136038BD2549254A0B6040F244435D
:10D3E000136038BD2349244A0B604FF45173136016
:10D3F00038BD2249224A0B604FF45173136038BD87
:10D40000212C3FF650AF7F29D4BF002101212046B7
:10D4100093E700BF3892FF1F088003400890034045
:10D4200008800B4010800B4048A0044018800B403F
:10D430004CA004401880034008B004401080034012
:10D4400004B004404080034018C0044038800340CA
:10D4500014C004402880034010B0044020800340E2
:10D460000CB004403080034010C0044048800340AA
:10D470001CC00440189003403490044010900340B6
:10D480003090044038B1102828BF1020044AC3B29D
:10D49000107813707047024A012310781370704798
:10D4A0003892FF1F2DE9F8430E4680463249334D2E
:10D4B000304603F055F847F6122300281ABF1D46E0
:10D4C0004FF002094FF00109002425FA04F002F0A0
:10D4D00051FE4FF05E51074602F0A4FE0146304671
:10D4E00003F052F830B90134072CEED1E80902F00C
:10D4F00041FE07463146384602F048FF4FF07C5166
:10D5000002F086FD03F07AF84FF6FF729042A8F120
:10D51000030328BF1046012B29D9B8F1170F17D8DC
:10D52000174B23FA08F303F0010383F0010223B938
:10D53000B8F1190F0FD0BDE8F883124B124D134903
:10D540001A6044EAC9042A6008601C60BDE8F883D8
:10D55000B8F1200FECD10E4B0E4D0F49002244EADA
:10D56000C9041A602A6008601C60BDE8F8830B4B90
:10D570000B4D0C49F2E700BF001BB740006CDC020A
:10D580006006F000008003400480034008800340F0
:10D5900000800B4004800B4008800B40009003404B
:10D5A0000490034008900340212801D8FFF73CBDB8
:10D5B000704700BF212806D8044B53F8303093F849
:10D5C0000002C0B270470020704700BF4C3D010010
:10D5D000212801D8FFF74ABD704700BF72B60C4939
:10D5E0000C4B0D4A1B680868126862B6520102D5DE
:10D5F000322B88BF01300949C3F5BB334FF47A722F
:10D60000FF33A1FB031302FB00F000EB9310704704
:10D61000009FFF1F18E000E004ED00E0ABAAAAAAFB
:10D620002DE9F843054672B6204F214B214A1B686D
:10D630003C68126862B6520102D5322B88BF0134B1
:10D6400095B3C3F5BB331C4EDFF86490DFF86480FC
:10D65000FF334FF47A72A6FB031302FB04F404EBCE
:10D66000931472B6D9F800103A68D8F800E062B6A0
:10D67000C1F5BB33FF33A6FB03031EF0806FC4EB81
:10D6800093134FF47A7002D0322988BF013200FB25
:10D690000233B3F57A7F04D3013D05D004F57A74E3
:10D6A000DFE701F029FCDCE7BDE8F883009FFF1FFE
:10D6B00018E000E004ED00E0ABAAAAAAF8B52D4BF3
:10D6C0002D49DFF8D0E0DFF8D0C02C4E2C4D2D4C8A
:10D6D0002D4A2E4F4FF4000018604FF080701860F4
:10D6E0004FF0007018604FF0806018604FF00060DD
:10D6F00018600020086028234BF6FF71CCF800105A
:10D70000CEF80030336013602B6023603B60B3625F
:10D710009362092245F8242CC4F8D80F05F57F65DB
:10D72000C7F8D41F07F5FF2707F5FA67C6F8F83FD3
:10D730002B6006F5FF26C4F8D42F05F5FD2504F56A
:10D74000FF24386006F2F4761148316005F5FF6574
:10D7500004F5FD642B6023600260FFF76BF919206C
:10D76000FFF75EFF00F0B6FF40F21310BDE8F8408F
:10D77000FFF756BF08E100E0048003401480034037
:10D78000248003402C8003401C80034034800340ED
:10D7900000800B400C800340088003402DE9F84FC7
:10D7A000214B1B6807460BB101221A70DFF88890E5
:10D7B0001E4D99F80040DFF884801D4E0134272C5F
:10D7C0008ABF4FF0000A5FFA84FA5446AB462B78C2
:10D7D000A34216D1FFF7E2FB40281FDC33791B067A
:10D7E000F5D59BF800300133272B86BF0022134666
:10D7F000DAB218F80330DBB2F3712A702B78A34247
:10D80000E8D00C490A4BFFB208F804700120AC22A2
:10D81000087089F800A0DA70BDE8F88FFF28D6DD1F
:10D8200001F06AFBD3E700BF789FFF1F759FFF1FC2
:10D8300000C00640749FFF1F7C9FFF1F0C9FFF1FAF
:10D840001C4BDFF894C01A681B49F0B542F48052B3
:10D850001A4D1A60DFF884E0194F1A4E1A4C002353
:10D860008CF800304FF451722B701F2840F21335A2
:10D870008EF800303B70337025600A6012D819466C
:10D880000124124A124D11701248547000212C27A5
:10D89000402693724FF4003491701174D7702E703B
:10D8A0000460F0BDC0F34431C0F3471400F01F031F
:10D8B000E7E700BF348004400CC00440099FFF1F0D
:10D8C000759FFF1F749FFF1F08C0044000C00640E3
:10D8D00031E400E004E100E0089FFF1F7C9FFF1F90
:10D8E000034B1B68DB0401D5FFF758BF704700BF2F
:10D8F0003480044010B5044C237823B101F0FCFAC5
:10D900002378002BFAD110BD749FFF1F054A064BE8
:10D9100010781B78C0B2DBB2984238BF4030C01AD2
:10D92000704700BF089FFF1F099FFF1F30B42B4B9C
:10D930001A7994061FD52A48DA79037829490133E0
:10D940003F2B0978C8BF00238B42D2B203D0264CAC
:10D95000D9B2E2540170254A116861B1244A1278A3
:10D96000D2B2934236BFC2F140029B1A9B18272BBA
:10D97000C4BF01230B70194AD378DBB2180611D447
:10D980005A060DD5154B1B795B0609D5194B1A495B
:10D990001B6800220A7003B11A70104B2C22DA7037
:10D9A00030BC704711790906EAD5144910480C7843
:10D9B0000178C9B28C420DD04A1C272A84BF0021AD
:10D9C0000A460F4D054C98BFD1B2AA5CD2B2E271A3
:10D9D0000170D5E76C21D170D2E700BF00C00640CE
:10D9E000089FFF1F099FFF1F349FFF1F049FFF1FFA
:10D9F000759FFF1F789FFF1F749FFF1F7C9FFF1F56
:10DA00000C9FFF1F21282FD8184B195CFF292BD002
:10DA1000174B184ADFF870C003EBC000F0B543683D
:10DA2000DFF868E0144F154D154E00241C60DEF839
:10DA30000030012043F020038840CEF8003014600D
:10DA40004FF4A07338602E60C2F800C0013BFDD1D6
:10DA500013689B05FCD42023013BFDD1094B09B27F
:10DA600033F8110080B2F0BD002070475C3E010029
:10DA70004C3D010000500440085004400450044054
:10DA8000000002030051044080014A003880044035
:10DA9000431E032B14D872B60A4951F8230068B10B
:10DAA00070B4094C058834F81320466841F82360A7
:10DAB000521B24F8132062B670BC704762B67047E0
:10DAC00000207047D89FFF1F1CA2FF1F01380328AA
:10DAD0000BD872B6074B53F8203043B100205B6877
:10DAE0000130002BFBD162B670470020704718460A
:10DAF000F9E700BF2CA0FF1F30B472B62B4A137891
:10DB00001D0706D52A4B196A002936D0996A0029C3
:10DB100041D053781C0706D5254B196C00293ED0FF
:10DB2000996C002939D09378190705D5204B196EC7
:10DB3000002936D0996E89B1D3781B0707D51C4BC5
:10DB4000D3F880207AB3D3F8882011213AB162B695
:10DB5000184B00221A7030BC00F04ABE0D21154C43
:10DB6000154D227843F8315003EBC1030830013AD8
:10DB70005860227062B630BC704704220D4C0F4DC5
:10DB8000217843F8325003EBC20308304A1E586034
:10DB9000227062B6EFE70521E1E70921DFE70822FD
:10DBA000ECE70C22EAE71022E8E700BF803E010024
:10DBB0000080FF1F55A0FF1FC800400088004000E4
:10DBC000431E032B1DD81B4A400140F0100030B407
:10DBD000104472B6184CE25C032A1BD8DFE802F04E
:10DBE0000212151703220D88E25410F0080F14BF1B
:10DBF000C823882343EA054308310360416062B6C5
:10DC000030BC704708300222EDE70522EBE7083010
:10DC10000422E8E7094A52F8230038B1084A52F8CA
:10DC20002300416042F8231062B6E9E742F823106E
:10DC3000034AF7E70080FF1F64A0FF1F2CA0FF1F0F
:10DC40003CA0FF1F00BE70472DE9F04FDFF818B36E
:10DC5000DFF818A387B044E0AD4F4FEA930807EB15
:10DC6000C809013ED9F8042003F00803F6B2A2F176
:10DC7000080003F0FF04002B40F0018157F8383012
:10DC80001B0C99B222F8081C002B00F0EF80A14B6E
:10DC900022F8064C42F8044C53F82620002A00F0E3
:10DCA000CF819D4D55F8263058609C4C45F8260094
:10DCB00034F81630194424F8161000F079FD0028C5
:10DCC00000F0C281964A974B19F0080F00F1080046
:10DCD00018BF1346C9F8040047F8383008238BF8FA
:10DCE00000309BF80040E4B265071CD58E4B1B78D2
:10DCF000B3B18E490A7802F0FF0322B1013BDBB2D7
:10DD00000B7003B900BE8A490A7802F0FF032AB1FA
:10DD1000013BDBB20B70002B00F0688100F066FE67
:10DD200004238BF8003004F0080303F0FF02002BFB
:10DD300000F0C9809AF80030DBB21E098CD19A0835
:10DD4000DFF8CC9159F8321009EBC200C1F383011E
:10DD5000013940680C2900F28580DFE801F07A7A09
:10DD60008383838383834683838307000168714DA4
:10DD70004068714F714E6860296088B240F28161DD
:10DD80000024674B49F832304FF0010E88423C6066
:10DD9000C9F81040C9F8184086F800E05C4A00F263
:10DDA000E780B0F5D06F80F01B82B0F5817F00F086
:10DDB000D98100F26981802800F02A82822840F00F
:10DDC000D781A98801F07F01042900F2D1815C4844
:10DDD0005C4A890008441470547001788C0740F143
:10DDE000608382F800E0022173E1534F3A682AB35E
:10DDF000554B524E554819883478057840298E463F
:10DE000045F0020828BF4FF0400E002C84F00104BA
:10DE10003470CEEB01010CBF8824C82409EBC8067E
:10DE200089B285F0010544EA0E447260198049F810
:10DE3000384072440570002965D03A603D4B1A881D
:10DE4000B2F5A06F0ED100219A785970404B1A702C
:10DE500008E038493F4C0D68A54200F098803049F1
:10DE600049F832103C4A0123137037E72C4A2D4BF6
:10DE700019F0080F18BF134647F838302EE700F0A6
:10DE8000B7FC364A364952F82630002B00F0E380C2
:10DE900058688C5D42F8260003F10802C9F8042096
:10DEA000032C05D8DFE804F02C02292602228A552B
:10DEB0001A8819F0080F0CBF8823C82343EA0243CD
:10DEC00047F838300AE7E00700F19380210600F1B7
:10DED000D180A20706D5234A234913780220DBB25A
:10DEE00013700870E30602D51F4B10221A7007B09A
:10DEF000BDE8F08F04228A55DAE705228A55D7E774
:10DF000003228A55D4E7BEF1400F18BF002294E7E0
:10DF10000080FF1FD89FFF1F849FFF1F1CA2FF1FB1
:10DF2000C80040008800400060A0FF1FE99FFF1F5D
:10DF3000D4A0FF1F4CA0FF1F809FFF1FE89FFF1F63
:10DF4000C020074058A0FF1F949FFF1F54A0FF1F31
:10DF50009820074021090003942007402CA0FF1FB0
:10DF600064A0FF1F882007408020074090200740C2
:10DF7000B0F5106F00F07C8140F2A38040F62112D2
:10DF8000904240F07B82A54A012313706AE74C68F7
:10DF9000A3498C427FF463AF0178A9297FF45FAF76
:10DFA000417845297FF45BAF8178C2297FF457AF70
:10DFB000C1786B297FF453AF9A489B4E017834782F
:10DFC00081F00105002C41F0020105700CBF882092
:10DFD000C82084F0010449F8310009EBC1019348DD
:10DFE0003470002505244D60047038E700F064FFAC
:10DFF00094E68F4B89488B491A614FF0020E80F8E6
:10E0000000E08C4F0A708C49196099608B4E8C4DE2
:10E010008C4C9A610D213970FF213170DFF84CE290
:10E0200029702270884D894A8EF800109F2701249C
:10E0300006F8047C5D600470DA6007B0BDE8F08F1C
:10E0400043F82600824D30E6824A47F838001378BC
:10E050000133137042E68B5D032B00F2BA8001A2FC
:10E0600052F823F0DDDC0000DDDC0000BDE0000044
:10E07000B7E000006F49724B80220D2008701A70C3
:10E08000A2077FF52FAF26E740F20232904240F020
:10E09000ED81AA8802F07F02042A69D86D88002DDC
:10E0A00066D16449CDF804E0920011440A7842F048
:10E0B00002020A70C1E101238B550FE600238B5544
:10E0C0000CE6B0F5086F53D16349644A09781170C2
:10E0D0007146ED888D4280F0E88252480478402DE8
:10E0E000AE4644F0020C28BF4FF0400E02EB0E0388
:10E0F00009EBCC01029301234A604FEA0E48CEEBB4
:10E10000050101930025C82242EA080384F00102B8
:10E1100049F83C3035700270DFF814C1424BDFF82B
:10E12000048149BBBEF1400F7FF42DAF42F0020CD9
:10E1300009EBCC03029ADFF8F8E05A608DBB0D04BE
:10E1400045F088059DF804304EF83C500A44337081
:10E150000470134640297FF416AF0021404A3B600B
:10E16000118010E7AA8802F07F02042A40F28B8116
:10E17000304A0F23137006E74029D7D942F0020234
:10E180000CEBC200029E4660BDB19DF804503548BC
:10E190001D703346403988F8004040334CF8320057
:10E1A000DCE79DF8043033700D04029B047045F0E9
:10E1B000C8050B444EF83C50CCE79DF804501D7048
:10E1C000029B1D4888F80040403940334CF832002B
:10E1D000C4E719F0080F0CBF022303238B557DE51C
:10E1E00021494A68002AC3D06C88B5F804E003E0EE
:10E1F0000C314A68002ABBD00B88A342F8D14B8867
:10E200007345F5D1240A032C0CBF1178098960E706
:10E21000124A0221147054705BE700BF942007403B
:10E220000100040054A0FF1FE89FFF1FE99FFF1F8C
:10E230000080FF1FC0200740880040008820074062
:10E240008020074098200740989FFF1FEC9FFF1FEA
:10E25000849FFF1F55A0FF1F60A0FF1F58A0FF1F36
:10E26000949FFF1FC8004000843E01008C2007409F
:10E27000B248116AAC7804700C0600F19881D9F8A4
:10E280002820AF49100600F1DB81D9F83020AC49D5
:10E29000120600F1D081D9F83820A949130600F1FF
:10E2A000C581D9F84020A649150600F1BA81D9F8F0
:10E2B0004820A349140600F1AF81D9F85020A049A5
:10E2C000100600F1A481D9F858209D49120600F1EA
:10E2D0009981D9F860209A49130600F18E81D9F806
:10E2E00068209749150600F18381D9F87020944978
:10E2F000140600F17881D9F878209149100600F1D0
:10E300006D81D9F880208E49120600F16181D9F81B
:10E3100088208B49130600F15581D9F8902088494F
:10E32000150600F14981D9F898208549140600F1B5
:10E33000FF808448844A854901908548854D864CF4
:10E34000049700230596029580460F4616461D4603
:10E350000394306828B1446800F04AFA2046002C43
:10E36000F9D100233360029B38681A46002342F833
:10E37000253028B1446800F03BFA2046002CF9D142
:10E3800000223A60019A98F800301146002241F8C4
:10E39000042B039A0191023B4FF0000122F8151063
:10E3A000032B07D8DFE803F05D025D024FF00103A5
:10E3B00088F800300135042D06F1040607F1040742
:10E3C00008F10108C5D1654C654D2278654B049F65
:10E3D000059E0021100729701A7000F19280624991
:10E3E00062780A700021C9F83010C9F83810110796
:10E3F000DFF84C816ED4A2785C49DFF844810A7062
:10E4000000211207C9F85010C9F858104BD4E2780F
:10E4100057494B4C0A7013074FF00001C9F87010B0
:10E42000C9F8781000F1AE8033780193002283F0B0
:10E430000105C9F89020C9F898200021029188466A
:10E440008E460A464B48047844F0020C09EBCC0394
:10E450000393019B002B039B5A600CBF8822C822A8
:10E4600052E64FF0000388F80030A3E7B0F5A06F44
:10E470007FF47EAE012300250193DEE740F62122E2
:10E480009042F7D074E66D88002D7FF471AE3A4962
:10E49000CDF804E0920011440A7822F002020A70DA
:10E4A000CBE7022115E600F083F9002800F0EB80AD
:10E4B0000830324AC8F86400C8F8602000F078F9E3
:10E4C000002800F0DA8008302D4AC9F86C00C9F83D
:10E4D00068209CE700F06CF9002800F0E08008302C
:10E4E000264AC8F84400C8F8402000F061F9002826
:10E4F00000F0CF800830224AC9F84C00C9F8482003
:10E5000079E700F055F9002800F0A58008301B4A93
:10E51000C9F82400C9F8202000F04AF9002800F0CA
:10E5200094800830164AC9F82C00C9F8282056E70C
:10E53000D1F89C00083800F05BF9FAE660A0FF1FF4
:10E540000080FF1F3CA0FF1FD89FFF1F2CA0FF1FB4
:10E5500064A0FF1F849FFF1F1CA2FF1F803E0100BD
:10E5600055A0FF1FC4200740C8200740CC2007400B
:10E57000D020074054A0FF1FC02007408800400063
:10E58000C800400000F014F9002870D008304F4A4D
:10E59000C4F88400C4F8802000F00AF9002860D094
:10E5A00008304B4AC9F88C00C9F888203CE7506A0B
:10E5B000083800F01DF962E6D1F89400083800F040
:10E5C00017F9B0E6D1F88C00083800F011F9A4E68C
:10E5D000D1F88400083800F00BF998E6C86F0838C5
:10E5E00000F006F98DE6486F083800F001F982E680
:10E5F000C86E083800F0FCF877E6486E083800F07E
:10E60000F7F86CE6C86D083800F0F2F861E6486D7E
:10E61000083800F0EDF856E6C86C083800F0E8F865
:10E620004BE6486C083800F0E3F840E6C86B083861
:10E6300000F0DEF835E6486B083800F0D9F82AE635
:10E64000C86A083800F0D4F81FE62A78C9F828000C
:10E6500001322A70C3E62A78C9F8200001322A70F4
:10E660005AE72A78C9F8880001322A70DCE62A784D
:10E67000C4F8800001322A708EE72A78C9F8680051
:10E6800001322A70C3E62A78C8F8600001322A7085
:10E6900014E72A78C9F8480001322A70ABE62A78D4
:10E6A000C8F8400001322A701FE740298E4628BF73
:10E6B0004FF0400E02EB0E0302930123CEEB01015B
:10E6C0004FEA0E4800250193BCE600BF88004000D9
:10E6D000C8004000F8B500F08FFD294B29482A4CAE
:10E6E0002A4F2B4DDFF8BCC0DFF8BCE0294E0022DA
:10E6F0001A605A609A60DA601A615A619A61DA6146
:10E700001A625A629A62DA621A635A639A63DA6325
:10E710001A645A649A64DA641A655A659A65DA6505
:10E720001A665A669A66DA661A675A679A67DA67E5
:10E73000C3F880200168C3F8842041F4802101607F
:10E74000C3F307212170C3F30740134938701B0E30
:10E750002B70FF238CF80030104D8EF800301048DD
:10E760000B700123337084F8642070264FF400741A
:10E77000102207F82C3C2E70046081F8F820F8BDB8
:10E780000080FF1F348004409C200740B0200740D9
:10E79000B4200740942007401020074049E400E0DF
:10E7A00008E100E08020074088200740704700BF54
:10E7B00072B60D480268B2FA82F30F2B10DC4FF0EC
:10E7C0000041D94022EA0102026062B6074803EB29
:10E7D000C303DB00C2180021C150104651607047CE
:10E7E00062B60020704700BF3C92FF1FBC83FF1F32
:10E7F0000D4B0E4AC31AA2FB03231B090F2B0CD887
:10E800000B4A127852B972B60A484FF000410268BA
:10E8100021FA03F31A43026062B67047064A12787F
:10E82000002AF0D0FFF768B9BC83FF1F398EE338A8
:10E8300055A0FF1F3C92FF1F60A0FF1F38B50E4B75
:10E840000E4C1B68218805468BB1B1F5917F05D22E
:10E850000B4A4B1C55549BB2238038BD00220848FC
:10E8600098470021064A55540123238038BDB1F54D
:10E87000917FEDD338BD00BF8CA0FF1F26A2FF1FE4
:10E880002CA2FF1F2DE9F843214E224F31680123AE
:10E8900080463B70B1B1204D4B8801EB83020133C0
:10E8A00000240F2BC2F808802C7004D84B80002362
:10E8B0003B70BDE8F88340230B800320FFF780F90D
:10E8C0003460F4E7DFF8549099F80030002BF0D072
:10E8D000114D45F6215408E0013C12D02B7883B944
:10E8E00000F00AFB99F800307BB10320FFF7EEF847
:10E8F0000528F1D8FFF75CFF014630600028EBD017
:10E90000CAE701232B70BDE8F883BDE8F88300BF98
:10E91000A8A0FF1F7CA0FF1FACA0FF1F60A0FF1FCF
:10E920001201F8B5D5B2A1B3012943D0437804460A
:10E9300000781B0643EA004040F4704045F00406AE
:10E940008F1E3043FFF79EFF022F04F1020314D9FC
:10E95000053414F8023C14F8032C14F8010C1B04C1
:10E9600043EA0223334343EA0060033FFFF78AFF91
:10E97000022F234604F10304EBD8022F23D0012FEA
:10E980000DD045F4774040F00500BDE8F840FFF7B2
:10E9900079BF14482843BDE8F840FFF773BF1878E3
:10E9A00045F4770545F0060545EA0020BDE8F84046
:10E9B000FFF768BF03780C4845EA03452843BDE8E4
:10E9C000F840FFF75FBF1A78587845F0774545F073
:10E9D000070545EA022545EA0040BDE8F840FFF793
:10E9E00051BF00BF06F0F70007F000F738B5084B3D
:10E9F0001C7824B9074D296809B14B8803B938BD83
:10EA00009B000B800320FFF7DBF82C6038BD00BFB4
:10EA10007CA0FF1FA8A0FF1F2DE9F041AD4E336879
:10EA20000746002B00F092801D885A88910803EB5E
:10EA300081010432AA428C6842D25A8004F00F0647
:10EA40004FEA1428A449A6F1080208F00F00C4F305
:10EA50000313062A00F101050B701AD9B31E012B0E
:10EA60005FFA88F04ED9052E48D0042E00F0A4811C
:10EA7000731F022B7FD90F2E0ED1F72842D8F02812
:10EA800002D0964B1B883BB1FFF7D8FE0020BDE8B3
:10EA9000F08127B1BD4202D00020BDE8F081082EF0
:10EAA000C4F3033300F08780092E11D00A2E40F002
:10EAB00094800A2BF0D18A4B8A4A1B68A02181E0FE
:10EAC0001846FFF795FE0420FEF7E2FF3060B5E739
:10EAD000092BE1D1270E00F07B81834B814A1B6813
:10EAE0009021C4F307461170EDB2FCB2002B00F088
:10EAF0009D80224631462846984797E0F02843D922
:10EB0000F72841D0F1380E28C6D801A353F820F0D9
:10EB1000C7EC0000ABEC000099EC000099EA0000A3
:10EB200099EA00008BEC000099EA00006BED000010
:10EB300099EA000035ED00004FED000073EC000095
:10EB400099EA00005BEC00003FEC0000674B1B788B
:10EB5000002BA1D00420FEF79BFF03463060002865
:10EB60009AD00588002D7FF460AFFFF741FE356035
:10EB70002846BDE8F081FFF761FEC4F30740FFF7C8
:10EB80005DFE072E02D1200EFFF758FE534B584A68
:10EB9000198858481468584D524A017000270E0AC7
:10EBA000F0201F802E7010700CB301225348A04734
:10EBB0000120BDE8F081082B7FF46EAF504B494A2D
:10EBC0001B688021C4F307461170EDB2240E6BB3AD
:10EBD000284622463146984728E00B2E11D10B2BB0
:10EBE0007FF45AAF474B3F4A1B68B021EAE7464BD8
:10EBF0001B68002B00F0FB80404898470120BDE8CF
:10EC0000F0810C2E40F000810C2B7FF445AF3F4B80
:10EC1000344A1B68C0211170EDB2C4F30746002BC3
:10EC200000F0C88028463146240E98473849314ABA
:10EC3000314B0D7016701C700120BDE8F081354B12
:10EC40001B68002B00F0D6809847C4F30746254B7D
:10EC5000EDB2240E83F80080E8E72F4B1B68002BF1
:10EC6000F2D12E4B1B68A3B1FE209847C4F3074690
:10EC7000EDE72B4B1B68002BE6D1284B1B6843B1FB
:10EC8000FC209847C4F30746E1E7264B1B68002B9E
:10EC9000DAD1C4F30746DAE7234B1B68C4F307460F
:10ECA000002BD4D030469847D1E7204B1A68002A71
:10ECB000EFD0260C630C06F07F0003F47E5318435C
:10ECC000F6B29047C3E71A4B1B68C4F30746002B04
:10ECD000E8D1BCE7B4A0FF1F2AA2FF1F26A2FF1F96
:10ECE00090A0FF1F24A2FF1FC4A0FF1F60A0FF1F52
:10ECF0008CA0FF1F28A2FF1F29A2FF1F2CA2FF1F0D
:10ED0000BCA0FF1FC0A0FF1FA4A0FF1F80A0FF1F6B
:10ED10002BA2FF1F6CA0FF1F70A0FF1F74A0FF1F7E
:10ED2000B0A0FF1FA0A0FF1FB8A0FF1F88A0FF1F5B
:10ED30009CA0FF1F3F4B1B68002B85D13E4B1B68DF
:10ED4000002BA6D0FA209847C4F307467FE73B4B39
:10ED50001B68002B7FF478AF374B1B68002B98D0D3
:10ED6000FB209847C4F3074671E7354B1B68002B1F
:10ED70007FF46AAF304B1B68002B8AD0F82098478D
:10ED8000C4F3074663E70E2B7FF486AE2D4A2E4B65
:10ED90001268E0211970002A47D0260C610C06F099
:10EDA0007F0301F47E511943EDB2A1F500512846CD
:10EDB0009047F6B2240E39E7FFF740FDC4F3074051
:10EDC000FFF73CFD200EFFF739FD0020BDE8F08184
:10EDD0001E4B1D4A1B6880211170EDB2C4F307461B
:10EDE00083B1314628463A4698473C461EE7012003
:10EDF000BDE8F081104B1B68002B3FF44AAFFF20A9
:10EE0000984746E71C4611E70D2EBCD10D2B7FF429
:10EE100043AE0F4B0C4A1B68D0211170EDB2C4F306
:10EE20000746002B7FF4FEAEC4E7C4F30746EDB2FD
:10EE3000240EFBE698A0FF1F74A0FF1F78A0FF1F01
:10EE400068A0FF1F84A0FF1F24A2FF1FBCA0FF1FFC
:10EE500094A0FF1F38B5164D2868E0B1018844889A
:10EE6000A14213DD03191B7A83B104F10803C21810
:10EE70000C1B002302E012F8011F21B10133A34251
:10EE8000F9D1204638BD1C46204638BDFFF7B0FCFE
:10EE90000020286038BD074B1B780BB9002038BD17
:10EEA0000220FEF7F5FD28600028D7D1F6E700BF65
:10EEB000D0A0FF1F60A0FF1F0D4B1B78BBB910B582
:10EEC0000C4C216803F0FF024B883F2B07DC073313
:10EED0000B4401F1470003F8012F8342FBD140238B
:10EEE0000B800120FEF76CFE0023236010BD7047ED
:10EEF000C8A0FF1FCCA0FF1F38B5224C237803B158
:10EF000038BD01232370FFF7A5FF70BB00F048F860
:10EF100040BB00F0DBF810BBFEF7F8FCE0B90023C3
:10EF20002370EFF30583002BEAD1EFF3108172B663
:10EF3000154B1868E0B1154C2278CAB945691D60B7
:10EF400001232370C5B1AA6101B962B600254577D6
:10EF5000836898472570D3E700F020F8DFE700F0DA
:10EF60001BF8D9E700F016F8D3E7FFF71FFCCDE751
:10EF70000029C5D162B638BD054B1D600029E5D119
:10EF8000E3E700BFD5A0FF1FEC9EFF1FF09EFF1F11
:10EF9000E89EFF1F704700BF704700BF704700BF6B
:10EFA000054A064B10781B78C0B2DBB2984238BFD6
:10EFB0004030C01A704700BFDCA0FF1FDDA0FF1F5C
:10EFC000F0B4384B1A7912F0300F2CD072B6997D0C
:10EFD00001F0FF0200293DD062B6334F3349387843
:10EFE0000D78334E1C46C0B2EDB2431C402BE17984
:10EFF00028BF0023AB4202F1FF32C9B21CBFF1545B
:10F00000184612F0FF02F0D12A4B1B68C2B23A70C8
:10F010004BB1A84236BFC5F14005401B4019272817
:10F02000C4BF01221A701F49CA78D2B2150616D47D
:10F0300052060DD51B4B1B795B0609D51E4B1F498C
:10F040001B6800220A7003B11A70164B3C22DA705A
:10F05000F0BC70474022D9795A7462B6E3E70B7965
:10F060001C06E5D5164B174E1C783378E4B2DBB29C
:10F070009C420ED0144D01E0A3420AD00133402B34
:10F0800028BF00230879E85CC0B2C871087D072852
:10F09000F2D9DBB2034933700B79180644BF7C23E5
:10F0A000CB70C5E700A00640DCA0FF1FDDA0FF1F5E
:10F0B00020A1FF1FD8A0FF1F64A1FF1F60A1FF1F99
:10F0C00068A1FF1F61A1FF1FE0A0FF1F054A064BBB
:10F0D00010781B78C0B2DBB2984238BF4030C01AFB
:10F0E000704700BFDCA1FF1F71A1FF1FF0B4384BB8
:10F0F0001A7912F0300F2CD072B6997D01F0FF0210
:10F1000000293DD062B6334F334938780D78334EFD
:10F110001C46C0B2EDB2431C402BE17928BF00234E
:10F12000AB4202F1FF32C9B21CBFF154184612F0D3
:10F13000FF02F0D12A4B1B68C2B23A704BB1A84211
:10F1400036BFC5F14005401B40192728C4BF012226
:10F150001A701F49CA78D2B2150616D452060DD5B8
:10F160001B4B1B795B0609D51E4B1F491B680022F0
:10F170000A7003B11A70164B3C22DA70F0BC70476B
:10F180004022D9795A7462B6E3E70B791C06E5D5BB
:10F19000164B174E1C783378E4B2DBB29C420ED08B
:10F1A000144D01E0A3420AD00133282B28BF0023CD
:10F1B0000879E85CC0B2C871087D0728F2D9DBB2D3
:10F1C000034933700B79180644BF7C23CB70C5E725
:10F1D00000B00640DCA1FF1F71A1FF1F9CA1FF1F13
:10F1E0006CA1FF1FE0A1FF1F70A1FF1FE4A1FF1F83
:10F1F000DDA1FF1F74A1FF1F70B584B072B6194B5B
:10F20000194D1A48702241260F2480211A702E7041
:10F210001A460470197013781B06FCD5144B186835
:10F2200062B6144B144C984298BF00EB800001A9C1
:10F2300098BF40000A22FDF7CFFE01A92046002317
:10F2400011F8012B01333AB10A2B20F8022FF7D124
:10F250001623237004B070BD5B00DBB2237004B0D2
:10F2600070BD00BF000002400700024006000240DF
:10F27000080002407F9698000893FF1FFFFFFFFFE2
:10F280002DE9F043DFF8EC808BB006460F4600F026
:10F2900073F898F90030013304460D4637D03046F4
:10F2A000394600F0DFF9002831D02BA3D3E9002341
:10F2B0003046394600F026FE814668BB28A3D3E9D4
:10F2C00000233046394600F0FFFD00B398F90030C6
:10F2D000254ACDF82090042400200021022BCDE9FE
:10F2E0000467CDE9026700940192CDE906012CD0B4
:10F2F000684600F0BDF940B3089B1BB101F0AAF9C4
:10F30000089B0360DDE906010BB0BDE8F0832046F1
:10F3100029460BB0BDE8F083134A98F900300192FA
:10F3200003210022CDE90467CDE90267009108922C
:10F330002BB90E4B4FF06042CDE90623D8E70C49BC
:10F340000020022BCDE90601D2D101F083F922235E
:10F350000360D1E7AFF30080EF39FAFE422E86401A
:10F3600051302DD5104987C0F03E0100FFFFEF4717
:10F370000000F07F1E93FF1F2DE9F04FB04F21F0EA
:10F380000042BA4283B00C464FEAD17605460DD909
:10F39000AC4FBA4225D9C1F31303034340F0EF80C9
:10F3A0000EB10020014603B0BDE8F08FA64B9A4293
:10F3B00000F2CC80A54B9A4200F2DE808AA3D3E90A
:10F3C000002300F05DF90022A14B00F09BFD002816
:10F3D00000F005812846214600229D4B00F050F99F
:10F3E000E1E783A3D3E9002300F08CFD002840F07F
:10F3F000CB802846214680A3D3E9002300F064FD9A
:10F400000028CED1934B284603EBC60821467CA3A7
:10F41000D3E9002300F0E6FAD8E9002300F030F940
:10F4200000F07AFD804600F077FA77A3D3E9002355
:10F4300006460F4600F0D6FA02460B4628462146FD
:10F4400000F01CF972A3D3E90023CDE90001304696
:10F45000394600F0C7FA82468B4652465B46DDE9E4
:10F46000000100F00BF905460C462A4623462846C3
:10F47000214600F0B7FA68A3D3E9002306460F46F9
:10F4800000F0B0FA66A3D3E9002300F0F7F83246A3
:10F490003B4600F0A7FA64A3D3E9002300F0F0F89C
:10F4A00032463B4600F09EFA61A3D3E9002300F008
:10F4B000E5F832463B4600F095FA5FA3D3E9002316
:10F4C00000F0DEF832463B4600F08CFA02460B466E
:10F4D0002846214600F0D2F806460F462846214627
:10F4E00032463B46B8F1000F56D000F07BFA324668
:10F4F00004460D463B4600204FF0804100F0BEF828
:10F5000002460B462046294600F096FB02460B4673
:10F510005046594600F0B2F8DDE9002300F0AEF89D
:10F520000B4602464A49002000F0A8F86FF47F73AA
:10F5300098454FDA08F57A7801EB085100224FF030
:10F54000B87300F04FFA03B0BDE8F08F424B9A4217
:10F550003FF658AF414BF4002344D3E9002300F0B9
:10F560008DF83F4BC6F101081C44CDE90001D4E9F8
:10F5700000ABC6EB080870E74FF0000875E70246DD
:10F580000B4600F07DF80EE717A3D3E900231046E1
:10F59000194600F027FA06E700F024FA0022804618
:10F5A00089464FF080433046394600F067F80246FE
:10F5B0000B464046494600F03FFB2A46234600F0F2
:10F5C0005DF802460B460020214900F057F803B0D1
:10F5D000BDE8F08F01EB085103B0BDE8F08F804625
:10F5E00043E700BFAFF300809C7500883CE4377EA2
:10F5F000EF39FAFE422E864051302DD5104987C092
:10F60000FE822B654715F73F0000E0FE422EE63FE5
:10F61000763C7935EF39EA3DD0A4BE726937663E53
:10F62000F16BD2C541BDBB3E2CDE25AF6A56113F02
:10F6300093BDBE166CC1663F3E5555555555C53FE9
:10F64000412E8640FFFFEF7F422ED63FFFFF2F3E29
:10F650000000F03FF83E0100B1A2F03F183F01006A
:10F66000083F010041F0004101F58010C00F7047D4
:10F670000020704781F0004102E000BF83F00043AA
:10F6800030B54FEA41044FEA430594EA050F08BF3D
:10F6900090EA020F1FBF54EA000C55EA020C7FEA01
:10F6A000645C7FEA655C00F0E2804FEA5454D4EB7E
:10F6B0005555B8BF6D420CDD2C4480EA020281EA48
:10F6C000030382EA000083EA010180EA020281EA80
:10F6D0000303362D88BF30BD11F0004F4FEA0131D2
:10F6E0004FF4801C4CEA113102D0404261EB4101E1
:10F6F00013F0004F4FEA03334CEA133302D0524267
:10F7000063EB430394EA050F00F0A780A4F1010422
:10F71000D5F1200E0DDB02FA0EFC22FA05F280185C
:10F7200041F1000103FA0EF2801843FA05F3594142
:10F730000EE0A5F120050EF1200E012A03FA0EFCC1
:10F7400028BF4CF0020C43FA05F3C01851EBE371EB
:10F7500001F0004507D54FF0000EDCF1000C7EEB08
:10F7600000006EEB0101B1F5801F1BD3B1F5001F46
:10F770000CD349085FEA30004FEA3C0C04F1010465
:10F780004FEA445212F5800F80F09A80BCF1004F8E
:10F7900008BF5FEA500C50F1000041EB045141EA10
:10F7A000050130BD5FEA4C0C404141EB010111F411
:10F7B000801FA4F10104E9D191F0000F04BF0146BC
:10F7C0000020B1FA81F308BF2033A3F10B03B3F19A
:10F7D00020020CDA0C3208DD02F1140CC2F10C022A
:10F7E00001FA0CF021FA02F10CE002F11402D8BF88
:10F7F000C2F1200C01FA02F120FA0CFCDCBF41EA54
:10F800000C019040E41AA2BF01EB0451294330BD22
:10F810006FEA04041F3C1CDA0C340EDC04F11404FF
:10F82000C4F1200220FA04F001FA02F340EA0300D6
:10F8300021FA04F345EA030130BDC4F10C04C4F11C
:10F84000200220FA02F001FA04F340EA03002946FC
:10F8500030BD21FA04F0294630BD94F0000F83F446
:10F86000801306BF81F480110134013D4EE77FEA29
:10F87000645C18BF7FEA655C29D094EA050F08BF75
:10F8800090EA020F05D054EA000C04BF1946104656
:10F8900030BD91EA030F1EBF0021002030BD5FEA9A
:10F8A000545C05D14000494128BF41F0004130BDC2
:10F8B00014F580043CBF01F5801130BD01F0004516
:10F8C00045F0FE4141F470014FF0000030BD7FEA89
:10F8D000645C1ABF194610467FEA655C1CBF0B4684
:10F8E000024650EA013406BF52EA033591EA030F9B
:10F8F00041F4002130BD00BF90F0000F04BF002193
:10F90000704730B54FF4806404F132044FF00005C5
:10F910004FF0000150E700BF90F0000F04BF00213E
:10F92000704730B54FF4806404F1320410F00045A4
:10F9300048BF40424FF000013EE700BF42004FEA9F
:10F94000E2014FEA31014FEA02701FBF12F07F431C
:10F9500093F07F4F81F06051704792F0000F14BF19
:10F9600093F07F4F704730B54FF4607401F000455D
:10F9700021F0004120E700BF50EA010208BF7047B4
:10F9800030B54FF000050AE050EA010208BF7047A9
:10F9900030B511F0004502D5404261EB41014FF412
:10F9A000806404F132045FEA915C3FF4DCAE4FF016
:10F9B00003025FEADC0C18BF03325FEADC0C18BFFD
:10F9C000033202EBDC02C2F1200300FA03FC20FA4E
:10F9D00002F001FA03FE40EA0E0021FA02F114449B
:10F9E000C1E600BF70B54FF0FF0C4CF4E06C1CEAB0
:10F9F00011541DBF1CEA135594EA0C0F95EA0C0F25
:10FA000000F0DEF82C4481EA030621EA4C5123EA97
:10FA10004C5350EA013518BF52EA033541F48011C6
:10FA200043F4801338D0A0FB02CE4FF00005E1FB79
:10FA300002E506F00042E0FB03E54FF00006E1FBC3
:10FA400003569CF0000F18BF4EF0010EA4F1FF0406
:10FA5000B6F5007F64F5407404D25FEA4E0E6D4146
:10FA600046EB060642EAC62141EA55514FEAC52057
:10FA700040EA5E504FEACE2EB4F1FD0C88BFBCF5D3
:10FA8000E06F1ED8BEF1004F08BF5FEA500E50F184
:10FA9000000041EB045170BD06F0004646EA01014A
:10FAA00040EA020081EA0301B4EB5C04C2BFD4EB7C
:10FAB0000C0541EA045170BD41F480114FF0000E75
:10FAC000013C00F3AB8014F1360FDEBF002001F0E3
:10FAD000004170BDC4F10004203C35DA0C341BDC5D
:10FAE00004F11404C4F1200500FA05F320FA04F02F
:10FAF00001FA05F240EA020001F0004221F0004163
:10FB000010EBD37021FA04F642EB06015EEA430ED5
:10FB100008BF20EAD37070BDC4F10C04C4F1200505
:10FB200000FA04F320FA05F001FA04F240EA0200B8
:10FB300001F0004110EBD37041F100015EEA430E89
:10FB400008BF20EAD37070BDC4F1200500FA05F2A9
:10FB50004EEA020E20FA04F301FA05F243EA020328
:10FB600021FA04F001F0004121FA04F220EA020037
:10FB700000EBD3705EEA430E08BF20EAD37070BD7D
:10FB800094F0000F0FD101F00046400041EB01015D
:10FB900011F4801F08BF013CF7D041EA060195F03F
:10FBA000000F18BF704703F00046520043EB0303F9
:10FBB00013F4801F08BF013DF7D043EA06037047E6
:10FBC00094EA0C0F0CEA135518BF95EA0C0F0CD0F1
:10FBD00050EA410618BF52EA4306D1D181EA030137
:10FBE00001F000414FF0000070BD50EA410606BF31
:10FBF0001046194652EA430619D094EA0C0F02D176
:10FC000050EA013613D195EA0C0F05D152EA0336BA
:10FC10001CBF104619460AD181EA030101F00041D8
:10FC200041F0FE4141F470014FF0000070BD41F021
:10FC3000FE4141F4780170BD70B54FF0FF0C4CF4FB
:10FC4000E06C1CEA11541DBF1CEA135594EA0C0F1A
:10FC500095EA0C0F00F0A7F8A4EB050481EA030E67
:10FC600052EA03354FEA013100F088804FEA03334E
:10FC70004FF0805545EA131343EA12634FEA02221C
:10FC800045EA111545EA10654FEA00260EF00041DD
:10FC90009D4208BF964244F1FD0404F5407402D22F
:10FCA0005B084FEA3202B61A65EB03055B084FEAC0
:10FCB00032024FF480104FF4002CB6EB020E75EBBD
:10FCC000030E22BFB61A754640EA0C005B084FEAE5
:10FCD0003202B6EB020E75EB030E22BFB61A754662
:10FCE00040EA5C005B084FEA3202B6EB020E75EBAD
:10FCF000030E22BFB61A754640EA9C005B084FEA25
:10FD00003202B6EB020E75EB030E22BFB61A754631
:10FD100040EADC0055EA060E18D04FEA051545EA20
:10FD200016754FEA06164FEAC30343EA52734FEAC9
:10FD3000C2025FEA1C1CC0D111F4801F0BD141EA42
:10FD400000014FF000004FF0004CB6E711F4801FA7
:10FD500004BF01430020B4F1FD0C88BFBCF5E06F87
:10FD60003FF6AFAEB5EB030C04BFB6EB020C5FEA97
:10FD7000500C50F1000041EB045170BD0EF0004EEC
:10FD80004EEA113114EB5C04C2BFD4EB0C0541EA1E
:10FD9000045170BD41F480114FF0000E013C90E61B
:10FDA00045EA060E8DE60CEA135594EA0C0F08BFDF
:10FDB00095EA0C0F3FF43BAF94EA0C0F0AD150EADE
:10FDC00001347FF434AF95EA0C0F7FF425AF104671
:10FDD00019462CE795EA0C0F06D152EA03353FF499
:10FDE000FDAE1046194622E750EA410618BF52EA16
:10FDF00043067FF4C5AE50EA41047FF40DAF52EAEA
:10FE000043057FF4EBAE12E74FF0FF3C06E000BF86
:10FE10004FF0010C02E000BF4FF0010C4DF804CD93
:10FE20004FEA410C7FEA6C5C4FEA430C18BF7FEA53
:10FE30006C5C1BD001B050EA410C0CBF52EA430C81
:10FE400091EA030F02BF90EA020F0020704710F101
:10FE5000000F91EA030F58BF994208BF90422CBF90
:10FE6000D8176FEAE37040F0010070474FEA410C89
:10FE70007FEA6C5C02D150EA013C07D14FEA430CA7
:10FE80007FEA6C5CD6D152EA033CD3D05DF8040B18
:10FE9000704700BF8446104662468C46194663464A
:10FEA00000E000BF01B5FFF7B7FF002848BF10F121
:10FEB000000F01BD4DF808EDFFF7F4FF0CBF012066
:10FEC00000205DF808FB00BF4DF808EDFFF7EAFFE2
:10FED00034BF012000205DF808FB00BF4DF808ED9D
:10FEE000FFF7E0FF94BF012000205DF808FB00BF92
:10FEF0004DF808EDFFF7CEFF94BF012000205DF81C
:10FF000008FB00BF4DF808EDFFF7C4FF34BF012028
:10FF100000205DF808FB00BF4FEA410212F5001215
:10FF200015D211D56FF47873B3EB625212D94FEA40
:10FF3000C12343F0004343EA505311F0004F23FA2A
:10FF400002F018BF404270474FF00000704750EA7F
:10FF5000013005D111F0004008BF6FF0004070473C
:10FF60004FF00000704700BF4FEA4102B2F1E0439A
:10FF700024BFB3F5001CDCF1FE5C0DD901F0004C90
:10FF80004FEAC0024CEA5070B2F1004F40EB8300E0
:10FF900008BF20F00100704711F0804F21D113F10C
:10FFA0003872BCBF01F00040704741F480114FEA45
:10FFB0005252C2F11802C2F1200C10FA0CF320FACE
:10FFC00002F018BF40F001004FEAC1234FEAD323EB
:10FFD00003FA0CFC40EA0C0023FA02F34FEA430355
:10FFE000CCE77FEA625307D150EA01331EBF4FF0DE
:10FFF000FE4040F44000704701F0004040F0FE40F9
:020000021000EC
:1000000040F40000704700BF80F0004002E000BFF5
:1000100081F0004142001FBF5FEA410392EA030FF3
:100020007FEA226C7FEA236C6AD04FEA1262D2EB3D
:100030001363C1BFD218414048404140B8BF5B4242
:10004000192B88BF704710F0004F40F4000020F0DB
:100050007F4018BF404211F0004F41F4000121F0F1
:100060007F4118BF494292EA030F3FD0A2F101023B
:1000700041FA03FC10EB0C00C3F1200301FA03F179
:1000800000F0004302D5494260EB4000B0F5000F9C
:1000900013D3B0F1807F06D340084FEA310102F15B
:1000A0000102FE2A51D2B1F1004F40EBC25008BF0D
:1000B00020F0010040EA03007047490040EB0000D7
:1000C00010F4000FA2F10102EDD1B0FA80FCACF106
:1000D000080CB2EB0C0200FA0CF0AABF00EBC25005
:1000E00052421843BCBFD0401843704792F0000FF3
:1000F00081F4000106BF80F400000132013BB5E746
:100100004FEA41037FEA226C18BF7FEA236C21D0BB
:1001100092EA030F04D092F0000F08BF0846704720
:1001200090EA010F1CBF0020704712F07F4F04D1EE
:10013000400028BF40F00040704712F100723CBF01
:1001400000F50000704700F0004343F0FE4040F42B
:10015000000070477FEA226216BF08467FEA2363E9
:100160000146420206BF5FEA412390EA010F40F4D4
:10017000800070474FF0000304E000BF10F0004320
:1001800048BF40425FEA000C08BF704743F0964307
:1001900001464FF000001CE050EA010208BF704722
:1001A0004FF000030AE000BF50EA010208BF7047A9
:1001B00011F0004302D5404261EB41015FEA010CBE
:1001C00002BF84460146002043F0B64308BFA3F1B6
:1001D0008053A3F50003BCFA8CF2083AA3EBC25398
:1001E00010DB01FA02FC634400FA02FCC2F12002B7
:1001F000BCF1004F20FA02F243EB020008BF20F0EE
:100200000100704702F1200201FA02FCC2F1200253
:1002100050EA4C0021FA02F243EB020008BF20EA48
:10022000DC7070474FF0FF0C1CEAD0521EBF1CEA76
:10023000D15392EA0C0F93EA0C0F6FD01A4480EA64
:10024000010C400218BF5FEA41211ED04FF000634D
:1002500043EA501043EA5111A0FB01310CF0004079
:10026000B1F5000F3EBF490041EAD3715B0040EA9F
:10027000010062F17F02FD2A1DD8B3F1004F40EB6F
:10028000C25008BF20F00100704790F0000F0CF042
:10029000004C08BF49024CEA502040EA51207F3A06
:1002A000C2BFD2F1FF0340EAC250704740F40000E1
:1002B0004FF00003013A5DDC12F1190FDCBF00F0D2
:1002C00000407047C2F10002410021FA02F1C2F180
:1002D000200200FA02FC5FEA310040F1000053EA1C
:1002E0004C0308BF20EADC70704792F0000F00F06A
:1002F000004C02BF400010F4000F013AF9D040EA70
:100300000C0093F0000F01F0004C02BF490011F403
:10031000000F013BF9D041EA0C018FE70CEAD15301
:1003200092EA0C0F18BF93EA0C0F0AD030F0004C81
:1003300018BF31F0004CD8D180EA010000F0004035
:10034000704790F0000F17BF90F0004F084691F0F3
:10035000000F91F0004F14D092EA0C0F01D142022D
:100360000FD193EA0C0F03D14B0218BF084608D1F6
:1003700080EA010000F0004040F0FE4040F4000040
:10038000704740F0FE4040F4400070474FF0FF0CD3
:100390001CEAD0521EBF1CEAD15392EA0C0F93EA1A
:1003A0000C0F69D0A2EB030280EA010C49024FEA6C
:1003B000402037D04FF0805343EA111143EA101325
:1003C0000CF000408B4238BF5B0042F17D024FF4DD
:1003D000000C8B4224BF5B1A40EA0C00B3EB510FB8
:1003E00024BFA3EB510340EA5C00B3EB910F24BFA1
:1003F000A3EB910340EA9C00B3EBD10F24BFA3EB26
:10040000D10340EADC001B0118BF5FEA1C1CE0D1ED
:10041000FD2A3FF650AF8B4240EBC25008BF20F0A0
:10042000010070470CF0004C4CEA50207F32C2BFF4
:10043000D2F1FF0340EAC250704740F400004FF091
:100440000003013A37E792F0000F00F0004C02BFC2
:10045000400010F4000F013AF9D040EA0C0093F08C
:10046000000F01F0004C02BF490011F4000F013BE6
:10047000F9D041EA0C0195E70CEAD15392EA0C0F4E
:1004800008D142027FF47DAF93EA0C0F7FF470AF86
:10049000084676E793EA0C0F04D14B023FF44CAFC9
:1004A00008466EE730F0004C18BF31F0004CCAD15E
:1004B00030F000427FF45CAF31F000437FF43CAF9A
:1004C0005FE700BF4FF0FF3C06E000BF4FF0010CBC
:1004D00002E000BF4FF0010C4DF804CD4FEA40029E
:1004E0004FEA41037FEA226C18BF7FEA236C11D0E8
:1004F00001B052EA530C18BF90EA010F58BFB2EB9B
:10050000030088BFC81738BF6FEAE17018BF40F01A
:10051000010070477FEA226C02D15FEA402C05D1CE
:100520007FEA236CE4D15FEA412CE1D05DF8040B53
:10053000704700BF844608466146FFE70FB5FFF7E6
:10054000C9FF002848BF10F1000F0FBD4DF808ED9E
:10055000FFF7F4FF0CBF012000205DF808FB00BF8F
:100560004DF808EDFFF7EAFF34BF012000205DF8E9
:1005700008FB00BF4DF808EDFFF7E0FF94BF012036
:1005800000205DF808FB00BF4DF808EDFFF7D2FF33
:1005900094BF012000205DF808FB00BF4DF808ED76
:1005A000FFF7C8FF34BF012000205DF808FB00BF43
:1005B0004FEA4002B2F1FE4F0FD34FF09E03B3EB70
:1005C00012620DD94FEA002343F0004310F0004FB0
:1005D00023FA02F018BF404270474FF00000704706
:1005E00012F1610F01D1420205D110F0004008BFA5
:1005F0006FF0004070474FF00000704742000ED28D
:10060000B2F1FE4F0BD34FF09E03B3EB126209D44D
:100610004FEA002343F0004323FA02F070474FF003
:100620000000704712F1610F01D1420202D14FF078
:10063000FF3070474FF00000704700BF0B46014687
:10064000184600F001B800BF13460A4601460220D2
:1006500000F0A8BE014B1868704700BF4897FF1F05
:1006600070B50F4E0F4D761BB61018BF002405D085
:10067000013455F8043B9847A642F9D10A4E0B4D78
:10068000761B03F053FCB61018BF002406D00134CB
:1006900055F8043B9847A642F9D170BD70BD00BF24
:1006A000383F0100383F01004C3F0100383F010056
:1006B000024B0146186800F00BB800BF4897FF1FB7
:1006C000024B0146186800F031BF00BF4897FF1F7A
:1006D0002DE9F04F01F10B05162D83B0064640F2CF
:1006E0009F8035F0070500F1BF80A94200F2BC8071
:1006F00000F058FBB5F5FC7FC0F09C826B0A00F05F
:10070000BA80042B00F28381A80900F1390E4FEA68
:100710004E033830C44F07EB8303A3F108015C6834
:10072000A14207D1ACE0002A80F2AC80E468A1428B
:1007300000F0A680636823F003035A1B0F2AF2DD42
:10074000B9493C6901F1080E744500F0B381636852
:1007500023F003035A1B0F2A00F39981002AC1F8E2
:1007600014E0C1F810E080F29E80B3F5007F80F0C5
:100770006781DB0803F1010C01229B1002FA03F3ED
:100780004A6851F83C80C4F8088001EBCC091A4350
:10079000A9F10803E3604A6041F83C40C8F80C4006
:1007A000831001249C40944200F28A80144206D1B6
:1007B00020F003006400144200F10400FAD007EBBB
:1007C000C009CC468046DCF80C108C4507D173E19B
:1007D000002A80F28181C9688C4500F06D814B68E8
:1007E00023F003035A1B0F2AF2DD0C46D1F80CC08C
:1007F00054F8088F4B1945F001054D6042F0010196
:10080000C8F80CC03046CCF808807B613B61C3F867
:100810000CE0C3F808E059609A5000F0C5FA1FE0F8
:10082000102921D800F0BEFA1025062302207E4FA1
:1008300007EB8303A3F108025C68944200F0458152
:100840006368E168A56823F00303234430465A68CF
:10085000E96042F001028D605A6000F0A5FA0834A8
:10086000204603B0BDE8F08F00240C2320463360FF
:1008700003B0BDE8F08F80234FF0400E3F2049E7E2
:1008800070465DE72344E1685A68A56842F00102BA
:10089000E96030468D605A6000F086FA08342046E0
:1008A00003B0BDE8F08F234430465A6842F001029D
:1008B0005A6000F079FA0834204603B0BDE8F08FA2
:1008C000BC68636823F00308A84504D3C5EB08039C
:1008D0000F2B00F38C80554BDFF860911A68D9F824
:1008E000003001332A4404EB080A00F0608102F56D
:1008F00080520F3222F47F6222F00F0211463046FE
:10090000019200F04BFCB0F1FF3F8346019A00F0EA
:100910005881824500F2FC80454B1968DA45114444
:10092000196000F05381D9F80000DFF810E10130C0
:100930001BBFCAEB0B0A5144CEF800B019601BF084
:10094000070100F01781C1F10800C1F5805183440F
:1009500008315A44C2F30B02C2EB01094946304642
:10096000019300F01BFC431C019B00F03F81CBEB8B
:1009700000024A4442F001021968C7F808B049442D
:10098000BC42CBF804201960DFF8A49016D0B8F16F
:100990000F0F40F2FD806268A8F10C0323F00703FB
:1009A000E01802F001024FF0050E1A430F2B6260AF
:1009B000C0F804E0C0F808E000F21C811D4BBC68E0
:1009C0001A68914288BF19601B4B1A68914262688D
:1009D00088BF196022F003029542A2EB050301D8FB
:1009E0000F2B04DC304600F0DFF9002438E76219F1
:1009F00043F0010345F0010565603046BA6053607D
:100A000000F0D2F90834204603B0BDE8F08F142B73
:100A100071D9542B00F2A480280B00F16F0E4FEA1D
:100A20004E036E3076E600BF4C97FF1FF0A1FF1F0C
:100A3000F4A1FF1FECA1FF1FE8A1FF1F589BFF1FA0
:100A40005A0A042A5ED9142A00F2B38002F15C012A
:100A500049005B3207EB810C57F82110DFF8DC818D
:100A6000ACF1080C8C4500F088804A6822F0030243
:100A7000934202D289688C45F7D1D1F80CC07A68CC
:100A8000C4F80CC0A160CCF80840CC6088E66319BB
:100A900042F0010745F00105656030464B610B618E
:100AA000C3F80CE0C3F808E05F609A50083400F027
:100AB0007BF9D5E64A6873E608F1010818F0030FE0
:100AC0000CF1080C7FF47FAE30E0DC68A34208BF75
:100AD00002303FF435AEB3E60B440C465A68C968A1
:100AE00054F8085F42F001025A603046E9608D60B8
:100AF00000F05AF9B4E603F15C0E03F15B004FEA33
:100B00004E0307E69A0902F1390149003832A1E79C
:100B1000BC424A4B3FF400AF9C68626822F003027B
:100B20005AE759F80839994540F0828010F0030FD0
:100B300000F1FF30F5D17B6823EA04037B60640099
:100B40009C423FF6BDAE002C3FF4BAAE1C4240467C
:100B50007FF435AE64001C4200F10400FAD02EE6AA
:100B6000B3F5AA7F18D8E80B00F1780E4FEA4E03D0
:100B70007730CFE54FF48051EBE60121D8F804300F
:100B8000921001FA02F21A43C8F80420614677E78E
:100B90000123CBF8043025E740F25452934220D889
:100BA000A80C00F17D0E4FEA4E037C30B2E5103206
:100BB000A4E6542A26D81A0B02F16F0149006E32BE
:100BC00048E7BC68626822F0030205E7CAF30B003D
:100BD00000287FF4A8AE4244BB6842F001025A608C
:100BE000ECE6FE234FF07F0E7E2093E501224FF0CE
:100BF0000009C1E604F10801304600F097FCD9F87D
:100C00000010DBE6B2F5AA7F05D8DA0B02F1780115
:100C1000490077321EE740F254518A4205D89A0CB7
:100C200002F17D0149007C3214E7FE217E2211E7AA
:100C30007B6884E7E808431C5B00F8E54C97FF1FDE
:100C40008842F0B50DD98B1898420AD28118002A33
:100C500051D09A1A13F8014D01F8014D9342F9D180
:100C6000F0BD0F2A48D941EA00039B0746D100F1A5
:100C7000100401F11003154653F8106C44F8106C81
:100C800053F80C6C44F80C6C53F8086C44F8086C7E
:100C9000103D53F8046C44F8046C0F2D03F110035D
:100CA00004F11004E8D8A2F1100323F00F0302F0BE
:100CB0000F0E1033BEF1030F1944034421D91E1F38
:100CC0000D467446043C55F8047B46F8047F032C1B
:100CD000F8D8AEF1040424F003040434234421447E
:100CE00002F0030262B1013B0A4411F8014B03F820
:100CF000014F8A42F9D1F0BD0346F3E70346F2E71C
:100D0000F0BD7246EEE700BF70B4840746D0541EB3
:100D1000002A41D0CDB2034602E0621EE4B314467D
:100D200003F8015B9A07F8D1032C2ED9CDB245EA1E
:100D300005250F2C45EA054519D903F11002264671
:100D4000103E0F2E42F8105C42F80C5C42F8085C32
:100D500042F8045C02F11002F2D8A4F1100222F071
:100D60000F0204F00F041032032C13440DD91E4659
:100D70002246043A032A46F8045BFAD8221F22F0DE
:100D800003020432134404F003042CB1C9B21C441E
:100D900003F8011BA342FBD170BC70471446034605
:100DA000C2E700BF704700BF704700BF024B0A4652
:100DB0000146186800F002B84897FF1F2DE9F04F70
:100DC000174683B0002900F0C1800E46814607F126
:100DD0000B05FFF7E7FF56F804EC162D2EF0030481
:100DE000A6F1080840D810221546AF4241D89442D7
:100DF00075DAC94B996808EB04008842416800F035
:100E0000D98021F0010303445B68DB077DD51EF028
:100E1000010F35D039464846FFF75AFC0746E0B186
:100E200056F8043C23F001034344A0F108029A421F
:100E300000F04481221F242A00F23181132A00F29B
:100E400004810346324611681960516859609268FE
:100E50009A603146484600F069FB4846FFF7A4FF18
:100E6000384603B0BDE8F08F25F00705002D2A466F
:100E7000BBDA0C230020C9F8003003B0BDE8F08FC6
:100E800056F8083CC3EB080ADAF8043023F0030CE8
:100E900004EB0C039342BDDB5746DAF80C1057F80D
:100EA000080F221F242AC160886000F21781132ACC
:100EB00040F212813168CAF808107168CAF80C1043
:100EC0001B2A00F22B8108360AF1100231681160EA
:100ED00071685160B16891603E461C46D046631B04
:100EE0000F2B1DD8D8F8043003F0010323434444EA
:100EF000C8F80430636843F0010363604846FFF7B5
:100F000053FF304603B0BDE8F08F21F003012144C8
:100F1000914221DBC36882680C46D3609A60DEE7A9
:100F2000D8F8042008EB050102F00102154343F054
:100F300001020B44C8F804504A605A6842F00102AA
:100F400008315A60484600F0F1FAD7E7114603B07D
:100F5000BDE8F04FFFF7BCBB1EF0010F7FF45AAFA6
:100F600056F8083CC3EB080ADAF8043023F0030C07
:100F700001EB0C0E96458BDBC36882685746D36045
:100F80009A6057F8081FDAF80C30CB60221F242A29
:100F9000996000F29980132A62D93368CAF8083040
:100FA0007368CAF80C301B2A00F2A08008360AF1D8
:100FB000100356E021F0030BA34405F11000834514
:100FC00059DA1EF0010F7FF425AF56F8081CC1EB6B
:100FD000080ADAF8041021F0030CE34458453FF7FF
:100FE00057AF5746DAF80C1057F8080F221F242A7B
:100FF000C160886000F2B480132A40F2A580316895
:10100000CAF808107168CAF80C101B2A00F2AF80E9
:1010100008360AF110023168116071685160B168D8
:1010200091600AEB0501C5EB0B0242F001029960E9
:101030004A60DAF8043003F001031D434846CAF859
:101040000450FFF7B1FE38465CE73368036073680D
:1010500043601B2A27D800F1080306F10802F2E6D4
:101060003B4632681A6072685A60B2689A603E46BF
:101070007446D04633E708EB0501C5EB0B0B4BF08C
:10108000010299604A6056F8043C03F001031D43D5
:10109000484646F8045CFFF787FE304632E73146A3
:1010A000FFF7CEFDD5E6B3688360F368C360242AFA
:1010B00028D000F1100306F11002C4E650F8043CF9
:1010C00023F003031C440AE7314638467446D046F1
:1010D000FFF7B6FD3E4602E73A46F7E631463846A8
:1010E0001C46D046FFF7ACFD3E46F8E6B368CAF8AA
:1010F0001030F368CAF81430242A1BD010360AF1D5
:101100001803AEE7336903617369436106F118029E
:1011100000F1180397E600BF4C97FF1FB168CAF8AB
:101120001010F168CAF81410242A0FD010360AF1F2
:101130001802CBE63369CAF818307369CAF81C3054
:1011400018360AF120038CE73A4664E73269CAF898
:1011500018207269CAF81C2018360AF12002B5E678
:10116000314638460193FFF76BFD019B59E7B168A3
:10117000CAF81010F168CAF81410242A03D01036E7
:101180000AF1180247E73269CAF818207269CAF8EA
:101190001C2018360AF120023DE700BF38B5074C85
:1011A0000023054608462360FBF7E0FE431C00D001
:1011B00038BD2368002BFBD02B6038BD50A3FF1F28
:1011C00090F800F06DE9024520F007016FF0000C87
:1011D00010F0070491F820F040F049804FF000042F
:1011E0006FF00700D1E9002391F840F000F108000A
:1011F00082FA4CF2A4FA8CF283FA4CF3A2FA8CF342
:101200004BBBD1E9022382FA4CF200F10800A4FAA8
:101210008CF283FA4CF3A2FA8CF3E3B9D1E90423FC
:1012200082FA4CF200F10800A4FA8CF283FA4CF333
:10123000A2FA8CF37BB9D1E9062301F1200182FAED
:101240004CF200F10800A4FA8CF283FA4CF3A2FAF3
:101250008CF3002BC6D0002A04BF04301A4612BA01
:10126000B2FA82F2FDE8024500EBD2007047D1E904
:10127000002304F00305C4F100004FEAC50514F093
:10128000040F91F840F00CFA05F562EA05021CBF64
:1012900063EA050362464FF00004A9E7002A41D043
:1012A00040EA010313F00303F0B425D1032A23D944
:1012B00004680D68AC421FD1043A35D0A4F1013561
:1012C00025EA040414F0803F31D1071D0D1D0DE007
:1012D00057F8043B0E68A3F10134B34224EA030437
:1012E0000AD1043A20D014F0803F23D1032A2946A2
:1012F000384605F10405EBD803780C789C4202F1DE
:10130000FF320CD182B114B916E06AB17BB110F88A
:10131000013F11F8014FA34202F1FF32F5D0181B33
:10132000F0BC7047104670471046F0BC7047184636
:10133000F0BC70470020F3E72046F1E740EA0103E4
:101340009B0770B42BD1032A29D90C4603462146AA
:1013500054F8046BA6F1013525EA060515F0803F27
:1013600006D1043A032A43F8046B2146EFD8A2B110
:101370000C781C70013A013301313CB16AB111F8AB
:10138000014B03F8014B013A002CF7D12AB11A4462
:10139000002103F8011B9A42FBD170BC7047034641
:1013A000E5E700BF2DE9F047254C2568D5F8484111
:1013B0000646884692469946C4B360681F2817DCE3
:1013C000431C76B104EB80050122C5F888A0D4F84F
:1013D000881182401143022EC4F88811C5F8089183
:1013E0001ED00230636044F820800020BDE8F08702
:1013F000144B03B34FF4C870FFF75AF90446D0B149
:10140000D5F84831002780E88800C5F848413846BB
:101410000123C4F88871C4F88C71002EE1D0D1E7A3
:10142000D4F88C110A43C4F88C21DAE705F5A674C8
:10143000C5F84841C1E74FF0FF30BDE8F08700BF75
:10144000283F0100B1060100024B13B1024800F031
:1014500005B8704700000000691401000023014630
:101460001A461846FFF79EBF38B5074D074C2C1B90
:10147000A41005D0013C55F8043D9847002CF9D143
:10148000BDE8384002F062BD00000000000000002E
:10149000F8B5234F0C460646FFF784FCBB685D6831
:1014A00025F00305291B01F6EF7121F47F6121F07E
:1014B0000F01A1F58054B4F5805F07DB00213046B1
:1014C000FFF76CFEBB682B44984204D03046FFF710
:1014D0006BFC0020F8BD61423046FFF75FFE013033
:1014E0000DD0104BBA6819682D1B45F00105304628
:1014F000091B55601960FFF757FC0120F8BD00215A
:101500003046FFF74BFEBA68831A0F2BDEDD064C20
:101510000449246843F00103001B53600860D5E7C9
:101520004C97FF1FF4A1FF1F589BFF1F002945D0B8
:101530002DE9F0410D468046FFF734FC55F8047C58
:101540006A4927F00103A5F10804E2188E68506883
:10155000B24220F0030062D0FE0750600BD455F871
:10156000087CE41B01F1080EA56875453B446FD06B
:10157000E768EF60BD6015186D68ED0742D543F070
:1015800001026260E350B3F5007F18D2DB085A1CF9
:101590004D6851F83270A76001209B1000FA03F3E8
:1015A00001EBC2001D430838E0604D6041F8324055
:1015B000FC604046BDE8F041FFF7F6BB70475A0AB1
:1015C000042A53D89A0902F139077F0002F138053D
:1015D00001EB870051F827204449083890424DD04C
:1015E000516821F003018B4202D292689042F7D1F8
:1015F000D068E060A2608460D4604046BDE8F041FD
:10160000FFF7D2BB95683A4FBD4203443FD0D06844
:10161000E86043F0010285606260E350B3E7FF07D2
:10162000034407D455F8082CA41A1344A068E268B0
:10163000C26090602F4A126843F0010093426060DC
:101640008C60B6D32C4B40461968FFF721FFB0E7FA
:1016500011184968C90744D49168D268CA60034424
:1016600043F0010091606060E350A2E7142A17D8AC
:1016700002F15C077F0002F15B05A9E7AA104B6845
:10168000012505FA02F213434B600246B1E743F02D
:1016900001024C610C61E560A5606260E35088E77F
:1016A000542A06D81A0B02F16F077F0002F16E056B
:1016B0008EE7B2F5AA7F06D8DA0B02F178077F0031
:1016C00002F1770584E740F25450824206D89A0C22
:1016D00002F17D077F0002F17C0579E7FE277E2578
:1016E00076E743F001026260E35062E74C97FF1F28
:1016F0005497FF1F549BFF1FF0A1FF1F00007805A8
:101700003408540B800C3C0F5C12E015FA19141EBF
:101710006022AC265C2B0C30BC34023AFF3FFFFF4A
:1017200000000000070000000C0000001000000096
:1017300013000000180000001C0000000000000062
:10174000070000000C000000100000001300000063
:101750001600000018000000000000000700000054
:101760000C00000013000000180000001F00000023
:1017700024000000000000000C0000001800000021
:1017800024000000300000003C0000004800000081
:10179000FDFFFFFFFBFFFFFFF8FFFFFFFDFFFFFF68
:1017A000FBFFFFFFF8FFFFFFFDFFFFFFFAFFFFFF5B
:1017B000F7FFFFFFFDFFFFFFFBFFFFFFF7FFFFFF4F
:1017C000FCFFFFFFFBFFFFFFF7FFFFFFFDFFFFFF3A
:1017D000FAFFFFFFF7FFFFFFFDFFFFFFFBFFFFFF2C
:1017E000F8FFFFFFFDFFFFFFFBFFFFFFF8FFFFFF1D
:1017F000FDFFFFFFFAFFFFFFF7FFFFFFFCFFFFFF0B
:10180000FBFFFFFFF7FFFFFFFDFFFFFFFBFFFFFFFA
:10181000F7FFFFFFFDFFFFFFFAFFFFFFF7FFFFFFEF
:10182000FDFFFFFFFBFFFFFFF7FFFFFFFDFFFFFFD8
:10183000FBFFFFFFF7FFFFFFFDFFFFFFFAFFFFFFCB
:10184000F7FFFFFFFDFFFFFFFAFFFFFFF8FFFFFFBE
:10185000FDFFFFFFFAFFFFFFF7FFFFFFFDFFFFFFA9
:10186000FAFFFFFFF7FFFFFFFDFFFFFFFAFFFFFF9C
:10187000F8FFFFFFFDFFFFFFFAFFFFFFF8FFFFFF8D
:10188000FDFFFFFFFAFFFFFFF7FFFFFFFCFFFFFF7A
:10189000FBFFFFFFF7FFFFFFFDFFFFFFFAFFFFFF6B
:1018A000F7FFFFFFFDFFFFFFFAFFFFFFF7FFFFFF5F
:1018B000FEFFFFFFFBFFFFFFF8FFFFFFFEFFFFFF45
:1018C000FBFFFFFFF8FFFFFFFDFFFFFFFAFFFFFF3A
:1018D000F7FFFFFFFCFFFFFFFAFFFFFFF7FFFFFF30
:1018E000FCFFFFFFFAFFFFFFF7FFFFFFFDFFFFFF1A
:1018F000FAFFFFFFF7FFFFFFFDFFFFFFF9FFFFFF0D
:10190000F7FFFFFFFDFFFFFFF9FFFFFFF7FFFFFFFF
:10191000FDFFFFFFFAFFFFFFF7FFFFFFFDFFFFFFE8
:10192000FAFFFFFFF7FFFFFFFDFFFFFFFAFFFFFFDB
:10193000F6FFFFFFFDFFFFFFFAFFFFFFF7FFFFFFCF
:10194000FEFFFFFFFBFFFFFFF7FFFFFFFEFFFFFFB5
:10195000FBFFFFFFF7FFFFFFFDFFFFFFFAFFFFFFAA
:10196000F7FFFFFFFDFFFFFFFBFFFFFFF8FFFFFF9C
:10197000FDFFFFFFFBFFFFFFF8FFFFFFFDFFFFFF86
:10198000FAFFFFFFF7FFFFFFFCFFFFFFF9FFFFFF7D
:10199000F7FFFFFFFCFFFFFFF9FFFFFFF7FFFFFF70
:1019A000FDFFFFFFFAFFFFFFF7FFFFFFFDFFFFFF58
:1019B000FAFFFFFFF7FFFFFFFDFFFFFFF9FFFFFF4C
:1019C000F6FFFFFFFDFFFFFFFAFFFFFFF7FFFFFF3F
:1019D000A41F0100801F01005C1F0100381F0100CF
:1019E000141C0100D01A0100F41A0100181B010098
:1019F000F01B0100AC1A01007C1D0100FC16010067
:101A0000381C010000000000070000000C0000006E
:101A10001000000013000000180000001C0000006F
:101A200000000000070000000C0000001000000093
:101A30001300000016000000180000000000000065
:101A4000070000000C000000130000001800000058
:101A50001F00000024000000000000000C00000037
:101A60001800000024000000300000003C000000CE
:101A70004800000000000000FBFFFFFFF4FFFFFF35
:101A8000EFFFFFFFE8FFFFFFE3FFFFFFDCFFFFFFCC
:101A900000000000F4FFFFFFE8FFFFFFDCFFFFFF97
:101AA000D0FFFFFFC4FFFFFFB8FFFFFF0000580299
:101AB00046056608540BD80E5C127017FC21F82AF4
:101AC00070305834DC37663A8C3C803EFF3FFFFF75
:101AD0000000580246056608540BD80E5C12E0154B
:101AE000FA19141E6022AC265C2B0C30BC34023A6E
:101AF000FF3FFFFF0000900120031405D0075A0AA2
:101B0000AC0DCC10B4146A18E81C342180252A2BA3
:101B100070301437FF3FFFFF0000C800F40184035A
:101B2000140508072E091C0CD80EF811AE159619CD
:101B3000401F1C25F22B5834FF3FFFFFFBFFFFFF28
:101B4000F8FFFFFFF4FFFFFFFAFFFFFFF7FFFFFFC4
:101B5000F4FFFFFFFDFFFFFFF9FFFFFFF4FFFFFFB3
:101B6000FAFFFFFFF7FFFFFFF4FFFFFFFCFFFFFFA0
:101B7000F7FFFFFFF4FFFFFFFBFFFFFFF8FFFFFF93
:101B8000F4FFFFFFFDFFFFFFFAFFFFFFF4FFFFFF82
:101B9000FDFFFFFFF9FFFFFFF4FFFFFFFDFFFFFF6A
:101BA000F8FFFFFFF4FFFFFFFCFFFFFFF7FFFFFF62
:101BB000F4FFFFFFFBFFFFFFF8FFFFFFF4FFFFFF56
:101BC000FCFFFFFFF7FFFFFFF4FFFFFF4006780574
:101BD000B004E80384032003BC025802F40190011E
:101BE0002C01FA00C8009600640032001900FFFFC3
:101BF00000006400C8009001BC021A04DC059E07C6
:101C0000F609800CA00F2413A2174C1D5424442F56
